:020000040000FA
:060000000AEFB6F0120049
:0600080004EF08F01200F5
:060018000CEF08F01200DD
:061000000AEFB6F0120039
:0610080047EFB1F01200F9
:061018004AEFB1F01200E6
:06102A000300806C0100D0
:101030001F0F00001B0000006B6C0100AB000000E4
:1010400015000000686C01003A0F0000030000006A
:10105000D9CFE6FFDACFE6FFE1CFD9FFE2CFDAFF63
:10106000E652E652DE6ADD6ADECF00F0DDCF01F047
:10107000D890015004E6030E005C000E01580EE209
:10108000DECFE9FFDDCFEAFF840EE926020EEA2279
:10109000010EEF6EDF2A01E3DB2AE6D70F012B6B8F
:1010A00039EC9EF0BE0EE66E020EE66E16EC0FF008
:1010B000E552E552006E016A0050011001E089D04E
:1010C0002CCFE9FF2DCFEAFFBE0EEE6E020EED6EC5
:1010D0002CCFE9FF2DCFEAFF060EEB6A070EEB6A75
:1010E0002CCFE9FF2DCFEAFF080EEB6A090EEB6A61
:1010F0002CCFE9FF2DCFEAFF0A0EE926000EEA22E7
:10110000EE6AEE6AEE6AEE6A2CCFE9FF2DCFEAFFB7
:101110000E0EE926000EEA22EE6AEE6AEE6AEE6A2A
:101120002CCFE9FF2DCFEAFF170EE926000EEA22A9
:101130005C0EEF6E010EDE6EDD6ADECF00F0DDCFFD
:1011400001F0D890015004E60B0E005C000E01582F
:1011500019E22CCFE9FF2DCFEAFF170EE926000E8A
:10116000EA22E9CF00F0EACF01F0DE500024E96E78
:10117000DD500120EA6E200EEF6EDF2A010E01E342
:10118000DB2ADBD72CCFE9FF2DCFEAFF220EEB6A5B
:10119000230EEB6A2CCFE9FF2DCFEAFF260EE926BE
:1011A000000EEA22100EEE6EED6A2CCFE9FF2DCF75
:1011B000EAFF280EEB6A290EEB6A2CCFE9FF2DCF50
:1011C000EAFF2A0EEB6A2B0EEB6A010EF36EF46A4D
:1011D00003D0F36AF46A00D0E552E552E552E5CF58
:1011E000DAFFE7CFD9FF1200D9CFE6FFDACFE6FF6B
:1011F000E1CFD9FFE2CFDAFF0B0EE12402E3E16891
:10120000E652E16EFC0EDBCFE9FFFD0EDBCFEAFF1D
:10121000220EE926000EEA22040EEECFDBFF050EB9
:10122000EDCFDBFF0A0EF36E080EF3CFDBFFFC0EF3
:10123000DBCFE9FFFD0EDBCFEAFF280EE926000E2B
:10124000EA22EECF00F0EFCF01F0FC0EDBCFE9FF9A
:10125000FD0EDBCFEAFF2A0EE926000EEA2200C0CF
:10126000EEFF01C0EDFFFA0EDBCFE9FFFB0EDBCF97
:10127000EAFF260EE926000EEA22EECF00F0EFCFBD
:1012800001F0FF0E001A011A020E00C0DBFF030E70
:1012900001C0DBFFD950040FE96E000EDA20EA6EC0
:1012A000EE50ED1025E1010EE66ED950040FE66E0A
:1012B000000EDA20E66EFC0EDBCFE6FFFD0EDBCF84
:1012C000E6FFA0EC20F0026E050EE15C02E2E16AAE
:1012D000E552E16E0250F3CF00F0F4CF01F0005080
:1012E000011005E11C0EF36E080EF3CFDBFF28D0D2
:1012F000040EDB500F0B24E0010EE66ED950040FF4
:10130000E66E000EDA20E66EFC0EDBCFE6FFFD0E89
:10131000DBCFE6FFA0EC20F0026E050EE15C02E2FE
:10132000E16AE552E16E0250F3CF00F0F4CF01F034
:101330000050011005E11C0EF36E080EF3CFDBFF29
:10134000080EDBCF00F0016A00BE01681C0E001819
:1013500001E1015001E171D2080EDBCF00F0016A1A
:1013600000BE01680050011040E0D950040FE66E45
:10137000000EDA20E66EFC0EDBCFE6FFFD0EDBCFC3
:10138000E6FF63EC2CF0E552E552E552E552E76EDC
:10139000060EE7CFDBFFDB50006E016A020E00187D
:1013A00001E1015001E149D2060EDB50006E016AF5
:1013B0000050011001E032D2FC0EDBCFE9FFFD0E40
:1013C000DBCFEAFF260EE926000EEA22EECFDEFF93
:1013D000EDCFDDFF3F0EDE16DD6AF80EDB50006E4E
:1013E000016A010E001803E101D027D2015001E18A
:1013F000A5D0005001E1015001E00FD2D9CFE9FFA3
:10140000DACFEAFF080EEE1801E1ED500DE0DECF75
:1014100002F0DDCF03F0020E0216000E0316020EDC
:10142000021801E1035002E1000E01D0010E006E2E
:10143000016A0050011001E180D0080EDB6A6D0ED8
:10144000F36E090EF3CFDBFF070EDB6ADB50006E95
:10145000016AD890015004E60B0E005C000E0158A2
:101460006CE2FC0EDBCFE9FFFD0EDBCFEAFF170ECF
:10147000E926000EEA22E9CF02F0EACF03F0070ED8
:10148000DB500F010224E96E000E0320EA6EEFCF5D
:1014900000F0016A00BE0168090E00C0DBFFFA0E11
:1014A000DBCFE9FFFB0EDBCFEAFF170EE926000ECC
:1014B000EA22E9CF02F0EACF03F0070EDB50022464
:1014C000E96E000E0320EA6EEFCF00F0016A00BE65
:1014D00001680A0E00C0DBFF090EDBCFE6FFE66AFB
:1014E00030ECB5F0E552E552F3CF00F0F4CF01F067
:1014F00000C0E6FF01C0E6FF0A0EDBCFE6FFE66AAA
:1015000030ECB5F0E552E552E552E7CF01F0E55297
:10151000E7CF00F0F3CF02F0F4CF03F00250001851
:1015200002E10350011806E00A0EF36E080EF3CF35
:10153000DBFF03D0070EDB2A89D76FD1020EDBCF8A
:1015400004F0030EDBCF05F0DE500414026EDD5014
:101550000514036E0250031009E1D9CFE9FFDACF79
:10156000EAFF0F0EEE1801E1ED5002E1000E01D08E
:10157000010E006E016A0050011001E14DD1080E0C
:10158000DB6A6D0EF36E090EF3CFDBFFFA0EDBCFD5
:10159000E9FFFB0EDBCFEAFF170EE926000EEA2279
:1015A000EFCF00F0016A00BE01682A0E001801E1C9
:1015B000015001E182D0070EDB6ADB50006E016A48
:1015C000D890015004E6080E005C000E015875E248
:1015D000FC0EDBCFE9FFFD0EDBCFEAFF170EE9269D
:1015E000000EEA22E9CF02F0EACF03F0070EDB504B
:1015F0000F010224E96E000E0320EA6EEFCF00F027
:10160000016A00BE0168090E00C0DBFFFA0EDBCFE5
:10161000E9FFFB0EDBCFEAFF170EE926000EEA22F8
:10162000E9CF02F0EACF03F0070EDB500224E96EA7
:10163000000E0320EA6EEFCF00F0016A00BE0168E1
:101640000A0E00C0DBFFDB50006E016A2A0E001894
:1016500001E1015001E131D0090EDBCFE6FFE66A7E
:1016600030ECB5F0E552E552F3CF00F0F4CF01F0E5
:1016700000C0E6FF01C0E6FF0A0EDBCFE6FFE66A28
:1016800030ECB5F0E552E552E552E7CF01F0E55216
:10169000E7CF00F0F3CF02F0F4CF03F002500018D0
:1016A00002E10350011806E00A0EF36E080EF3CFB4
:1016B000DBFF03D0070EDB2A80D7FA0EDBCFE9FF72
:1016C000FB0EDBCFEAFF170EE926000EEA22080E1A
:1016D000E926000EEA22EFCF02F0036A02BE036899
:1016E0002A0E021801E1035009E0080EDBCF04F0D6
:1016F000056A04BE05680450051002E0000E01D022
:10170000010E006E016A0050011001E185D0080E43
:10171000F36E070EF3CFDBFFDB50006E016AD8904B
:10172000015004E60B0E005C000E015875E2FC0E41
:10173000DBCFE9FFFD0EDBCFEAFF170EE926000E37
:10174000EA22E9CF02F0EACF03F0070EDB500F01E7
:101750000224E96E000E0320EA6EEFCF00F0016A6A
:1017600000BE0168090E00C0DBFFFA0EDBCFE9FF07
:10177000FB0EDBCFEAFF170EE926000EEA22E9CFC7
:1017800002F0EACF03F0070EDB500224E96E000EF0
:101790000320EA6EEFCF00F0016A00BE01680A0E76
:1017A00000C0DBFFDB50006E016A2A0E001801E169
:1017B000015001E131D0090EDBCFE6FFE66A30ECE3
:1017C000B5F0E552E552F3CF00F0F4CF01F000C0E0
:1017D000E6FF01C0E6FF0A0EDBCFE6FFE66A30EC6B
:1017E000B5F0E552E552E552E7CF01F0E552E7CF1B
:1017F00000F0F3CF02F0F4CF03F00250001802E142
:101800000350011806E00A0EF36E080EF3CFDBFF5B
:1018100003D0070EDB2A80D700D009D0F90EDB50A9
:10182000006E016A0050011002E1080EDB6A040E2E
:10183000DB2A050E01E3DB2A8FD5080EDBCF00F093
:10184000016A00BE0168005000D0006E0B0EE15C22
:1018500002E2E16AE552E16E0050E552E5CFDAFFBF
:10186000E7CFD9FF1200D9CFE6FFDACFE6FFE1CF0D
:10187000D9FFE2CFDAFF080EE12402E3E168E65285
:10188000E16E070EDB6AFC0EDBCFE9FFFD0EDBCF5E
:10189000EAFFEECFDEFFEDCFDDFFDECFE9FFDDCFEC
:1018A000EAFF1D0EE926000EEA22EF50006E016AE3
:1018B0000050011006E1060EF36E070EF3CFDBFFBA
:1018C000A8D1FC0EDBCFE9FFFD0EDBCFEAFF280E2F
:1018D000E926000EEA22EECF00F0EFCF01F0FC0E79
:1018E000DBCFE9FFFD0EDBCFEAFF2A0EE926000E73
:1018F000EA2200C0EEFF01C0EDFFFA0EDBCFE9FFE8
:10190000FB0EDBCFEAFFEE50ED1025E1010EE66E97
:10191000FA0EDBCFE6FFFB0EDBCFE6FFFC0EDBCFE4
:10192000E6FFFD0EDBCFE6FFA0EC20F0026E050E19
:10193000E15C02E2E16AE552E16E0250F3CF00F0B1
:10194000F4CF01F00050011005E11C0EF36E070EFC
:10195000F3CFDBFF31D0FA0EDBCFE9FFFB0EDBCF9D
:10196000EAFFEECF52F0EDCF53F052500F0B24E0D0
:10197000010EE66EFA0EDBCFE6FFFB0EDBCFE6FFD5
:10198000FC0EDBCFE6FFFD0EDBCFE6FFA0EC20F088
:10199000026E050EE15C02E2E16AE552E16E025080
:1019A000F3CF00F0F4CF01F00050011005E11C0E60
:1019B000F36E070EF3CFDBFFFA0EDBCFE6FFFB0E75
:1019C000DBCFE6FFFC0EDBCFE6FFFD0EDBCFE6FF55
:1019D00063EC2CF0E552E552E552E552E76E020E5B
:1019E000E7CFDBFFDB50006E016A0050011006E01C
:1019F0000A0EF36E070EF3CFDBFF0BD1FC0EDBCF2D
:101A0000E9FFFD0EDBCFEAFF0A0EE926000EEA220F
:101A1000EE6AEE6AEE6AEE6AFC0EDBCFE9FFFD0EBF
:101A2000DBCFEAFF020EE926000EEA22EECF00F03D
:101A3000EFCF01F0FC0EDBCFE9FFFD0EDBCFEAFFBD
:101A4000040EE926000EEA2200C0EEFF01C0EDFF01
:101A5000FC0EDBCFE9FFFD0EDBCFEAFF060EEB6AE3
:101A6000070EEB6AFC0EDBCFE9FFFD0EDBCFEAFFD2
:101A7000080EEB6A090EEB6A020EDB50006E016A7B
:101A8000010E001801E1015006E10A0EF36E070E87
:101A9000F3CFDBFF7ED0FC0EDBCFE9FFFD0EDBCF0B
:101AA000EAFF040EE926000EEA22EECFE6FFEFCFB2
:101AB000E6FFDECFE6FFDDCFE6FF79EC3FF0E55253
:101AC000E552E552E552030E50C0DBFF040E51C053
:101AD000DBFF050E52C0DBFF060E53C0DBFF0F011C
:101AE0002A51006E016A0050011006E019EC44F022
:101AF000000902E0FF0E95D0FC0EDBCF24FFFD0EA7
:101B0000DBCF25FFD950030FE96E000EDA20EA6E15
:101B10000F012651EE1809E12751EE1806E1285170
:101B2000EE1803E12951EE1800E133E02B6BDECF14
:101B3000E9FFDDCFEAFFEECFE6FFEFCFE6FFD950BA
:101B4000030FE96E000EDA20EA6EEECFE6FFEECF6D
:101B5000E6FFEECFE6FFEFCFE6FF8DECA1F0006EE3
:101B6000060EE15C02E2E16AE552E16E0050000916
:101B700004E1070EF36EF3CFDBFF030EDBCF26FF8E
:101B8000040EDBCF27FF050EDBCF28FF060EDBCFD1
:101B900029FFFC0EDBCFE9FFFD0EDBCFEAFF120EC3
:101BA000E926000EEA22EF92F90EDBCF02F0036A7B
:101BB00002BE0368770E021801E103500DE0F90E32
:101BC000DBCF04F0056A04BE0568610E041801E16C
:101BD000055002E0000E01D0010E006E016A0050B7
:101BE00001100CE0FC0EDBCFE9FFFD0EDBCFEAFFBE
:101BF000120EE926000EEA22EF800BD0FC0EDBCF9E
:101C0000E9FFFD0EDBCFEAFF120EE926000EEA2205
:101C1000EF90070EDBCF00F0016A00BE01680050B4
:101C200000D0006E080EE15C02E2E16AE552E16E6E
:101C30000050E552E5CFDAFFE7CFD9FF1200D9CF48
:101C4000E6FFDACFE6FFE1CFD9FFE2CFDAFF070EFA
:101C5000E12402E3E168E652E16E040EDB6AFC0E69
:101C6000DBCFE9FFFD0EDBCFEAFF050EEECFDBFF9A
:101C7000060EEDCFDBFFFC0EDBCFE9FFFD0EDBCF69
:101C8000EAFF040EE926000EEA22020EEECFDBFF89
:101C9000030EEDCFDBFF020EDBCFE6FF030EDBCF43
:101CA000E6FF050EDBCFE6FF060EDBCFE6FF59ECC5
:101CB00053F0E552E552E552E552F3CFDEFFF4CFA3
:101CC000DDFFDECF00F0DDCF01F00001001C01E1FF
:101CD000011C06E1070EF36E040EF3CFDBFF68D0A4
:101CE000DECF00F0DDCF01F0026A036A050EDBCF24
:101CF000E9FF060EDBCFEAFF140EE926000EEA220A
:101D0000EE50005CEE500158EE500258EE50035871
:101D100005E3090EF36E040EF3CFDBFF050EDBCFF8
:101D2000E9FF060EDBCFEAFF1C0EE926000EEA22D1
:101D3000EF50006E016A020E001801E1015008E147
:101D4000F80EF36E020EF3CFDBFF030EDB681CD040
:101D5000050EDBCFE9FF060EDBCFEAFF1C0EE926FE
:101D6000000EEA22EF50006E016A010E001801E138
:101D700001500AE1F80EF36E020EF3CFDBFF0F0EF7
:101D8000F36E030EF3CFDBFFDECF00F0DDCF01F00B
:101D9000020EDBCF02F0030EDBCF03F00250005C3B
:101DA0000350015805E33C0EF36E040EF3CFDBFF46
:101DB000FC0EDBCFE9FFFD0EDBCFEAFF040EE926C8
:101DC000000EEA22DECFEEFFDDCFEDFFFA0EDB06DE
:101DD000DBCF02F0FB0E01E2DB06DBCF03F0000EEF
:101DE000D8800254000E035407E2040EDB50046E48
:101DF000056A0450051002E0000E01D0010E006ECD
:101E0000016A0050011001E036D7040EDB50006E6D
:101E1000070EE15C03E200D0E16AE552E16E00509A
:101E2000E552E5CFDAFFE7CFD9FF1200D9CFE6FFC1
:101E3000DACFE6FFE1CFD9FFE2CFDAFFE652DF6A81
:101E4000FC0EDBCFE9FFFD0EDBCFEAFF1D0EE9261E
:101E5000000EEA22EF6AFC0EDBCFE9FFFD0EDBCFBE
:101E6000EAFF000EEE6E080EED6E3EEC9EF0006E88
:101E7000016A010E001801E1015003E0050EDF6E5A
:101E80002AD0FC0EDBCFE6FFFD0EDBCFE6FF2CD821
:101E9000E552E552DF6E006E016A005001101BE151
:101EA000FC0EDBCFE6FFFD0EDBCFE6FFFED9E552F1
:101EB000E552DF6E006E016A005001100CE1FC0E6D
:101EC000DBCFE9FFFD0EDBCFEAFF1D0EE926000E9A
:101ED000EA22010EEF6EDF5000D0E552E552E5CF69
:101EE000DAFFE7CFD9FF1200D9CFE6FFDACFE6FF5E
:101EF000E1CFD9FFE2CFDAFF060EE12402E3E16889
:101F0000E652E16E020EDB6AFC0EDBCFE9FFFD0E4E
:101F1000DBCFEAFFEECFE6FFEFCFE6FFE66AE66A49
:101F2000E66AE66A8DECA1F0026E060EE15C02E262
:101F3000E16AE552E16E0250006E016A010E00187E
:101F400001E1015006E0070EF36E020EF3CFDBFF56
:101F50009BD1FC0EDBCFE9FFFD0EDBCFEAFF040EC9
:101F6000EECFDBFF050EEDCFDBFF040EDBCFE9FF8D
:101F7000050EDBCFEAFFFE0EE926010EEA22EF5046
:101F8000026E036A550E021801E1035012E1040EBD
:101F9000DBCFE9FF050EDBCFEAFFFF0EE926010EDE
:101FA000EA22EF50046E056AAA0E041801E10550FA
:101FB00002E0000E01D0010E006E016A0050011017
:101FC00001E1A0D0040EDBCFE9FF050EDBCFEAFF75
:101FD000360EE926000EEA22EF50086E096A460E18
:101FE000081801E1095016E1040EDBCFE9FF050EE8
:101FF000DBCFEAFF360EE926000EEA22010EE926C3
:10200000000EEA22EF500A6E0B6A410E0A1801E137
:102010000B5002E0000E01D0010E066E076A06505A
:10202000071016E0040EDBCFE9FF050EDBCFEAFF59
:10203000360EE926000EEA22020EE926000EEA22FA
:10204000EF500C6E0D6A540E0C1801E10D5002E0B9
:10205000000E01D0010E046E056A0450051016E052
:10206000040EDBCFE9FF050EDBCFEAFF360EE926D3
:10207000000EEA22030EE926000EEA22EF500E6E51
:102080000F6A310E0E1801E10F5002E0000E01D070
:10209000010E026E036A0250031012E0040EDBCF41
:1020A000E9FF050EDBCFEAFF260EE926000EEA2245
:1020B000EF50106E116A290E101801E1115002E064
:1020C000000E01D0010E006E016A005001101AE0EE
:1020D000FC0EDBCFE9FFFD0EDBCFEAFF020EE926A7
:1020E000000EEA22EE6AEE6AEE6AEE6AFC0EDBCFC2
:1020F000E9FFFD0EDBCFEAFF1C0EE926000EEA2207
:10210000020EEF6EFC0EDBCFE9FFFD0EDBCFEAFF28
:10211000EECFDEFFEDCFDDFFDECFE9FFDDCFEAFF63
:10212000FE0EE926010EEA22EF50026E036A550EFA
:10213000021801E1035012E1DECFE9FFDDCFEAFF33
:10214000FF0EE926010EEA22EF50046E056AAA0E80
:10215000041801E1055002E1000E01D0010E006EED
:10216000016A0050011006E0040EF36E020EF3CF78
:10217000DBFF8AD0DECFE9FFDDCFEAFFBE0EE92626
:10218000010EEA22080EE926000EEA22EECF00F048
:10219000EECF01F0EECF02F0EFCF03F0FC0EDBCF7D
:1021A000E9FFFD0EDBCFEAFF020EE926000EEA2270
:1021B00000C0EEFF01C0EEFF02C0EEFF03C0EEFF65
:1021C000DECFE9FFDDCFEAFFBE0EE926010EEA22EF
:1021D000040EE926000EEA22EF50E76E030EE7CF69
:1021E000DBFFDB50006E016A0B0E001801E10150AD
:1021F00034E00C0E001801E101502FE0040E00182D
:1022000001E101501DE0060E001801E1015018E047
:102210000E0E001801E1015013E0010E001801E15B
:10222000015001E02CD0FC0EDBCFE9FFFD0EDBCF2F
:10223000EAFF1C0EE926000EEA22010EEF6E24D002
:10224000FC0EDBCFE9FFFD0EDBCFEAFF1C0EE9261B
:10225000000EEA22020EEF6E17D0FC0EDBCFE9FF74
:10226000FD0EDBCFEAFF1C0EE926000EEA22030E6C
:10227000EF6E1D0EF36E020EF3CFDBFF05D0040EE2
:10228000F36E020EF3CFDBFF020EDB5000D0006EC8
:10229000060EE15C02E2E16AE552E16E0050E552B1
:1022A000E5CFDAFFE7CFD9FF1200D9CFE6FFDACFCB
:1022B000E6FFE1CFD9FFE2CFDAFF0F0EE12402E320
:1022C000E168E652E16E0A0EDB6AFC0EDBCFE9FF45
:1022D000FD0EDBCFEAFFEECFE6FFEFCFE6FFFC0E11
:1022E000DBCFE9FFFD0EDBCFEAFF020EE926000E91
:1022F000EA22EECFE6FFEECFE6FFEECFE6FFEFCF2E
:10230000E6FF8DECA1F0026E060EE15C02E2E16AEE
:10231000E552E16E0250006E016A010E001801E103
:10232000015006E0070EF36E0A0EF3CFDBFF08D371
:10233000FC0EDBCFE9FFFD0EDBCFEAFF0B0EEECF8D
:10234000DBFF0C0EEDCFDBFF0B0EDBCFE9FF0C0E3E
:10235000DBCFEAFFFE0EE926010EEA22EF50026E05
:10236000036A550E021801E1035014E10B0EDBCF96
:10237000E9FF0C0EDBCFEAFFFF0EE926010EEA2291
:10238000EF50046E056AAA0E041801E1055002E13F
:10239000000E01D0010E006E016A0050011006E02F
:1023A000030EF36E0A0EF3CFDBFFCAD20B0EDBCFA8
:1023B000E9FF0C0EDBCFEAFF160EE926000EEA223B
:1023C000EECF00F0EFCF01F0FC0EDBCFE9FFFD0E0A
:1023D000DBCFEAFF180EE926000EEA2200C0EEFF6E
:1023E00001C0EDFF0B0EDBCFE9FF0C0EDBCFEAFFE8
:1023F000130EE926000EEA22EE50ED1019E00B0E46
:10240000DBCFE9FF0C0EDBCFEAFF130EE926000E4F
:10241000EA22EECF00F0EFCF01F0020E00C0DBFFAA
:10242000030E01C0DBFF040EDB6A050EDB6A16D06B
:102430000B0EDBCFE9FF0C0EDBCFEAFF200EE92607
:10244000000EEA22020EEECFDBFF030EEECFDBFF23
:10245000040EEECFDBFF050EEECFDBFF0B0EDBCF66
:10246000E9FF0C0EDBCFEAFF0D0EE926000EEA2293
:10247000EF50E66EFC0EDBCFE9FFFD0EDBCFEAFF8F
:102480001B0EE926000EEA22E552E750EF6E0B0E16
:10249000DBCFE9FF0C0EDBCFEAFF0E0EE926000EC4
:1024A000EA22EECF00F0EFCF01F0026A036AFC0EE1
:1024B000DBCFE9FFFD0EDBCFEAFF020EE926000EBF
:1024C000EA22EE500026EE500122EE500222EE509B
:1024D0000322FC0EDBCFE9FFFD0EDBCFEAFF060E89
:1024E000E926000EEA2200C0EEFF01C0EEFF02C0A6
:1024F000EEFF03C0EEFF0B0EDBCFE9FF0C0EDBCFD0
:10250000EAFF100EE926000EEA22EF50E66EFC0EFE
:10251000DBCFE9FFFD0EDBCFEAFF1A0EE926000E46
:10252000EA22E552E750EF6E0B0EDBCFE9FF0C0E0F
:10253000DBCFEAFF110EE926000EEA22EECF00F013
:10254000EFCF01F0FC0EDBCFE9FFFD0EDBCFEAFFA2
:10255000120EE926000EEA2200C0EEFF01C0EDFFD8
:10256000FC0EDBCFE9FFFD0EDBCFEAFF180EE926FC
:10257000000EEA22EECF06F0EFCF07F0FC0EDBCF25
:10258000E9FFFD0EDBCFEAFF1A0EE926000EEA2274
:10259000EF50046E056A04C052F005C053F006C047
:1025A00057F007C058F03DECB3F050C000F051C0F8
:1025B00001F0026A036AFC0EDBCFE9FFFD0EDBCF00
:1025C000EAFF060EE926000EEA22EE500026EE5043
:1025D0000122EE500222EE500322FC0EDBCFE9FF77
:1025E000FD0EDBCFEAFF0A0EE926000EEA2200C04C
:1025F000EEFF01C0EEFF02C0EEFF03C0EEFF0B0EC8
:10260000DBCFE9FF0C0EDBCFEAFF0B0EE926000E55
:10261000EA220D0EEECFDBFF0E0EEDCFDBFFD95021
:102620000D0FE96E000EDA20EA6EEE50ED1012E0AA
:10263000010EE76E0D0EDBCF02F00E0EDBCF03F0C6
:10264000E7500216036A010E021801E1035002E08E
:10265000000E01D0010E006E016A0050011002E070
:10266000030E71D10B0EDBCFE9FF0C0EDBCFEAFFBF
:102670000B0EE926000EEA22EECF06F0EFCF07F0B0
:102680000B0EDBCFE9FF0C0EDBCFEAFF110EE926C4
:10269000000EEA22EECF02F0EFCF03F0050ED89045
:1026A00002360336E806FBE10B0EDBCFE9FF0C0E2A
:1026B000DBCFEAFF0B0EE926000EEA22EECF04F094
:1026C000EFCF05F00406055A02500424006E0350B3
:1026D0000520016E00C052F001C053F006C057F053
:1026E00007C058F0E2ECB5F052C0DEFF53C0DDFF8A
:1026F000DECF08F0DDCF09F00A6A0B6AFC0EDBCFF3
:10270000E9FFFD0EDBCFEAFF0A0EE926000EEA2202
:10271000EE500826EE500922EE500A22EE500B220F
:10272000D950020FE96E000EDA20EA6E0850EE5C16
:10273000046E0950EE58056E0A50EE58066E0B50A6
:10274000EE58076EFC0EDBCFE9FFFD0EDBCFEAFF94
:10275000020EE926000EEA220450EE24006E055017
:10276000EE20016E0650EE20026E0750EE20036E42
:10277000020E0026000E012202220322060E00C0D5
:10278000DBFF070E01C0DBFF080E02C0DBFF090EF6
:1027900003C0DBFFFC0EDBCFE9FFFD0EDBCFEAFF62
:1027A0001B0EE926000EEA22EF50046E056A066A47
:1027B000076A05AE02D00668076804C055F005C078
:1027C00056F006C057F007C058F0060EDBCF50F0A9
:1027D000070EDBCF51F0080EDBCF52F0090EDBCF36
:1027E00053F0BEECB5F050C000F051C001F052C043
:1027F00002F053C003F0FC0EDBCFE9FFFD0EDBCF90
:10280000EAFF140EE926000EEA2200C0EEFF01C026
:10281000EEFF02C0EEFF03C0EEFFFC0EDBCFE9FFD0
:10282000FD0EDBCFEAFF140EE926000EEA22F50EBC
:10283000EE5C0F0EEE58000EEE58000EEE580DE254
:10284000FC0EDBCFE9FFFD0EDBCFEAFF1C0EE92615
:10285000000EEA22010EEF6E25D0FC0EDBCFE9FF61
:10286000FD0EDBCFEAFF140EE926000EEA22F50E7C
:10287000EE5CFF0EEE58000EEE58000EEE580DE224
:10288000FC0EDBCFE9FFFD0EDBCFEAFF1C0EE926D5
:10289000000EEA22020EEF6E05D01D0EF36E0A0E38
:1028A000F3CFDBFFFC0EDBCFE9FFFD0EDBCFEAFF52
:1028B000120EE926000EEA22EECF00F0EFCF01F073
:1028C000040ED89001320032E804FBE1026A036A88
:1028D000FC0EDBCFE9FFFD0EDBCFEAFF0A0EE92697
:1028E000000EEA22EE500026EE500122EE500222A7
:1028F000EE500322FC0EDBCFE9FFFD0EDBCFEAFF3B
:102900000E0EE926000EEA2200C0EEFF01C0EEFF27
:1029100002C0EEFF03C0EEFF0B0EDBCFE9FF0C0E93
:10292000DBCFEAFF0B0EE926000EEA22EE5002E1B1
:10293000020EED1805E0030EF36E0A0EF3CFDBFF77
:102940000A0EDB5000D0006E0F0EE15C02E2E16A7D
:10295000E552E16E0050E552E5CFDAFFE7CFD9FF4F
:102960001200D9CFE6FFDACFE6FFE1CFD9FFE2CF01
:10297000DAFF3E0EE12402E3E168E652E16ED9504F
:10298000100F006E000EDA20016E2E0E00C0DBFF6D
:102990002F0E01C0DBFFD9503C0FE96EDACFEAFF02
:1029A000000EEA22000EEE6E080EED6E2E0EDBCF4C
:1029B000E9FF2F0EDBCFEAFF000EEE6E080EED6E84
:1029C00039EC9EF03EEC9EF0006E016A010E00189C
:1029D00001E1015004E0F368F468C4EF1EF0000E5A
:1029E000E66E080EE66EE66AE66AE66AE66A8DEC70
:1029F000A1F0026E060EE15C02E2E16AE552E16ED0
:102A00000250006E016A0050011004E1F368F4689E
:102A1000C4EF1EF02E0EDBCFE9FF2F0EDBCFEAFF57
:102A20000E0EEECFDBFF0F0EEDCFDBFF0E0EDBCF7A
:102A3000E9FF0F0EDBCFEAFFFE0EE926010EEA22C8
:102A4000EF50026E036A550E021801E1035012E1C5
:102A50000E0EDBCFE9FF0F0EDBCFEAFFFF0EE926FC
:102A6000010EEA22EF50046E056AAA0E041801E175
:102A7000055002E0000E01D0010E006E016A005008
:102A8000011001E1E8D00E0EDBCFE9FF0F0EDBCF26
:102A9000EAFF360EE926000EEA22EF50086E096AB8
:102AA000460E081801E1095016E10E0EDBCFE9FFD2
:102AB0000F0EDBCFEAFF360EE926000EEA22010EEA
:102AC000E926000EEA22EF500A6E0B6A410E0A1840
:102AD00001E10B5002E0000E01D0010E066E076A04
:102AE0000650071016E00E0EDBCFE9FF0F0EDBCF0E
:102AF000EAFF360EE926000EEA22020EE926000E53
:102B0000EA22EF500C6E0D6A540E0C1801E10D50C4
:102B100002E0000E01D0010E046E056A045005109B
:102B200016E00E0EDBCFE9FF0F0EDBCFEAFF360E0D
:102B3000E926000EEA22030EE926000EEA22EF50F3
:102B40000E6E0F6A310E0E1801E10F5002E0000EFA
:102B500001D0010E026E036A0250031012E00E0E45
:102B6000DBCFE9FF0F0EDBCFEAFF260EE926000ED2
:102B7000EA22EF50106E116A290E101801E111506F
:102B800002E0000E01D0010E006E016A005001103B
:102B900038E0FD0EDBCF00F0016A00BE0168005096
:102BA00001E101500BE0010E001801E1015001E0CC
:102BB00026D0F368F468C4EF1EF022D02E0EDBCFCF
:102BC000E9FF2F0EDBCFEAFF020EE926000EEA2214
:102BD000EE6AEE6AEE6AEE6A2E0EDBCFE6FF2F0E8D
:102BE000DBCFE6FF55EC11F0E552E552006E016ACD
:102BF0000050011004E0F368F468C4EF1EF000D048
:102C00002AD0000EDE6E080EDD6EDECFE9FFDDCFCE
:102C1000EAFFBE0EE926010EEA22080EE926000EA2
:102C2000EA22EECF00F0EECF01F0EECF02F0EFCFD0
:102C300003F02E0EDBCFE9FF2F0EDBCFEAFF020EF3
:102C4000E926000EEA2200C0EEFF01C0EEFF02C03E
:102C5000EEFF03C0EEFFFD0EDBCF00F0016A00BE09
:102C60000168005001E1015002E1DCEF1BF0010EB0
:102C7000001801E1015004E0F368F468C4EF1EF0AD
:102C8000DECFE9FFDDCFEAFFBE0EE926010EEA2224
:102C90000C0EE926000EEA22020EEECFDBFF030E39
:102CA000EECFDBFF040EEECFDBFF050EEECFDBFF3A
:102CB000D950020FE96E000EDA20EA6E390EEE5C92
:102CC000100EEE58000EEE58000EEE5874E22E0E66
:102CD000DBCFE9FF2F0EDBCFEAFF1C0EE926000E4B
:102CE000EA22010EEF6EDECFE9FFDDCFEAFFBE0E76
:102CF000E926010EEA22040EE926000EEA22010E60
:102D0000EF6EE66E000EE66E080EE66EE66AE66AA6
:102D1000E66AE66A19ECA4F0026E070EE15C02E2D4
:102D2000E16AE552E16E0250006E016A0050011046
:102D300004E1F368F468C4EF1EF0D950020FE96EA5
:102D4000000EDA20EA6E280EEE5C100EEE58000E31
:102D5000EE58000EEE580DE32E0EDBCFE9FF2F0EDE
:102D6000DBCFEAFF1B0EE926000EEA22020EEF6E11
:102D70000CD02E0EDBCFE9FF2F0EDBCFEAFF1B0EB0
:102D8000E926000EEA22010EEF6EE66A020EE66EFA
:102D9000E66A000EE66E080EE66EC7ECB3F0006E53
:102DA000050EE15C02E2E16AE552E16E00500801C5
:102DB000320E3A6FD0D0D950020FE96E000EDA20F1
:102DC000EA6ED8805F0EEE54FD0EEE543F0EEE54C8
:102DD000000EEE5401E2BBD02E0EDBCFE9FF2F0E2A
:102DE000DBCFEAFF1C0EE926000EEA22020EEF6E90
:102DF000DECFE9FFDDCFEAFFBE0EE926010EEA22B3
:102E0000040EE926000EEA22060EEF6E010EE66EB3
:102E1000000EE66E080EE66EE66AE66AE66AE66AA6
:102E200019ECA4F0026E070EE15C02E2E16AE552E1
:102E3000E16E0250006E016A0050011004E1F36877
:102E4000F468C4EF1EF0020EDBCF00F0030EDBCF00
:102E500001F0040EDBCF02F0050EDBCF03F0180EFD
:102E6000005E020E015A000E025A035A060E00C0FE
:102E7000DBFF070E01C0DBFF080E02C0DBFF090EFF
:102E800003C0DBFF2E0EDBCFE9FF2F0EDBCFEAFF07
:102E90001B0EE926000EEA22010EEF6ED950060F36
:102EA000E96E000EDA20EA6ED880ED0EEE54FF0EC9
:102EB000EE54000EEE54000EEE541BE22E0EDBCF4D
:102EC000E9FF2F0EDBCFEAFF1B0EE926000EEA22F8
:102ED000EF9EEF46D950060FE96E000EDA20EA6E3B
:102EE000D890030EEB32020EEB32010EEB32EF32D2
:102EF000D5D72E0EDBCFE9FF2F0EDBCFEAFF1B0E5F
:102F0000E926000EEA22EF50006E016A013404E265
:102F100000508008000E015404E2F368F468C4EF26
:102F20001EF0E66A020EE66EE66A000EE66E080E17
:102F3000E66EC7ECB3F0006E050EE15C02E2E16AFA
:102F4000E552E16E00500801360E3A6F04D0F36886
:102F5000F468C4EF1EF0020EDBCF00F0030EDBCFEF
:102F600001F0040EDBCF02F0050EDBCF03F0210EE3
:102F7000005E000E015A025A035A2E0EDBCFE9FF03
:102F80002F0EDBCFEAFF1B0EE926000EEA22EF50E0
:102F9000086E096A020E526E536A08C057F009C0E3
:102FA00058F010ECB3F050C004F051C005F0066AC0
:102FB000076A05AE02D0066807680450002605506F
:102FC00001220650022207500322340E00C0DBFF0C
:102FD000350E01C0DBFF360E02C0DBFF370E03C02B
:102FE000DBFF2E0EDBCFE9FF2F0EDBCFEAFF1C0E3F
:102FF000E926000EEA22EF50006E016A010E001869
:1030000001E1015032E12E0EDBCFE9FF2F0EDBCFC5
:10301000EAFF1B0EE926000EEA22EF50046E056A55
:10302000550E526E010E536E04C057F005C058F095
:1030300010ECB3F050C000F051C001F0020E0026B9
:10304000000E0122026A036A01AE02D00268036820
:10305000380E00C0DBFF390E01C0DBFF3A0E02C0A4
:10306000DBFF3B0E03C0DBFF30D02E0EDBCFE9FFD2
:103070002F0EDBCFEAFF1B0EE926000EEA22EF50EF
:10308000046E056A526A010E536E04C057F005C003
:1030900058F010ECB3F050C000F051C001F0020E37
:1030A0000026000E0122026A036A01AE02D0026805
:1030B0000368380E00C0DBFF390E01C0DBFF3A0E9B
:1030C00002C0DBFF3B0E03C0DBFF380EDBCF00F09E
:1030D000390EDBCF01F03A0EDBCF02F03B0EDBCF37
:1030E00003F00006000E015A025A035AD950340F59
:1030F000E96E000EDA20EA6EEE500026EE50012254
:10310000EE500222EE50032200C050F001C051F0F8
:1031100002C052F003C053F0380EDBCF55F0390E29
:10312000DBCF56F03A0EDBCF57F03B0EDBCF58F03B
:10313000BEECB5F0340E50C0DBFF350E51C0DBFFE6
:10314000360E52C0DBFF370E53C0DBFF0801EB0E1B
:10315000006F3C0E016F900E026F4D0E036F430E19
:10316000046F480E056F500E066F200E076F460E57
:10317000086F410E096F540E0A6F0B6B020E0C6F35
:103180002E0EDBCFE9FF2F0EDBCFEAFF1B0EE92669
:10319000000EEA22EF500D6F080E0E6F0F6B2E0E11
:1031A000DBCFE9FF2F0EDBCFEAFF020EE926000E90
:1031B000EA22EECF00F0EECF01F0EECF02F0EFCF3B
:1031C00003F0080E0026000E0122022203222E0E1A
:1031D000DBCFE9FF2F0EDBCFEAFF060EE926000E5C
:1031E000EA2200C0EEFF01C0EEFF02C0EEFF03C006
:1031F000EEFF020E106F2E0EDBCFE9FF2F0EDBCF9E
:10320000EAFF1A0EE926000EEA22020EEF6E116B9B
:10321000126F2E0EDBCFE9FF2F0EDBCFEAFF120E6F
:10322000E926000EEA22EE6A020EED6E136B146BB5
:10323000F80E156F340EDBCF00F0350EDBCF01F04A
:10324000360EDBCF02F0370EDBCF03F00050166FE7
:10325000340EDBCF00F0350EDBCF01F0360EDBCFC6
:1032600002F0370EDBCF03F0080ED89003320232A3
:1032700001320032E806F9E100500801176F2E0E06
:10328000DBCFE9FF2F0EDBCFEAFF180EE926000E99
:10329000EA22340EDBCFEEFF350EDBCFEDFF3F0E23
:1032A000186F196B1A691B6B2E0EDBCFE9FF2F0EFF
:1032B000DBCFEAFF020EE926000EEA22EECF00F095
:1032C000EECF01F0EECF02F0EFCF03F000501C6F15
:1032D0002E0EDBCFE9FF2F0EDBCFEAFF020EE92631
:1032E000000EEA22EECF00F0EECF01F0EECF02F0BA
:1032F000EFCF03F0080ED8900332023201320032D1
:10330000E806F9E1005008011D6F2E0EDBCFE9FF42
:103310002F0EDBCFEAFF020EE926000EEA22EECFE7
:1033200000F0EECF01F0EECF02F0EFCF03F0100E81
:10333000D8900332023201320032E806F9E100503F
:1033400008011E6F2E0EDBCFE9FF2F0EDBCFEAFF49
:10335000020EE926000EEA22EECF00F0EECF01F0D9
:10336000EECF02F0EFCF03F0180ED8900332023206
:1033700001320032E806F9E1005008011F6F020E29
:10338000DBCF00F0030EDBCF01F0040EDBCF02F049
:10339000050EDBCF03F00050206F020EDBCF00F0F4
:1033A000030EDBCF01F0040EDBCF02F0050EDBCF06
:1033B00003F0080ED8900332023201320032E806E0
:1033C000F9E100500801216F020EDBCF00F0030E7F
:1033D000DBCF01F0040EDBCF02F0050EDBCF03F0F4
:1033E000100ED8900332023201320032E806F9E1C1
:1033F00000500801226F020EDBCF00F0030EDBCF7E
:1034000001F0040EDBCF02F0050EDBCF03F0180E47
:10341000D8900332023201320032E806F9E100505E
:103420000801236F246B256B290E266FF90EDBCF65
:1034300000F0FA0EDBCF01F0FB0EDBCF02F0FC0E4A
:10344000DBCF03F00050276FF90EDBCF00F0FA0E50
:10345000DBCF01F0FB0EDBCF02F0FC0EDBCF03F085
:10346000556A010E566E576A586A00C050F001C086
:1034700051F002C052F003C053F0DCECB2F050C087
:1034800000F051C001F052C002F053C003F00050F0
:103490000801286FF90EDBCF00F0FA0EDBCF01F048
:1034A000FB0EDBCF02F0FC0EDBCF03F0556A566A51
:1034B000010E576E586A00C050F001C051F002C0B2
:1034C00052F003C053F0DCECB2F050C000F051C039
:1034D00001F052C002F053C003F000500801296F00
:1034E000F90EDBCF00F0FA0EDBCF01F0FB0EDBCFE5
:1034F00002F0FC0EDBCF03F0556A566A576A010EE4
:10350000586E00C050F001C051F002C052F003C02C
:1035100053F0DCECB2F050C000F051C001F052C0EA
:1035200002F053C003F0005008012A6FD950F70F82
:10353000E96EFF0EDA20EA6EEE50ED1001E178D070
:10354000300EDB6A310EDB6A300EDBCF04F0310E59
:10355000DBCF05F0F70EDB500424E96EF80EDB50EC
:103560000520EA6EEFCF02F0036A02BE0368025044
:1035700003100BE0300EDBCF06F0310EDBCF07F08F
:103580000B0E065C000E075802E3000E01D0010E80
:10359000006E016A005001102BE0300EDBCF02F00C
:1035A000310EDBCF03F0F70EDB500224E96EF80E8C
:1035B000DB500320EA6EEFCF00F0016A00BE016825
:1035C0002B0EE76E300EDBCFE9FF310EDBCFEAFFCB
:1035D000E750E926000EEA22000EE926080EEA224C
:1035E00000C0EFFF300EDB2A310E01E3DB2AACD73F
:1035F000300EDBCF00F0310EDBCF01F00B0E005CA4
:10360000000E015814E2300EDBCFE9FFDB2A310E49
:10361000DBCFEAFF01E3DB2A2B0EE926000EEA22CC
:10362000000EE926080EEA22200EEF6EE1D726D022
:10363000300EDB6A310EDB6A300EDBCF00F0310E6C
:10364000DBCF01F00B0E005C000E015817E22B0ED1
:10365000E76E300EDBCFE9FF310EDBCFEAFFE7503C
:10366000E926000EEA22000EE926080EEA22EF6A99
:10367000300EDB2A310E01E3DB2ADED70801460ECD
:10368000366F410E376F540E386F310E396F200E82
:103690003B6F3C6F3D6F3C0EDBCFE9FF3D0EDBCF58
:1036A000EAFFFE0EE926010EEA22550EEF6E3C0EF1
:1036B000DBCFE9FF3D0EDBCFEAFFFF0EE926010E6F
:1036C000EA22AA0EEF6E2E0EDBCFE9FF2F0EDBCF24
:1036D000EAFF180EE926000EEA22EECF06F0EFCF41
:1036E00007F02E0EDBCFE9FF2F0EDBCFEAFF1A0E1D
:1036F000E926000EEA22EF50046E056A04C052F07B
:1037000005C053F006C057F007C058F03DECB3F0C9
:1037100050C000F051C001F0026A036A2E0EDBCFE8
:10372000E9FF2F0EDBCFEAFF060EE926000EEA22A4
:10373000EE500026EE500122EE500222EE500322FF
:103740002E0EDBCFE9FF2F0EDBCFEAFF0A0EE926B4
:10375000000EEA2200C0EEFF01C0EEFF02C0EEFF45
:1037600003C0EEFFE66A000EE66E080EE66E2E0E51
:10377000DBCFE9FF2F0EDBCFEAFF020EE926000EBA
:10378000EA22EECFE6FFEECFE6FFEECFE6FFEFCF89
:10379000E6FF19ECA4F0026E070EE15C02E2E16ABA
:1037A000E552E16E0250006E016A0050011003E123
:1037B000F368F468E9D213D02E0EDBCFE6FF2F0EAC
:1037C000DBCFE6FF55EC11F0E552E552006E016AE1
:1037D0000050011003E0F368F468D6D200D0E66A26
:1037E000020EE66EE66A000EE66E080EE66EC7ECA6
:1037F000B3F0006E050EE15C02E2E16AE552E16EB3
:1038000000500801F80E006F016902692E0EDBCF2F
:10381000E9FF2F0EDBCFEAFF1C0EE926000EEA229D
:10382000EF50006E016A020E001801E1015001E143
:1038300003692E0EDBCFE9FF2F0EDBCFEAFF1A0E56
:10384000E926000EEA22EF50006E016A0006000E23
:10385000015A320E00C0DBFF330E01C0DBFFD9502E
:10386000320FE96E000EDA20EA6EFF0EEE1802E16A
:10387000FF0EED1857E0E66A000EE66E080EE66EE3
:103880002E0EDBCFE9FF2F0EDBCFEAFF180EE92665
:10389000000EEA22EECF06F0EFCF07F0320EDBCFBC
:1038A00052F0330EDBCF53F006C057F007C058F08C
:1038B0003DECB3F050C002F051C003F0046A056A59
:1038C0002E0EDBCFE9FF2F0EDBCFEAFF060EE92637
:1038D000000EEA22EE500226EE500322EE500422A1
:1038E000EE50052202C0E6FF03C0E6FF04C0E6FF7B
:1038F00005C0E6FF19ECA4F0086E070EE15C02E2D9
:10390000E16AE552E16E0850006E016A0050011054
:1039100003E1F368F46838D2320EDB06330E01E2BD
:10392000DB069DD7040EE66EE66AE66A000EE66EDA
:10393000080EE66EC7ECB3F0006E050EE15C02E225
:10394000E16AE552E16E0050010E006E016A026A02
:10395000036A2E0EDBCFE9FF2F0EDBCFEAFF060E48
:10396000E926000EEA22EE500026EE500122EE502B
:103970000222EE500322300E00C0DBFF310E01C0E8
:10398000DBFF300EDBCF00F0310EDBCF01F0026A3F
:10399000036A2E0EDBCFE9FF2F0EDBCFEAFF180EF6
:1039A000E926000EEA22EECF04F0EFCF05F0066A1A
:1039B000076A2E0EDBCFE9FF2F0EDBCFEAFF060EE4
:1039C000E926000EEA22EE500426EE500522EE50C3
:1039D0000622EE5007220450005C055001580650A4
:1039E00002580750035875E22E0EDBCFE9FF2F0E69
:1039F000DBCFEAFF1A0EE926000EEA22EF50006E36
:103A0000016A0006000E015A320E00C0DBFF330EC1
:103A100001C0DBFFD950320FE96E000EDA20EA6EEA
:103A2000FF0EEE1802E1FF0EED184DE0E66A000E03
:103A3000E66E080EE66E300EDBCF06F0310EDBCF01
:103A400007F02E0EDBCFE9FF2F0EDBCFEAFF180EBB
:103A5000E926000EEA22EECF08F0EFCF09F0320E91
:103A6000DBCF52F0330EDBCF53F008C057F009C064
:103A700058F03DECB3F006505024026E0750512030
:103A8000036E046A056A02C0E6FF03C0E6FF04C0D5
:103A9000E6FF05C0E6FF19ECA4F00A6E070EE15C34
:103AA00002E2E16AE552E16E0A50006E016A0050DE
:103AB000011003E1F368F46867D1320EDB06330EC0
:103AC00001E2DB06A7D7300EDB2A310E01E3DB2A49
:103AD00058D72E0EDBCFE9FF2F0EDBCFEAFF120EF9
:103AE000E926000EEA22EECF00F0EFCF01F0050E3E
:103AF000D89000360136E806FBE1FF0E0026010EE5
:103B00000122090E0F0B05E0D89001320032E806C1
:103B1000FBE10A0E00C0DBFF0B0E01C0DBFF0C0E49
:103B2000DB6A0D0EDB6A010EF36E300EF3CFDBFFA6
:103B3000310EDB6A300EDBCF00F0310EDBCF01F04F
:103B4000026A036AD9500A0FE96E000EDA20EA6EA3
:103B5000EE50005CEE500158EE500258EE50035803
:103B60003FE2E66A000EE66E080EE66E300EDBCF30
:103B700002F0310EDBCF03F0046A056A2E0EDBCFB4
:103B8000E9FF2F0EDBCFEAFF0A0EE926000EEA223C
:103B9000EE500226EE500322EE500422EE50052293
:103BA00002C0E6FF03C0E6FF04C0E6FF05C0E6FF73
:103BB00019ECA4F0066E070EE15C02E2E16AE55240
:103BC000E16E0650006E016A0050011003E1F368D7
:103BD000F468DAD0300EDB2A310E01E3DB2AAAD7F3
:103BE000D950F70FE96EFF0EDA20EA6EEE50ED10B5
:103BF00001E19ED0300EDB6A310EDB6A300EDBCF86
:103C000004F0310EDBCF05F0F70EDB500424E96E33
:103C1000F80EDB500520EA6EEFCF02F0036A02BE19
:103C20000368025003100BE0300EDBCF06F0310EBC
:103C3000DBCF07F00B0E065C000E075802E3000E08
:103C400001D0010E006E016A0050011025E0300E17
:103C5000DBCF02F0310EDBCF03F0F70EDB50022496
:103C6000E96EF80EDB500320EA6EEFCF00F0016A38
:103C700000BE0168300EDBCFE9FF310EDBCFEAFF7B
:103C8000000EE926080EEA2200C0EFFF300EDB2A04
:103C9000310E01E3DB2AB2D7300EDBCF00F0310E5C
:103CA000DBCF01F00B0E005C000E015810E2300E6D
:103CB000DBCFE9FFDB2A310EDBCFEAFF01E3DB2AB2
:103CC000000EE926080EEA22200EEF6EE5D7080165
:103CD000080E0B6F110E116F136F176FE66A000E4F
:103CE000E66E080EE66E2E0EDBCFE9FF2F0EDBCF61
:103CF000EAFF0A0EE926000EEA22EECFE6FFEECF3B
:103D0000E6FFEECFE6FFEFCFE6FF19ECA4F0026E80
:103D1000070EE15C02E2E16AE552E16E0250006EDC
:103D2000016A0050011003E1F368F4682DD029D036
:103D3000E66A000EE66E080EE66E2E0EDBCFE9FF99
:103D40002F0EDBCFEAFF0A0EE926000EEA22EECFA5
:103D5000E6FFEECFE6FFEECFE6FFEFCFE6FF19EC92
:103D6000A4F0026E070EE15C02E2E16AE552E16E48
:103D70000250006E016A0050011003E1F368F4681C
:103D800003D0F36AF46A00D03E0EE15C02E2E16A1D
:103D9000E552E16EE552E5CFDAFFE7CFD9FF120039
:103DA000D9CFE6FFDACFE6FFE1CFD9FFE2CFDAFFE6
:103DB0000A0EE12402E3E168E652E16EFC0EDBCF7D
:103DC000E9FFFD0EDBCFEAFFEECFDEFFEDCFDDFF3B
:103DD000FC0EDBCFE9FFFD0EDBCFEAFF2A0EE92662
:103DE000000EEA22080EEECFDBFF090EEDCFDBFF5F
:103DF000FA0EDBCFE9FFFB0EDBCFEAFFEECF00F0E0
:103E0000EFCF01F0040ED89001320032E804FBE15C
:103E1000030E00C0DBFFD950080FE96E000EDA2058
:103E2000EA6EEE50ED1022E0DECFE9FFDDCFEAFFD3
:103E30001B0EE926000EEA22EF50026E036A030E03
:103E4000DB50006E016A00C052F001C053F002C0A6
:103E500057F003C058F0B6ECB2F003AE04D04E6C8D
:103E60004F1E000E4F22030E4EC0DBFF080EDBCFAD
:103E7000E6FF090EDBCFE6FFDECFE6FFDDCFE6FF94
:103E800079EC3FF0E552E552E552E552040E50C0A0
:103E9000DBFF050E51C0DBFF060E52C0DBFF070E35
:103EA00053C0DBFFE66ADECFE9FFDDCFEAFFEECFEE
:103EB000E6FFEFCFE6FF030EDB50006E016A026AF9
:103EC000036A01AE02D002680368D950040FE96E9C
:103ED000000EDA20EA6EEE500026EE500122EE507F
:103EE0000222EE50032200C0E6FF01C0E6FF02C03E
:103EF000E6FF03C0E6FF19ECA4F0046E070EE15CD8
:103F000002E2E16AE552E16E0450000903E1020EAB
:103F1000DB6A05D0010EF36E020EF3CFDBFFDB5040
:103F2000006E0A0EE15C03E200D0E16AE552E16E48
:103F30000050E552E5CFDAFFE7CFD9FF1200D9CF25
:103F4000E6FFDACFE6FFE1CFD9FFE2CFDAFFE652B4
:103F5000E652E652E652E652040EDB6AD950FC0FF6
:103F6000E96EFF0EDA20EA6EEE50ED100DE0D9504A
:103F7000FC0FE96EFF0EDA20EA6E010EEE1801E189
:103F8000ED5002E0000E01D0010E006E016A0050FB
:103F9000011006E0020EF36E040EF3CFDBFF9BD0A0
:103FA000040EDBCF00F0016A00BE01680050011072
:103FB00001E091D0FC0EDBCFE6FFFD0EDBCFE6FF8C
:103FC000FA0EDBCFE6FFFB0EDBCFE6FF59EC53F03A
:103FD000E552E552E552E552F3CFDEFFF4CFDDFFC7
:103FE000DECF00F0DDCF01F00001001C01E1011C7B
:103FF00006E1010EF36E040EF3CFDBFF6BD0D9CFD9
:10400000E9FFDACFEAFFEE50ED100BE0D9CFE9FF80
:10401000DACFEAFF010EEE1801E1ED5002E0000EEA
:1040200001D0010E006E016A0050011006E0020E80
:10403000F36E040EF3CFDBFF4DD0F80EF36E020EDD
:10404000F3CFDBFF030EDB68DECF00F0DDCF01F046
:10405000020EDBCF02F0030EDBCF03F00250005C58
:104060000350015805E3020EF36E040EF3CFDBFF9D
:10407000E66A000EE66EE66AFC0EDBCFE6FFFD0E9A
:10408000DBCFE6FFFA0EDBCFE6FFFB0EDBCFE6FF72
:1040900000EC57F0026E070EE15C02E2E16AE552C5
:1040A000E16E0250F3CF00F0F4CF01F00001001CEC
:1040B00001E1011C05E1010EF36E040EF3CFDBFFFD
:1040C000D9CFE9FFDACFEAFFFC0EEECFDBFFFD0E22
:1040D000EDCFDBFF65D7010EE66E000EE66EE66AF9
:1040E000E66EE66AFA0EDBCFE6FFFB0EDBCFE6FFFD
:1040F00000EC57F0006E070EE15C02E2E16AE55267
:10410000E16E0050040EDBCF00F0016A00BE0168D2
:10411000020E001801E1015003E1010E03D002D0AC
:10412000000E00D0006E050EE15C02E2E16AE5528D
:10413000E16E0050E552E5CFDAFFE7CFD9FF12007C
:10414000D9CFE6FFDACFE6FFE1CFD9FFE2CFDAFF42
:104150000E0EE12402E3E168E652E16EFC0EDBCFD5
:10416000E9FFFD0EDBCFEAFF020EEECFDBFF030E11
:10417000EDCFDBFFFC0EDBCFE9FFFD0EDBCFEAFF6F
:10418000280EE926000EEA22080EEECFDBFF090E0C
:10419000EDCFDBFFFC0EDBCFE9FFFD0EDBCFEAFF4F
:1041A0002A0EE926000EEA220A0EEECFDBFF0B0EE6
:1041B000EDCFDBFFFA0EDBCFE9FFFB0EDBCFEAFF33
:1041C000EECF00F0EFCF01F0040ED89001320032B4
:1041D000E804FBE10C0E00C0DBFFDB50E76E0C0EC9
:1041E000E7CFDBFFD950080FE96E000EDA20EA6E48
:1041F000EE50ED1024E0020EDBCFE9FF030EDBCF23
:10420000EAFF1B0EE926000EEA22EF50026E036A57
:104210000C0EDB50006E016A00C052F001C053F07A
:1042200002C057F003C058F0B6ECB2F003AE04D0B1
:104230004E6C4F1E000E4F220C0E4EC0DBFFF90ECF
:10424000DB50026E036A025003100FE1FA0EDBCF5F
:10425000E9FFFB0EDBCFEAFFEECF52F0EDCF53F0DC
:1042600052500F0B02E0000E01D0010E006E016AE9
:104270000050011001E1ADD10C0EDB50046E056A57
:10428000045005100FE1FA0EDBCFE9FFFB0EDBCF88
:10429000EAFFEECF06F0EFCF07F0100E065C000E3F
:1042A000075802E2000E01D0010E026E036A0250AE
:1042B000031009E1F90EDB50086E096A0850091075
:1042C00002E1000E01D0010E006E016A00500110E3
:1042D00001E177D0D950080FE96E000EDA20EA6EBE
:1042E000EE50ED1005E10A0EDB6A0B0EDB6A69D0B9
:1042F000F90EDB50006E016A005001102EE0020E34
:10430000DBCFE9FF030EDBCFEAFF1B0EE926000E31
:10431000EA22EF50026E036A100E526E536A02C018
:1043200057F003C058F03DECB3F050C000F051C05E
:1043300001F0FA0EDBCFE9FFFB0EDBCFEAFFEECF99
:1043400052F0EDCF53F000C057F001C058F0E2EC4E
:10435000B5F00D0E52C0DBFF05D0010EF36E0D0E51
:10436000F3CFDBFF0D0EDB50006E016A0050011031
:1043700028E00A0EDBCFE6FF0B0EDBCFE6FF020ED6
:10438000DBCFE6FF030EDBCFE6FF59EC53F0E5523F
:10439000E552E552E5520A0EF3CFDBFF0B0EF4CFE8
:1043A000DBFF0A0EDBCF00F00B0EDBCF01F0F80EC7
:1043B000005CFF0E015802E304D002D00D0EDB06B4
:1043C000D1D70A0EDBCF00F00B0EDBCF01F0F80ED9
:1043D000005CFF0E015801E3F9D0FC0EDBCFE9FFD2
:1043E000FD0EDBCFEAFF2A0EE926000EEA220A0EB6
:1043F000DBCFEEFF0B0EDBCFEDFF0A0EDBCFE6FFD0
:104400000B0EDBCFE6FF020EDBCFE6FF030EDBCFAA
:10441000E6FF79EC3FF0E552E552E552E552040E35
:1044200050C0DBFF050E51C0DBFF060E52C0DBFFA4
:10443000070E53C0DBFFD9500A0FE96E000EDA20D9
:10444000EA6EEE50ED102BE10C0EDB50026E036AAB
:10445000046A056A03AE02D004680568D950040FE7
:10446000E96E000EDA20EA6EEE500226EE500322CC
:10447000EE500422EE500522020EDBCFE9FF030EC0
:10448000DBCFEAFF0E0EE926000EEA22EE50025CB8
:10449000EE500358EE500458EE50055802E2000E5C
:1044A00001D0010E006E016A0050011003E0DE6AC7
:1044B000DD6A8BD00F012A51006E016A0050011095
:1044C00007E019EC44F0000903E0F36AF46AAED0A7
:1044D0000F01246B256B2B6B020EDBCFE9FF030E64
:1044E000DBCFEAFFEECFE6FFEFCFE6FF0C0EDB50AF
:1044F000026E036A046A056A03AE02D004680568A6
:10450000D950040FE96E000EDA20EA6EEE50022652
:10451000EE500322EE500422EE50052202C0E6FFC8
:1045200003C0E6FF04C0E6FF05C0E6FF8DECA1F086
:10453000066E060EE15C02E2E16AE552E16E0650AB
:10454000006E016A010E001801E1015003E0DE6A0D
:10455000DD6A36D0F90EDB50006E016A00500110A2
:1045600025E0FA0EDBCFE9FFFB0EDBCFEAFFEECF53
:1045700002F0EFCF03F00001036A0F0E0216050EE2
:10458000D89002360336E806FBE1020EDBCFE9FFE6
:10459000030EDBCFEAFF0250EE24006E0350EE2044
:1045A000016E00C0DEFF01C0DDFF0AD0020EDBCFCE
:1045B000E9FF030EDBCFEAFFEECFDEFFEDCFDDFF3D
:1045C0000F01266927692869296902D0DE6ADD6A38
:1045D00024D0FA0EDBCFE9FFFB0EDBCFEAFFEECFF4
:1045E00002F0EFCF03F00001036A0F0E0216050E72
:1045F000D89002360336E806FBE1020EDBCFE9FF76
:10460000030EDBCFEAFF0250EE24006E0350EE20D3
:10461000016E00C0DEFF01C0DDFFDECF00F0DDCFA8
:1046200001F000C0F3FF01C0F4FF00D00E0EE15C0A
:1046300002E2E16AE552E16EE552E5CFDAFFE7CF4B
:10464000D9FF1200D9CFE6FFDACFE6FFE1CFD9FFDD
:10465000E2CFDAFF0D0EE12402E3E168E652E16EFB
:10466000010EDB6ADF6ADF50006E016AD8900150EC
:1046700004E60B0E005C000E01582AE2FC0EDBCFB4
:10468000E9FFFD0EDBCFEAFF170EE926000EEA2256
:10469000E9CF04F0EACF05F0DF500F010424E96E02
:1046A000000E0520EA6EEFCF02F0036A02BE036837
:1046B000D950020F006E000EDA20016EDF50002488
:1046C000E96E000E0120EA6E02C0EFFFDF2ACBD7B1
:1046D000010EDBCF00F0016A00BE0168005001103E
:1046E00056E1FA0EDBCFE9FFFB0EDBCFEAFFEE6A05
:1046F000ED6AFA0EDBCFE6FFFB0EDBCFE6FFFC0E2A
:10470000DBCFE6FFFD0EDBCFE6FFE7D8E552E55253
:10471000E552E552000938E0F90EDB50E66EFA0E7C
:10472000DBCFE6FFFB0EDBCFE6FFD950020FE66ED4
:10473000000EDA20E66EFC0EDBCFE6FFFD0EDBCFCF
:10474000E6FF3DDA026E070EE15C02E2E16AE55245
:10475000E16E0250E76E010EE7CFDBFFDBCF00F02A
:10476000016A00BE0168005001100DE1FC0EDBCFB4
:10477000E6FFFD0EDBCFE6FF20D8E552E552E76EFF
:10478000010EE7CFDBFF03D0DE52110EDD6E010E0E
:10479000DBCF00F0016A00BE01680050006E0D0E14
:1047A000E15C03E200D0E16AE552E16E0050E552BF
:1047B000E5CFDAFFE7CFD9FF1200D9CFE6FFDACF96
:1047C000E6FFE1CFD9FFE2CFDAFF070EE12402E3F3
:1047D000E168E652E16EFC0EDBCFE9FFFD0EDBCFB8
:1047E000EAFF220EE926000EEA22030EEECFDBFFDF
:1047F000040EEDCFDBFFD950010FE66E000EDA207C
:10480000E66EFC0EDBCFE6FFFD0EDBCFE6FFD0EC65
:104810003DF0E552E552E552E552DF6E006E016A69
:1048200000BE01680050011043E1D950030FE66E4D
:10483000000EDA20E66EFC0EDBCFE6FFFD0EDBCFCE
:10484000E6FF06EC2FF0E552E552E552E552050E83
:10485000F3CFDBFF060EF4CFDBFF050EDBCFE9FF66
:10486000060EDBCFEAFF1A0EE926000EEA22010E41
:10487000DBCFEEFF020EDBCFEDFFD950030FE66E6C
:10488000000EDA20E66EFC0EDBCFE6FFFD0EDBCF7E
:10489000E6FFD0EC1EF0E552E552E552E552006E1F
:1048A000016A010E001801E1015002E0080EDF6EFE
:1048B000DFCF00F0016A00BE01680050006E070EF5
:1048C000E15C03E200D0E16AE552E16E0050E5529E
:1048D000E5CFDAFFE7CFD9FF1200D9CFE6FFDACF75
:1048E000E6FFE1CFD9FFE2CFDAFF090EE12402E3D0
:1048F000E168E652E16E010EDF6EFC0EDBCFE9FFF0
:10490000FD0EDBCFEAFF280EE926000EEA22EECFED
:1049100000F0EFCF01F0FC0EDBCFE9FFFD0EDBCFA7
:10492000EAFF2A0EE926000EEA2200C0EEFF01C0CF
:10493000EDFF010EE66EFA0EDBCFE6FFFB0EDBCFDE
:10494000E6FFFC0EDBCFE6FFFD0EDBCFE6FFA0ECC3
:1049500020F0026E050EE15C02E2E16AE552E16ED2
:104960000250070EF3CFDBFF080EF4CFDBFFF3CFCF
:1049700000F0F4CF01F00050011003E11C0EDF6ED7
:1049800005D1DF50006E016A010E001801E10150EF
:1049900001E0F0D0010EDB6AFA0EDBCFE9FFFB0E7F
:1049A000DBCFEAFF030EEECFDBFF040EEDCFDBFF24
:1049B000E66AFA0EDBCFE6FFFB0EDBCFE6FFFC0E6E
:1049C000DBCFE6FFFD0EDBCFE6FFA0EC20F0006EB4
:1049D000050EE15C02E2E16AE552E16E0050070E6D
:1049E000F3CFDBFF080EF4CFDBFF070EDBCFE9FFD1
:1049F000080EDBCFEAFFEFCF00F0016A00BE0168CE
:104A0000020E00C0DBFFFA0EDBCFE9FFFB0EDBCFAF
:104A1000EAFFEE2A000EEF22020EDB50066E076A56
:104A2000E50E061801E1075009E0020EDB50086EA2
:104A3000096A0850091002E0000E01D0010E046E50
:104A4000056A0450051009E0D950070FE96E000E01
:104A5000DA20EA6EEE50ED1002E1000E01D0010EF8
:104A6000026E036A025003100DE0010EDB2ADB50D8
:104A70000A6E0B6AD8900B5004E6010E0A5C000E19
:104A80000B5802E3000E01D0010E006E016A0050C7
:104A900001108EE1D950070FE96E000EDA20EA6EA0
:104AA000EE50ED1050E1FC0EDBCFE9FFFD0EDBCF49
:104AB000EAFF2A0EE926000EEA22050EEECFDBFF02
:104AC000060EEDCFDBFFD950050FE96E000EDA20A0
:104AD000EA6EEE50ED1003E1020EDF6E33D0FC0EF5
:104AE000DBCFE9FFFD0EDBCFEAFF040EE926000E67
:104AF000EA22050EDBCFEEFF060EDBCFEDFF010E47
:104B0000E66EFC0EDBCFE6FFFD0EDBCFE6FF3DDA07
:104B1000E552E552E552006E016A120E001801E1FD
:104B2000015003E1020EDF6E0DD0FA0EDBCFE9FF7C
:104B3000FB0EDBCFEAFF030EDBCFEEFF040EDBCF75
:104B4000EDFFDF6A16D0010EDB50006E016A010E28
:104B5000001801E101500DE1DF6AFA0EDBCFE9FF39
:104B6000FB0EDBCFEAFF030EDBCFEEFF040EDBCF45
:104B7000EDFF07D7FA0EDBCFE9FFFB0EDBCFEAFF35
:104B8000030EDBCFEEFF040EDBCFEDFFDF50006E38
:104B9000016A0050011003E1010E03D002D0000EA3
:104BA00000D0006E090EE15C02E2E16AE552E16EBE
:104BB0000050E552E5CFDAFFE7CFD9FF1200D9CF99
:104BC000E6FFDACFE6FFE1CFD9FFE2CFDAFFE65228
:104BD000E652E652DF6AFC0EDBCFE9FFFD0EDBCFCB
:104BE000EAFF280EE926000EEA22EECF00F0EFCF12
:104BF00001F0FC0EDBCFE9FFFD0EDBCFEAFF2A0E52
:104C0000E926000EEA2200C0EEFF01C0EDFF010E12
:104C1000E66EF80EDBCFE6FFF90EDBCFE6FFFC0E0B
:104C2000DBCFE6FFFD0EDBCFE6FFA0EC20F0006E51
:104C3000050EE15C02E2E16AE552E16E0050DE52EF
:104C4000F3CFDEFFF4CFDDFFDD52D950010FE96E67
:104C5000000EDA20EA6EEE50ED1002E11C0E8CD14F
:104C60000B0EE66EE66AFA0EDBCFE6FFFB0EDBCF3D
:104C7000E6FF010EDBCFE9FF020EDBCFEAFFE9CF53
:104C800000F0EACF01F000C0E6FF01C0E6FF49EC0A
:104C9000B4F0026E060EE15C02E2E16AE552E16EFA
:104CA0000250F70EDB50006E016A120E001801E18F
:104CB00001500DE1010EDBCFE9FF020EDBCFEAFF71
:104CC0000B0EE926000EEA22100EEF6E0CD0010E3C
:104CD000DBCFE9FF020EDBCFEAFF0B0EE926000E69
:104CE000EA22200EEF6E010EDBCFE9FF020EDBCFD2
:104CF000EAFF0C0EE926000EEA22EF6A010EDBCF76
:104D0000E9FF020EDBCFEAFF140EEB6A150EEB6A29
:104D1000010EDBCFE9FF020EDBCFEAFF1A0EEB6AD2
:104D20001B0EEB6A010EDBCFE9FF020EDBCFEAFFC1
:104D30001C0EE926000EEA22EE6AEE6AEE6AEE6AC0
:104D4000010EDBCFE9FF020EDBCFEAFF0D0EE926F5
:104D5000000EEA22B20EEF6E010EDBCFE9FF020E6B
:104D6000DBCFEAFF0E0EE926000EEA22780EEE6E89
:104D7000720EED6E010EDBCFE9FF020EDBCFEAFF14
:104D8000100EE926000EEA22B00EEE6E320EED6E27
:104D9000F70EDB50006E016A120E001801E101509F
:104DA0002BE0010EDBCFE9FF020EDBCFEAFF120E94
:104DB000E926000EEA22B00EEE6E320EED6E010E06
:104DC000DBCFE9FF020EDBCFEAFF160EE926000E6D
:104DD000EA22790EEE6E720EED6E010EDBCFE9FF68
:104DE000020EDBCFEAFF180EE926000EEA22B00E13
:104DF000EE6E320EED6E1ED0010EDBCFE9FF020E1D
:104E0000DBCFEAFF120EEB6A130EEB6A010EDBCF6B
:104E1000E9FF020EDBCFEAFF160EEB6A170EEB6A14
:104E2000010EDBCFE9FF020EDBCFEAFF180EEB6AC3
:104E3000190EEB6A010EDBCFE9FF020EDBCFEAFFB2
:104E40001C0EE926000EEA22EECF00F0EECF01F0B4
:104E5000EECF02F0EFCF03F0FC0EDBCFE9FFFD0E4B
:104E6000DBCFEAFF0E0EE926000EEA2200C0EEFFBD
:104E700001C0EEFF02C0EEFF03C0EEFF010EDBCF6C
:104E8000E9FF020EDBCFEAFF0E0EE926000EEA2252
:104E9000EECF00F0EFCF01F0FC0EDBCFE9FFFD0E0F
:104EA000DBCFEAFF130EE926000EEA2200C0EEFF78
:104EB00001C0EDFF010EDBCFE9FF020EDBCFEAFF01
:104EC000100EE926000EEA22EECF00F0EFCF01F03F
:104ED000FC0EDBCFE9FFFD0EDBCFEAFF150EE92666
:104EE000000EEA2200C0EEFF01C0EDFF010EDBCF95
:104EF000E9FF020EDBCFEAFF0B0EE926000EEA22E5
:104F0000EF50E66EFC0EDBCFE9FFFD0EDBCFEAFFD4
:104F1000260EE926000EEA22E552E750EE6EED6A13
:104F2000F80EDBCFE9FFF90EDBCFEAFFEECF00F0A2
:104F3000EFCF01F0FC0EDBCFE9FFFD0EDBCFEAFF88
:104F4000220EE926000EEA2200C0EEFF01C0EDFFAE
:104F5000F80EDBCFE6FFF90EDBCFE6FFFC0EDBCF72
:104F6000E6FFFD0EDBCFE6FFD0EC1EF0E552E5528A
:104F7000E552E552DF5000D0E552E552E552E552E8
:104F8000E5CFDAFFE7CFD9FF1200D9CFE6FFDACFBE
:104F9000E6FFE1CFD9FFE2CFDAFF060EE12402E31C
:104FA000E168E652E16EFC0EDBCFE9FFFD0EDBCFE0
:104FB000EAFFEECFDEFFEDCFDDFFFC0EDBCFE9FF3A
:104FC000FD0EDBCFEAFF040EE926000EEA22020EF8
:104FD000EECFDBFF030EEDCFDBFFFC0EDBCFE6FFFA
:104FE000FD0EDBCFE6FFBBD8E552E552020EF3CF54
:104FF000DBFF030EF4CFDBFFD950020FE96E000E8A
:10500000DA20EA6EEE50ED1002E1120E9AD0DECFF9
:10501000E9FFDDCFEAFF1C0EE926000EEA22EF5081
:10502000006E016A010E001801E101501AE1E66A02
:10503000F80EE66E0F0EE66E020EDBCFE6FF030EF5
:10504000DBCFE6FFDECFE6FFDDCFE6FF00EC57F07B
:10505000006E070EE15C02E2E16AE552E16E00508B
:1050600018D0E66AF80EE66EE668020EDBCFE6FFC1
:10507000030EDBCFE6FFDECFE6FFDDCFE6FF00EC81
:1050800057F0006E070EE15C02E2E16AE552E16E64
:105090000050FC0EDBCFE9FFFD0EDBCFEAFF040E74
:1050A000E926000EEA22040EEECFDBFF050EEDCF5F
:1050B000DBFFE66A020EDBCFE6FF030EDBCFE6FF87
:1050C000040EDBCFE6FF050EDBCFE6FFDECFE6FF0B
:1050D000DDCFE6FF00EC57F0006E070EE15C02E268
:1050E000E16AE552E16E0050FC0EDBCFE9FFFD0EF8
:1050F000DBCFEAFF040EE926000EEA22020EDBCF28
:10510000EEFF030EDBCFEDFFFB0EDB50006E016AFE
:10511000010E001801E1015012E1020EDBCFE6FFA3
:10512000030EDBCFE6FFDECFE6FFDDCFE6FFA5EC2B
:105130003EF0E552E552E552E55203D002D0000EB2
:1051400000D0006E060EE15C02E2E16AE552E16E1B
:105150000050E552E5CFDAFFE7CFD9FF1200D9CFF3
:10516000E6FFDACFE6FFE1CFD9FFE2CFDAFF080EA4
:10517000E12402E3E168E652E16E020EDB6A030E0F
:10518000DB6AFC0EDBCFE9FFFD0EDBCFEAFFEECFE3
:10519000DEFFEDCFDDFFFC0EDBCFE9FFFD0EDBCF49
:1051A000EAFF040EE926000EEA22040EEECFDBFF32
:1051B000050EEDCFDBFF040EDBCF00F0050EDBCFDD
:1051C00001F0020E005C000E015807E2020EF36EC1
:1051D000040EF3CFDBFF050EDB6A040EDBCF52F0CB
:1051E000050EDBCF53F0060E52C0DBFF070E53C097
:1051F000DBFFD950040FE96E000EDA20EA6EEE50A4
:10520000ED1001E17BD0040EDBCFE6FF050EDBCF16
:10521000E6FFDECFE6FFDDCFE6FF59EC53F0E552C7
:10522000E552E552E552020EF3CFDBFF030EF4CF59
:10523000DBFFF3CF00F0F4CF01F00001001C01E12F
:10524000011C05E1040EDB6A050EDB6A57D0D9505C
:10525000020FE96E000EDA20EA6EEE50ED1001E169
:105260004DD0040EDB2A050E01E3DB2AD950040FD2
:10527000E96E000EDA20EA6EFE0EEE1802E1FF0E75
:10528000ED181BE0040EDBCF02F0050EDBCF03F0C0
:10529000046A056ADECFE9FFDDCFEAFF140EE926D6
:1052A000000EEA22EE50025CEE500358EE50045815
:1052B000EE50055802E2000E01D0010E006E016AA8
:1052C0000050011007E0020EF36E040EF3CFDBFF77
:1052D000050EDB6A040EDBCF00F0050EDBCF01F01C
:1052E000060EDB50001803E1070EDB50011805E144
:1052F000040EDB6A050EDB6A01D07BD7040EDBCF20
:1053000000F0050EDBCF01F000C0F3FF01C0F4FF99
:10531000080EE15C03E200D0E16AE552E16EE5527D
:10532000E5CFDAFFE7CFD9FF1200D9CFE6FFDACF1A
:10533000E6FFE1CFD9FFE2CFDAFF080EE12402E376
:10534000E168E652E16E480EF36E040EF3CFDBFF28
:10535000050EDB6AFC0EDBCFE9FFFD0EDBCFEAFFBB
:10536000220EE926000EEA22EECFDEFFEDCFDDFFB2
:10537000FC0EDBCFE9FFFD0EDBCFEAFF120EE926C4
:10538000000EEA22EF50010B006E016A005001107E
:1053900001E1ACD00F012A51006E016A00500110EA
:1053A00007E019EC44F0000903E0F368F468FAD070
:1053B000010EE66E000EE66EE66A000EE66EE66A26
:1053C000FC0EDBCFE9FFFD0EDBCFEAFFEECFE6FF01
:1053D000EFCFE6FF00EC57F0006E070EE15C02E253
:1053E000E16AE552E16E0050D9CFE6FFDACFE6FF81
:1053F000FC0EDBCFE6FFFD0EDBCFE6FF06EC2FF069
:10540000E552E552E552E552060EF3CFDBFF070EFB
:10541000F4CFDBFFD950060FE96E000EDA20EA6EFA
:10542000EE50ED100FE1040EDB68050EDB68040E94
:10543000DBCF00F0050EDBCF01F000C0F3FF01C0B1
:10544000F4FFB0D0060EDBCFE6FF070EDBCFE6FFA2
:10545000B5D8E552E5520000FC0EDBCFE9FFFD0EAA
:10546000DBCFEAFF0E0EE926000EEA22EECF00F0B7
:10547000EECF01F0EECF02F0EFCF03F0060EDBCF60
:10548000E9FF070EDBCFEAFF1C0EE926000EEA2239
:1054900000C0EEFF01C0EEFF02C0EEFF03C0EEFF52
:1054A000D9CFE6FFDACFE6FFFC0EDBCFE6FFFD0E3D
:1054B000DBCFE6FFD0EC1EF0E552E552E552E552B7
:1054C000000905E0040EDB6A050EDB6A04D0040E59
:1054D000DB68050EDB68FC0EDBCFE9FFFD0EDBCFE2
:1054E000EAFF120EE926000EEA22EF90020EDB6AB6
:1054F000030EDB6A020EDBCF00F0030EDBCF01F000
:10550000030E005C000E015833E2FC0EDBCF00F00E
:10551000FD0EDBCF01F0020EDBCF02F0030EDBCF7E
:1055200003F02C0E0302F3CF03F02C0E0202F3CF94
:1055300002F0F4500326000E0226020E032202504F
:10554000001802E1035001180DE1020EDBCFE9FF64
:10555000030EDBCFEAFF840EE926020EEA22010EDB
:10556000EF6E06D0020EDB2A030E01E3DB2AC2D760
:10557000D950040FE96E000EDA20EA6E480EEE18DC
:1055800001E1ED5004E1040EDB6A050EDB6A040E56
:10559000DBCF00F0050EDBCF01F000C0F3FF01C050
:1055A000F4FF00D0080EE15C02E2E16AE552E16E30
:1055B000E552E5CFDAFFE7CFD9FF1200D9CFE6FFFA
:1055C000DACFE6FFE1CFD9FFE2CFDAFF060EE12422
:1055D00002E3E168E652E16EFC0EDBCFE9FFFD0E6F
:1055E000DBCFEAFF160EE926000EEA22EECF00F02E
:1055F000EFCF01F01F0E0014DF6EFC0EDBCFE9FFD2
:10560000FD0EDBCFEAFF160EE926000EEA22EECFF2
:1056100000F0EFCF01F0E00E0016070E0116050EA8
:10562000D89001320032E804FBE1010E00C0DBFF3C
:10563000FC0EDBCFE9FFFD0EDBCFEAFF160EE926FD
:10564000000EEA22EECF00F0EFCF01F00016F80EC8
:1056500001160150016AE830E830E8301F0B006E97
:10566000020E00C0DBFFFC0EDBCFE9FFFD0EDBCF3F
:10567000EAFF180EE926000EEA22EECF00F0EFCF87
:1056800001F01F0E0016000E0116030E00C0DBFF16
:10569000FC0EDBCFE9FFFD0EDBCFEAFF180EE9269B
:1056A000000EEA22EECF00F0EFCF01F0E00E001680
:1056B000010E0116050ED89001320032E804FBE11C
:1056C000040E00C0DBFFFC0EDBCFE9FFFD0EDBCFDD
:1056D000EAFF180EE926000EEA22EECF00F0EFCF27
:1056E00001F00016FE0E011601C000F0016AD8900C
:1056F0000032050E00C0DBFFDF50006E016AD8905B
:10570000015004E61D0E005C000E015802E2DF2A83
:105710004DD0DF6A010EDB50006E016AD890015057
:1057200004E63B0E005C000E015803E2010EDB2A8A
:105730003DD0010EDB6A020EDB50006E016AD8908C
:10574000015004E6170E005C000E015803E2020E41
:10575000DB2A2CD0020EDB6A030EDB50006E016ADE
:10576000D890015004E61E0E005C000E015803E2C2
:10577000030EDB2A1BD0010EF36E030EF3CFDBFF0B
:10578000040EDB50006E016AD890015004E60C0E46
:10579000005C000E015803E2040EDB2A07D0010E64
:1057A000F36E040EF3CFDBFF050EDB2ADF50E66E4F
:1057B000FC0EDBCFE9FFFD0EDBCFEAFF160EE9267C
:1057C000000EEA22E552E750EE6EED6A010EDB5064
:1057D000006E016A050ED89000360136E804FBE140
:1057E000FC0EDBCFE9FFFD0EDBCFEAFF160EE9264C
:1057F000000EEA220050EE120150ED12020EDB50B4
:10580000006E016A0050006AE834E834E834F80BAE
:10581000016EFC0EDBCFE9FFFD0EDBCFEAFF160EBB
:10582000E926000EEA220050EE120150ED12030E9E
:10583000DB50E66EFC0EDBCFE9FFFD0EDBCFEAFFAF
:10584000180EE926000EEA22E552E750EE6EED6AE8
:10585000040EDB50006E016A050ED890003601364A
:10586000E804FBE1FC0EDBCFE9FFFD0EDBCFEAFF36
:10587000180EE926000EEA220050EE120150ED1239
:10588000050EDB50006E016A00C001F0006AD8907E
:105890000136FC0EDBCFE9FFFD0EDBCFEAFF180E71
:1058A000E926000EEA220050EE120150ED12060E1B
:1058B000E15C02E2E16AE552E16EE552E5CFDAFF32
:1058C000E7CFD9FF1200D9CFE6FFDACFE6FFE1CF6D
:1058D000D9FFE2CFDAFF0B0EE12402E3E168E652E2
:1058E000E16E0A0EDB6AFA0EDBCFE9FFFB0EDBCFBF
:1058F000EAFFEECF52F0EDCF53F052500F0B09E11B
:10590000FA0EDBCFE9FFFB0EDBCFEAFFEE50ED1026
:1059100002E1000E01D0010E006E016A005001107C
:1059200039E0FC0EDBCFE9FFFD0EDBCFEAFF280EEE
:10593000E926000EEA22EECF00F0EFCF01F0FC0ED8
:10594000DBCFE9FFFD0EDBCFEAFF2A0EE926000ED2
:10595000EA2200C0EEFF01C0EDFF010EE66EFA0E76
:10596000DBCFE6FFFB0EDBCFE6FFFC0EDBCFE6FF77
:10597000FD0EDBCFE6FFA0EC20F0006E050EE15C33
:1059800002E2E16AE552E16E0050F3CFDEFFF4CFB0
:10599000DDFF1BD0E66AFA0EDBCFE6FFFB0EDBCFA6
:1059A000E6FFFC0EDBCFE6FFFD0EDBCFE6FFA0EC53
:1059B00020F0006E050EE15C02E2E16AE552E16E64
:1059C0000050F3CFDEFFF4CFDDFFDECFE9FFDDCF08
:1059D000EAFFEFCF00F0016A00BE0168030E00C0CD
:1059E000DBFFD9CFE9FFDACFEAFFEE50ED1009E097
:1059F000030EDB50026E036A0250031002E0000E39
:105A000001D0010E006E016A0050011006E0020E86
:105A1000F36E050EF3CFDBFFE8D1030EDB50006E13
:105A2000016AE50E001801E1015006E1010EF36E76
:105A3000050EF3CFDBFFD9D1DECFE9FFDDCFEAFFE3
:105A40000B0EE926000EEA22EF50E76E030EE7CFB9
:105A5000DBFF020EDB6ADB50006E016AD89001505A
:105A600004E6080E005C000E015843E2DECFE9FFB9
:105A7000DDCFEAFFE9CF02F0EACF03F0020EDB5000
:105A80000F010224E96E000E0320EA6EEFCF00F052
:105A9000016A00BE0168040E00C0DBFFDBCFE6FF39
:105AA000E66A44ECB5F0E552E552040EF3CFDBFFB5
:105AB000DB50E66EFC0EDBCFE9FFFD0EDBCFEAFF2D
:105AC000170EE926000EEA22E9CF00F0EACF01F036
:105AD0000A0EDBCFF3FFDB2AF3500F010024E96E3F
:105AE000000E0120EA6EE552E750EF6E020EDB2A4F
:105AF000B2D7DECFE9FFDDCFEAFF0B0EE926000EBD
:105B0000EA22EF50E76E030EE7CFDBFFDECFE9FFBF
:105B1000DDCFEAFF080EE926000EEA22EFCF00F003
:105B2000016A00BE0168040E00C0DBFF020EDB6AE2
:105B3000DB50006E016AD890015004E6030E005C51
:105B4000000E015847E2DECFE9FFDDCFEAFF080E85
:105B5000E926000EEA22E9CF02F0EACF03F0020EB6
:105B6000DB500F010224E96E000E0320EA6EEFCF36
:105B700000F0016A00BE0168040E00C0DBFFDBCF4D
:105B8000E6FFE66A44ECB5F0E552E552040EF3CFC9
:105B9000DBFFDB50E66EFC0EDBCFE9FFFD0EDBCF5B
:105BA000EAFF170EE926000EEA22E9CF00F0EACF5D
:105BB00001F00A0EDBCFF3FFDB2AF3500F010024C4
:105BC000E96E000E0120EA6EE552E750EF6E020E1C
:105BD000DB2AAED7FA0EDBCFE9FFFB0EDBCFEAFF05
:105BE000EECF00F0EFCF01F0FC0EDBCFE9FFFD0EB2
:105BF000DBCFEAFF220EE926000EEA2200C0EEFF0C
:105C000001C0EDFFDECFE9FFDDCFEAFFEFCF00F00F
:105C1000016A00BE0168030E00C0DBFFDB50006EAE
:105C2000016AE50E001801E1015006E1010EF36E74
:105C3000050EF3CFDBFF02D0050EDB6ADECFE9FFF6
:105C4000DDCFEAFF1C0EE926000EEA22EECF00F0BF
:105C5000EECF01F0EECF02F0EFCF03F0FC0EDBCF82
:105C6000E9FFFD0EDBCFEAFF0E0EE926000EEA2269
:105C700000C0EEFF01C0EEFF02C0EEFF03C0EEFF6A
:105C8000DECFE9FFDDCFEAFF140EE926000EEA229F
:105C9000EECF00F0EFCF01F0060E00C0DBFF070EE5
:105CA00001C0DBFF080EDB6A090EDB6A060EDBCFE4
:105CB00000F0070EDBCF01F0080EDBCF02F0090E7B
:105CC000DBCF03F0100E1F0B07E0D8900036013633
:105CD00002360336E806F9E1060E00C0DBFF070EC8
:105CE00001C0DBFF080E02C0DBFF090E03C0DBFFB3
:105CF000DECFE9FFDDCFEAFF1A0EE926000EEA2229
:105D0000EECF00F0EFCF01F0026A036AD950060F20
:105D1000E96E000EDA20EA6E0050EE120150EE122B
:105D20000250EE120350EE12FC0EDBCFE9FFFD0E27
:105D3000DBCFEAFF020EE926000EEA22060EDBCFD9
:105D4000EEFF070EDBCFEDFFDECFE9FFDDCFEAFF91
:105D5000160EE926000EEA22EECF00F0EFCF01F09A
:105D6000FC0EDBCFE9FFFD0EDBCFEAFF130EE926C9
:105D7000000EEA2200C0EEFF01C0EDFFDECFE9FF1A
:105D8000DDCFEAFF180EE926000EEA22EECF00F082
:105D9000EFCF01F0FC0EDBCFE9FFFD0EDBCFEAFF1A
:105DA000150EE926000EEA2200C0EEFF01C0EDFF4D
:105DB000DECFE9FFDDCFEAFF0B0EE926000EEA2277
:105DC000EF50E76E030EE7CFDBFFDB50E66EFC0E15
:105DD000DBCFE9FFFD0EDBCFEAFF260EE926000E42
:105DE000EA22E552E750EE6EED6A050EDB50006EDA
:105DF0000B0EE15C03E200D0E16AE552E16E005077
:105E0000E552E5CFDAFFE7CFD9FF1200D9CFE6FFA1
:105E1000DACFE6FFE1CFD9FFE2CFDAFFE652E65272
:105E2000E652FC0EDBCFE9FFFD0EDBCFEAFF280ECA
:105E3000E926000EEA22EECF00F0EFCF01F0FC0ED3
:105E4000DBCFE9FFFD0EDBCFEAFF2A0EE926000ECD
:105E5000EA2200C0EEFF01C0EDFF010EE66EFA0E71
:105E6000DBCFE6FFFB0EDBCFE6FFFC0EDBCFE6FF72
:105E7000FD0EDBCFE6FFA0EC20F0006E050EE15C2E
:105E800002E2E16AE552E16E0050F3CFDEFFF4CFAB
:105E9000DDFFD9CFE9FFDACFEAFFEE50ED1003E1E5
:105EA000F36AF46A81D0DECFE9FFDDCFEAFFEFCFFE
:105EB00000F0016A00BE0168020E00C0DBFFDB508B
:105EC000006E016A0050011002E1DE6ADD6AD9CF7E
:105ED000E9FFDACFEAFFEE50ED105DE0020EDB5095
:105EE000006E016AE50E001801E1015003E1DE6A6F
:105EF000DD6A51D0DECFE9FFDDCFEAFF0B0EE926E8
:105F0000000EEA22EF50E76E020EE7CFDBFFDB5018
:105F1000006E016A0F0E001801E101503CE1FA0E1B
:105F2000DBCFE9FFFB0EDBCFEAFFEE2A000EEF220C
:105F3000E66AFA0EDBCFE6FFFB0EDBCFE6FFFC0ED8
:105F4000DBCFE6FFFD0EDBCFE6FFA0EC20F0006E1E
:105F5000050EE15C02E2E16AE552E16E0050F3CF2A
:105F6000DEFFF4CFDDFFD9CFE9FFDACFEAFFEE5055
:105F7000ED1003E1F36AF46A17D0DECFE9FFDDCF5D
:105F8000EAFF0B0EE926000EEA22EF50E76E020E42
:105F9000E7CFDBFFBCD7DECF00F0DDCF01F000C0E4
:105FA000F3FF01C0F4FF00D0E552E552E552E5529F
:105FB000E5CFDAFFE7CFD9FF1200D9CFE6FFDACF7E
:105FC000E6FFE1CFD9FFE2CFDAFF080EE12402E3DA
:105FD000E168E652E16E030EDB6AFC0EDBCFE9FFFF
:105FE000FD0EDBCFEAFF060EEECFDBFF070EEDCF97
:105FF000DBFFFC0EDBCFE9FFFD0EDBCFEAFF280E57
:10600000E926000EEA22040EEECFDBFF050EEDCFEF
:10601000DBFFFC0EDBCFE9FFFD0EDBCFEAFF2A0E34
:10602000E926000EEA22040EDBCFEEFF050EDBCFE1
:10603000EDFF010EE66EFA0EDBCFE6FFFB0EDBCFC7
:10604000E6FFFC0EDBCFE6FFFD0EDBCFE6FFA0ECAC
:1060500020F0006E050EE15C02E2E16AE552E16EBD
:106060000050F3CFDEFFF4CFDDFFD9CFE9FFDACF69
:10607000EAFFEE50ED1002E11C0EB8D0DECFE9FFD2
:10608000DDCFEAFFEFCF00F0016A00BE0168020E2B
:1060900000C0DBFFD9CFE9FFDACFEAFFEE50ED1009
:1060A00009E0020EDB50026E036A0250031002E0A8
:1060B000000E01D0010E006E016A0050011006E0D2
:1060C0000A0EF36E030EF3CFDBFF88D0020EDB5017
:1060D000006E016AE50E001801E1015006E10A0EAA
:1060E000F36E030EF3CFDBFF79D0DECFE9FFDDCF18
:1060F000EAFF0B0EE926000EEA22EF50E76E020ED1
:10610000E7CFDBFFDECFE9FFDDCFEAFFE50EEF6E85
:10611000DECFE9FFDDCFEAFF1A0EE926000EEA2204
:10612000040EEECFDBFF050EEDCFDBFF030EDBCF62
:1061300002F0036A02BE03680250031016E1FA0E71
:10614000DBCFE6FFFB0EDBCFE6FFFC0EDBCFE6FF8F
:10615000FD0EDBCFE6FFD0EC1EF0E552E552E55236
:10616000E552000902E0000E01D0010E006E016A46
:106170000050011006E0010EF36E030EF3CFDBFFBB
:106180002DD0D950040FE96E000EDA20EA6EEE50E1
:10619000ED1024E0F90EDB50006E016A0050011092
:1061A0001DE0060EDBCFE6FF070EDBCFE6FF040E99
:1061B000DBCFE6FF050EDBCFE6FF9FEC1FF0E552DD
:1061C000E552E552E552000903E0006A016A03D096
:1061D000010E006E016A030E00C0DBFF030EDBCF71
:1061E00000F0016A00BE0168005000D0006E080E89
:1061F000E15C02E2E16AE552E16E0050E552E5CF72
:10620000DAFFE7CFD9FF1200D9CFE6FFDACFE6FFFA
:10621000E1CFD9FFE2CFDAFF1B0EE12402E3E16810
:10622000E652E16E010EDB6AF36E0E0EF3CFDBFF7A
:106230000F0EDB6AD950FA0FE96EFF0EDA20EA6E14
:10624000EE50ED1002E0A8EF35F02CCFE9FF2DCF96
:10625000EAFF280EE926000EEA22EE50ED1004E1D6
:10626000F368F468D8EF37F0DF6ADF50026E036A34
:10627000D890035004E60B0E025C000E035814E2A3
:10628000DF50E76EFC0EDBCFE9FFFD0EDBCFEAFF50
:10629000E750E926000EEA22EFCF04F0056A04BEBB
:1062A00005680450051002E1000E01D0010E006ED9
:1062B000016A0050011022E0DF50E76EFC0EDBCFD8
:1062C000E9FFFD0EDBCFEAFFE750E926000EEA22E8
:1062D000EFCF02F0036A02BE0368D950020F006ECE
:1062E000000EDA20016EDF500F010024E96E000E6F
:1062F0000120EA6E02C0EFFFDF2AB7D7DF50006E41
:10630000016AD890015004E60B0E005C000E0158A3
:1063100011E2D950020F006E000EDA20016EDF503C
:10632000DF2A0F010024E96E000E0120EA6E200E24
:10633000EF6EE4D7E66AD950020FE66E000EDA205F
:10634000E66EB1EC7BF0E552E552E5522CCFE9FF69
:106350002DCFEAFF280EE926000EEA22140EEECF1A
:10636000DBFF150EEDCFDBFF2CCFE9FF2DCFEAFFD2
:10637000280EE926000EEA22EECF00F0EFCF01F062
:106380002CCFE9FF2DCFEAFF2A0E00C0EBFF2B0E2A
:1063900001C0EBFF010EE66ED9500E0FE66E000E47
:1063A000DA20E66E2CCFE6FF2DCFE6FFA0EC20F042
:1063B000006E050EE15C02E2E16AE552E16E00501A
:1063C000120EF3CFDBFF130EF4CFDBFF120EDBCF89
:1063D000E9FF130EDBCFEAFF1A0EE926000EEA22D0
:1063E000EECF00F0EFCF01F02CCFE9FF2DCFEAFF89
:1063F0002A0E00C0EBFF2B0E01C0EBFF120EDBCF0D
:10640000E9FF130EDBCFEAFF1A0EE926000EEA229F
:10641000EECF00F0EFCF01F02CCFE9FF2DCFEAFF58
:10642000280E00C0EBFF290E01C0EBFF0E0EDB6A49
:106430000F0EDB6A010EE66ED9500E0FE66E000EEF
:10644000DA20E66E2CCFE6FF2DCFE6FFA0EC20F0A1
:10645000006E050EE15C02E2E16AE552E16E005079
:10646000120EF3CFDBFF130EF4CFDBFFD950120F68
:10647000E96E000EDA20EA6EEE50ED1004E1F368EA
:10648000F468D8EF37F0DF6ADF50006E016AD89009
:10649000015004E60B0E005C000E015832E2120EB1
:1064A000DBCFE9FF130EDBCFEAFFE9CF02F0EACF43
:1064B00003F0DF500F010224E96E000E0320EA6EA4
:1064C000EFCF00F0016A00BE0168D950020F066EDE
:1064D000000EDA20076EDF500624E96E000E07205A
:1064E000EA6EEFCF04F0056A04BE05680450001898
:1064F00002E10550011803E0DE52010EDD6EDF2AD5
:10650000C3D7010EDB50006E016A0050011005E197
:10651000F368F468D8EF37F002D0010EDB6A120E90
:10652000DBCFE9FF130EDBCFEAFF1A0EE926000EE0
:10653000EA22EECF02F0EFCF03F0140EDB50021888
:1065400003E1150EDB50031867E1120EDBCFE9FF04
:10655000130EDBCFEAFF1A0EE926000EEA22EECF79
:1065600006F0EFCF07F0140EDB50061803E1150E0E
:10657000DB50071847E1120EDBCFE9FF130EDBCF2C
:10658000EAFFEFCF0EF00F6A0EBE0F680E500C6ED2
:106590000D6AE50E0C1801E10D5014E0120EDBCF70
:1065A000E9FF130EDBCFEAFF0B0EE926000EEA220D
:1065B000EF50106E116A080E101801E1115002E040
:1065C000000E01D0010E0A6E0B6A0A500B1014E186
:1065D000120EDBCFE9FF130EDBCFEAFF0B0EE9262D
:1065E000000EEA22EF50126E136A0F0E121801E12C
:1065F000135002E0000E01D0010E086E096A085027
:10660000091002E1000E01D0010E046E056A04506B
:10661000051002E1000E01D0010E006E016A00506B
:10662000011001E17AD0E66AD9500E0FE66E000E35
:10663000DA20E66E2CCFE6FF2DCFE6FFA0EC20F0AF
:10664000006E050EE15C02E2E16AE552E16E005087
:10665000120EF3CFDBFF130EF4CFDBFFD950120F76
:10666000E96E000EDA20EA6EEE50ED1004E1F368F8
:10667000F468D8EF37F0DF6ADF50006E016AD89017
:10668000015004E60B0E005C000E015832E2120EBF
:10669000DBCFE9FF130EDBCFEAFFE9CF02F0EACF51
:1066A00003F0DF500F010224E96E000E0320EA6EB2
:1066B000EFCF00F0016A00BE0168D950020F066EEC
:1066C000000EDA20076EDF500624E96E000E072068
:1066D000EA6EEFCF04F0056A04BE056804500018A6
:1066E00002E10550011803E0DE52010EDD6EDF2AE3
:1066F000C3D7010EDB50006E016A0050011005E1A6
:10670000F368F468D8EF37F002D0010EDB6A0E0EA2
:10671000DB2A0F0E01E3DB2A02D70E0EDB060F0E7B
:1067200001E2DB060E0EDBCF00F0DB2A0F0EDBCF23
:1067300001F001E3DB2A100E00C0DBFF110E01C0E7
:10674000DBFFE66AD9500E0FE66E000EDA20E66E29
:106750002CCFE6FF2DCFE6FFA0EC20F0006E050E5B
:10676000E15C02E2E16AE552E16E0050120EF3CF05
:10677000DBFF130EF4CFDBFFD950120FE96E000ED2
:10678000DA20EA6EEE50ED1004E1F368F468D8EF19
:1067900037F0120EDBCFE9FF130EDBCFEAFFEFCFAE
:1067A00000F0016A00BE01680050011035E1100ED2
:1067B000DBCF52F0110EDBCF53F00E0E52C0DBFFD9
:1067C0000F0E53C0DBFF2CCFE9FF2DCFEAFF280EC1
:1067D000E926000EEA22EECF00F0EFCF01F02CCF39
:1067E000E9FF2DCFEAFF2A0E00C0EBFF2B0E01C000
:1067F000EBFF010EE66ED9500E0FE66E000EDA20AA
:10680000E66E2CCFE6FF2DCFE6FFA0EC20F0006E69
:10681000050EE15C54E251D0DF6ADF50006E016A80
:10682000D890015004E60B0E005C000E015832E2D5
:10683000120EDBCFE9FF130EDBCFEAFFE9CF02F048
:10684000EACF03F0DF500F010224E96E000E0320AF
:10685000EA6EEFCF00F0016A00BE0168D950020F66
:10686000066E000EDA20076EDF500624E96E000E79
:106870000720EA6EEFCF04F0056A04BE05680450F5
:10688000001802E10550011803E0DE52010EDD6E32
:10689000DF2AC3D7010EDB50006E016A00500110E1
:1068A00004E1F368F46884D302D0010EDB6A0E0EB3
:1068B000DB2A0F0E01E3DB2A44D7E16AE552E16EE1
:1068C0000050120EF3CFDBFF130EF4CFDBFFDF6AB5
:1068D000DF50006E016AD890015004E60B0E005C98
:1068E000000E01584BE2D950020F046E000EDA2060
:1068F000056EDF500F010424E96E000E0520EA6EDC
:10690000EFCF02F0036A02BE03682CCFE9FF2DCF60
:10691000EAFF170EE926000EEA22E9CF00F0EACFDF
:1069200001F0DF500024E96E000E0120EA6E02C083
:10693000EFFFD950020F046E000EDA20056EDF5013
:106940000424E96E000E0520EA6EEFCF02F0036A20
:1069500002BE0368120EDBCFE9FF130EDBCFEAFFA6
:10696000E9CF00F0EACF01F0DF500024E96E000E1D
:106970000120EA6E02C0EFFFDF2AAAD72CCFE9FF81
:106980002DCFEAFF2A0EE926000EEA22EECFE6FF1F
:10699000EFCFE6FF2CCFE9FF2DCFEAFFEECFE6FFEA
:1069A000EFCFE6FF79EC3FF0E552E552E552E552D4
:1069B000160E50C0DBFF170E51C0DBFF180E52C081
:1069C000DBFF190E53C0DBFF0E0EDBCF00F00F0E06
:1069D000DBCF01F0040ED89001320032E804FBE175
:1069E0001A0E00C0DBFF2CCFE9FF2DCFEAFF280EE7
:1069F000E926000EEA22EE50ED1026E02CCFE9FF4A
:106A00002DCFEAFFEE50EFCFEAFFE96E1B0EE9262D
:106A1000000EEA22EF50026E036A1A0EDB50006E7F
:106A2000016A00C052F001C053F002C057F003C029
:106A300058F0B6ECB2F003AE04D04E6C4F1E000E10
:106A40004F221A0E4EC0DBFFE66A2CCFE9FF2DCF96
:106A5000EAFFEE50EFCFEAFFE96EEECFE6FFEFCFB1
:106A6000E6FF1A0EDB50026E036A046A056A03AE83
:106A700002D004680568D950160FE96E000EDA20BE
:106A8000EA6EEE500226EE500322EE500422EE5043
:106A9000052202C0E6FF03C0E6FF04C0E6FF05C012
:106AA000E6FF19ECA4F0066E070EE15C02E2E16A73
:106AB000E552E16E0650006E016A0050011003E1DC
:106AC000F368F46875D2DF6AD950020F046E000EC5
:106AD000DA20056EDF500F010424E96E000E052058
:106AE000EA6EEFCF02F0036A02BE0368200E0218BE
:106AF00001E103500BE0DF50066E076AD8900750A3
:106B000004E60B0E065C000E075802E3000E01D0EF
:106B1000010E006E016A0050011002E0DF2AD4D796
:106B2000D950020F006E000EDA20016EDF500024F3
:106B3000E96E000E0120EA6EEF6AD950020FE66E90
:106B4000000EDA20E66EECEC5AF0E552E5522DD25A
:106B5000E66AFA0EDBCFE9FFFB0EDBCFEAFF170E8A
:106B6000E926000EEA22E9CF02F0EACF03F002C0E4
:106B7000E6FF03C0E6FFFC0EDBCFE6FFFD0EDBCF3A
:106B8000E6FFD3EC47F0046E050EE15C02E2E16A39
:106B9000E552E16E0450006E016A0050011004E1FC
:106BA000F368F46805D201D2DF6ADF50006E016A33
:106BB000D890015004E60B0E005C000E01582AE24A
:106BC000FA0EDBCFE9FFFB0EDBCFEAFF170EE9265B
:106BD000000EEA22E9CF04F0EACF05F0DF500F0102
:106BE0000424E96E000E0520EA6EEFCF02F0036A7E
:106BF00002BE0368D950020F006E000EDA20016E4B
:106C0000DF500024E96E000E0120EA6E02C0EFFFA3
:106C1000DF2ACBD7FA0EDBCFE9FFFB0EDBCFEAFF93
:106C2000220EE926000EEA22100EEECFDBFF110E37
:106C3000EDCFDBFF0E0EDB6A0F0EDB6AFA0EDBCF49
:106C4000E9FFFB0EDBCFEAFF280EE926000EEA2261
:106C5000EECF00F0EFCF01F0FA0EDBCFE9FFFB0E35
:106C6000DBCFEAFF2A0EE926000EEA2200C0EEFF83
:106C700001C0EDFF010EE66ED9500E0FE66E000E5C
:106C8000DA20E66EFA0EDBCFE6FFFB0EDBCFE6FF87
:106C9000A0EC20F0006E050EE15C02E2E16AE55234
:106CA000E16E0050120EF3CFDBFF130EF4CFDBFFCB
:106CB000D950120FE96E000EDA20EA6EEE50ED1098
:106CC00003E1F368F46874D1DF6ADF50006E016A93
:106CD000D890015004E60B0E005C000E015832E221
:106CE000120EDBCFE9FF130EDBCFEAFFE9CF02F094
:106CF000EACF03F0DF500F010224E96E000E0320FB
:106D0000EA6EEFCF00F0016A00BE0168D950020FB1
:106D1000066E000EDA20076EDF500624E96E000EC4
:106D20000720EA6EEFCF04F0056A04BE0568045040
:106D3000001802E10550011803E0DE52010EDD6E7D
:106D4000DF2AC3D7010EDB50006E016A005001102C
:106D500004E1F368F4682CD102D0010EDB6AE66A24
:106D6000D9500E0FE66E000EDA20E66EFA0EDBCF7B
:106D7000E6FFFB0EDBCFE6FFA0EC20F0006E050E79
:106D8000E15C02E2E16AE552E16E0050120EF3CFDF
:106D9000DBFF130EF4CFDBFFD950120FE96E000EAC
:106DA000DA20EA6EEE50ED1003E1F368F46800D1EA
:106DB000120EDBCFE9FF130EDBCFEAFFEFCF00F0BF
:106DC000016A00BE01680050011001E151D0DF6A84
:106DD000DF50006E016AD890015004E60B0E005C93
:106DE000000E015832E2120EDBCFE9FF130EDBCFAB
:106DF000EAFFE9CF02F0EACF03F0DF500F010224EF
:106E0000E96E000E0320EA6EEFCF00F0016A00BECB
:106E10000168D950020F066E000EDA20076EDF50AF
:106E20000624E96E000E0720EA6EEFCF04F0056A33
:106E300004BE05680450001802E10550011803E083
:106E4000DE52010EDD6EDF2AC3D7010EDB50006E6D
:106E5000016A0050011004E1F368F468A9D002D07F
:106E6000010EDB6A0E0EDB2A0F0E01E3DB2A77D759
:106E7000100EDBCF52F0110EDBCF53F00E0E52C0CE
:106E8000DBFF0F0E53C0DBFFFA0EDBCFE9FFFB0E7B
:106E9000DBCFEAFF280EE926000EEA22EECF00F053
:106EA000EFCF01F0FA0EDBCFE9FFFB0EDBCFEAFFFD
:106EB0002A0EE926000EEA2200C0EEFF01C0EDFF17
:106EC000D9500E0FE66E000EDA20E66EFA0EDBCF1A
:106ED000E6FFFB0EDBCFE6FF06EC2FF0E552E552B6
:106EE000E552E552120EF3CFDBFF130EF4CFDBFFBA
:106EF000D950120FE96E000EDA20EA6EEE50ED1056
:106F000003E1F368F46854D0DF6ADF50006E016A71
:106F1000D890015004E60B0E005C000E01582EE2E2
:106F2000FA0EDBCFE9FFFB0EDBCFEAFF170EE926F7
:106F3000000EEA22E9CF04F0EACF05F0DF500F019E
:106F40000424E96E000E0520EA6EEFCF02F0036A1A
:106F500002BE0368120EDBCFE9FF130EDBCFEAFFA0
:106F6000E9CF00F0EACF01F0DF500024E96E000E17
:106F70000120EA6E02C0EFFFDF2AC7D7D9500E0FFB
:106F8000E66E000EDA20E66EFA0EDBCFE6FFFB0EB1
:106F9000DBCFE6FFD0EC1EF0E552E552E552E552BC
:106FA000000903E1F368F46803D0F36AF46A00D0DF
:106FB0001B0EE15C02E2E16AE552E16EE552E5CFCB
:106FC000DAFFE7CFD9FF1200D9CFE6FFDACFE6FF2D
:106FD000E1CFD9FFE2CFDAFF340EE12402E3E1682A
:106FE000E652E16E06ECA5F0000903E0F36AF46AEC
:106FF000BAD3DE6ADD6A020EDB6A030EDB6A020EBA
:10700000DBCF00F0030EDBCF01F0D890015004E697
:10701000030E005C000E015839E2020EDBCFE9FFDF
:10702000030EDBCFEAFF840EE926020EEA22EF50C0
:10703000006E016A0050011023E0020EDBCFE9FF71
:10704000030EDBCFEAFF840EE926020EEA22EF6A86
:10705000020EDBCF00F0030EDBCF01F02C0E01029D
:10706000F3CF01F00002F3CF00F0F4500126000E40
:107070000026020E012200C0DEFF01C0DDFF06D0A7
:10708000020EDB2A030E01E3DB2AB9D7D9CFE9FFD1
:10709000DACFEAFFEE50ED1003E1F36AF46A63D34E
:1070A000E66ADECFE9FFDDCFEAFF170EE926000E24
:1070B000EA22E9CF00F0EACF01F000C0E6FF01C00C
:1070C000E6FFFC0EDBCFE6FFFD0EDBCFE6FFD3ECE9
:1070D00047F0026E050EE15C02E2E16AE552E16E04
:1070E000025000090FE1020EDBCFE9FF030EDBCFF8
:1070F000EAFF840EE926020EEA22010EEF6EF36A21
:10710000F46A31D3FA0EDBCFE9FFFB0EDBCFEAFFE7
:10711000EFCF00F0016A00BE0168300E00C0DBFF57
:10712000DECFE9FFDDCFEAFFBE0EEE6E020EED6EA2
:10713000DECFE9FFDDCFEAFF020EEB6A030EEB6A5A
:10714000DECFE9FFDDCFEAFF040EEB6A050EEB6A46
:10715000DECFE9FFDDCFEAFF220EEB6A230EEB6AFA
:10716000DECFE9FFDDCFEAFF260EE926000EEA2298
:10717000200EEE6EED6A2CCFE9FF2DCFEAFF280E30
:10718000E926000EEA22EECF00F0EFCF01F0DECFCD
:10719000E9FFDDCFEAFF280EE926000EEA2200C053
:1071A000EEFF01C0EDFF2CCFE9FF2DCFEAFF2A0E45
:1071B000E926000EEA22EECF00F0EFCF01F0DECF9D
:1071C000E9FFDDCFEAFF2A0EE926000EEA2200C021
:1071D000EEFF01C0EDFFDECFE6FFDDCFE6FFD950C9
:1071E000040FE66E000EDA20E66E6DEC3DF0E5521F
:1071F000E552E552E552E66A010EE66ED950040FFB
:10720000E66E000EDA20E66EDECFE6FFDDCFE6FFAB
:10721000F4EC08F0026E060EE15C02E2E16AE5526F
:10722000E16E0250006E016A00BE0168005001105C
:1072300001E0C9D1300EDB50006E016A520E001819
:1072400001E1015001E195D1720E001801E10150F8
:1072500001E18FD1410E001801E1015001E19FD001
:10726000610E001801E1015001E199D0770E00187C
:1072700001E1015008E0570E001801E1015003E060
:10728000330EDB689FD1DECFE9FFDDCFEAFF220EB0
:10729000E926000EEA22310EEECFDBFF320EEDCFF3
:1072A000DBFF010EE66ED950310FE66E000EDA20DC
:1072B000E66EDECFE6FFDDCFE6FFDDEC2FF0006E01
:1072C000050EE15C02E2E16AE552E16E0050E76E14
:1072D000330EE7CFDBFFDBCF00F0016A00BE0168B1
:1072E000005001105BE1E66AD950310FE66E000EE6
:1072F000DA20E66EDECFE6FFDDCFE6FF22EC23F0FC
:10730000006E050EE15C02E2E16AE552E16E0050BA
:10731000E76E330EE7CFDBFFDBCF00F0016A00BE84
:107320000168005001103AE1770EE66ED950310F36
:10733000E66E000EDA20E66EDECFE6FFDDCFE6FF7A
:1073400033EC0CF0006E050EE15C02E2E16AE552FE
:10735000E16E0050E76E330EE7CFDBFFDBCF00F0CE
:10736000016A00BE01680050011018E1020EE66ECD
:10737000E66AE66AE66AE66AE66ADECFE6FFDDCF3F
:10738000E6FFDCEC4DF0006E080EE15C02E2E16A23
:10739000E552E16E0050330EF3CFDBFF13D1DECFA9
:1073A000E9FFDDCFEAFF0E0EE926000EEA22EECF5E
:1073B00000F0EECF01F0EECF02F0EFCF03F000507F
:1073C00001100210031049E0DECFE9FFDDCFEAFF34
:1073D000220EE926000EEA22310EEECFDBFF320E3E
:1073E000EDCFDBFF770EE66ED950310FE66E000E63
:1073F000DA20E66EDECFE6FFDDCFE6FF33EC0CF001
:10740000006E050EE15C02E2E16AE552E16E0050B9
:10741000E76E330EE7CFDBFFDBCF00F0016A00BE83
:1074200001680050011018E1020EE66EE66AE66A95
:10743000E66AE66AE66ADECFE6FFDDCFE6FFDCEC71
:107440004DF0006E080EE15C02E2E16AE552E16E89
:107450000050330EF3CFDBFF8BD0DECFE9FFDDCF63
:10746000EAFF220EE926000EEA22310EEECFDBFF04
:10747000320EEDCFDBFF010EE66ED950310FE66E16
:10748000000EDA20E66EDECFE6FFDDCFE6FFDDECB4
:107490002FF0006E050EE15C02E2E16AE552E16E5A
:1074A0000050E76E330EE7CFDBFFDBCF00F0016A61
:1074B00000BE0168005001105BE1E66AD950310F4F
:1074C000E66E000EDA20E66EDECFE6FFDDCFE6FFE9
:1074D00022EC23F0006E050EE15C02E2E16AE55267
:1074E000E16E0050E76E330EE7CFDBFFDBCF00F03D
:1074F000016A00BE0168005001103AE1770EE66EA5
:10750000D950310FE66E000EDA20E66EDECFE6FFD0
:10751000DDCFE6FF33EC0CF0006E050EE15C02E21D
:10752000E16AE552E16E0050E76E330EE7CFDBFF14
:10753000DBCF00F0016A00BE01680050011018E1C5
:10754000020EE66EE66AE66AE66AE66AE66ADECF9A
:10755000E6FFDDCFE6FFDCEC4DF0006E080EE15CEF
:1075600002E2E16AE552E16E0050330EF3CFDBFF39
:1075700029D0DECFE9FFDDCFEAFF220EE926000E9B
:10758000EA22310EEECFDBFF320EEDCFDBFF720EC3
:10759000E66ED950310FE66E000EDA20E66EDECFD1
:1075A000E6FFDDCFE6FF33EC0CF0006E050EE15C8C
:1075B00002E2E16AE552E16E0050E76E330EE7CF7A
:1075C000DBFF00D0B0D0D950040FE66E000EDA20F9
:1075D000E66EDECFE6FFDDCFE6FF7FDAE552E5526D
:1075E000E552E552300EDB50066E076A770E06183C
:1075F00001E107500BE0300EDB50086E096A570EB0
:10760000081801E1095002E0000E01D0010E046EDD
:10761000056A045005100BE1300EDB500A6E0B6A50
:10762000610E0A1801E10B5002E0000E01D0010EBC
:10763000026E036A025003100BE1300EDB500C6E39
:107640000D6A410E0C1801E10D5002E0000E01D050
:10765000010E006E016A0050011060E0310EDB6A1D
:10766000320EDB6AE66AD950310FE66E000EDA2080
:10767000E66EDECFE6FFDDCFE6FF22EC23F0006E04
:10768000050EE15C02E2E16AE552E16E0050E76E50
:10769000330EE7CFDBFFDBCF00F0016A00BE0168ED
:1076A000005001103AE1770EE66ED950310FE66EC8
:1076B000000EDA20E66EDECFE6FFDDCFE6FF33EC2C
:1076C0000CF0006E050EE15C02E2E16AE552E16E4B
:1076D0000050E76E330EE7CFDBFFDBCF00F0016A2F
:1076E00000BE01680050011018E1020EE66EE66A65
:1076F000E66AE66AE66AE66ADECFE6FFDDCFE6FF27
:10770000DCEC4DF0006E080EE15C02E2E16AE5524D
:10771000E16E0050330EF3CFDBFF05D00A0EF36E9F
:10772000330EF3CFDBFF330EDBCF00F0016A00BE78
:107730000168005001100EE0020EDBCFE9FF030EDE
:10774000DBCFEAFF840EE926020EEA22010EEF6E7D
:10775000DE6ADD6ADECF00F0DDCF01F000C0F3FFAE
:1077600001C0F4FF00D0340EE15C02E2E16AE552B0
:10777000E16EE552E5CFDAFFE7CFD9FF1200D9CFAE
:10778000E6FFDACFE6FFE1CFD9FFE2CFDAFFFC0E6A
:10779000DBCFE9FFFD0EDBCFEAFF0A0EE926000E84
:1077A000EA22EECF00F0EECF01F0EECF02F0EFCF05
:1077B00003F000C050F001C051F002C052F003C00D
:1077C00053F000D0E552E5CFDAFFE7CFD9FF120042
:1077D000D9CFE6FFDACFE6FFE1CFD9FFE2CFDAFF7C
:1077E0005B0EE12402E3E168E652E16ED9CF00F0DE
:1077F000DACF01F0580E00C0DBFF590E01C0DBFFED
:1078000006ECA5F0000903E0F368F46801D1E66A2C
:10781000580EDBCFE9FF590EDBCFEAFF170EE92642
:10782000000EEA22E9CF00F0EACF01F000C0E6FF47
:1078300001C0E6FFFC0EDBCFE6FFFD0EDBCFE6FF6F
:10784000D3EC47F0026E050EE15C02E2E16AE5521C
:10785000E16E0250000903E1F368F468D9D0580ED4
:10786000DBCFE9FF590EDBCFEAFFBE0EEE6E020E54
:10787000ED6E580EDBCFE9FF590EDBCFEAFF020EAB
:10788000EB6A030EEB6A580EDBCFE9FF590EDBCF34
:10789000EAFF040EEB6A050EEB6A580EDBCFE9FF38
:1078A000590EDBCFEAFF220EEB6A230EEB6A580E6D
:1078B000DBCFE9FF590EDBCFEAFF260EE926000EEB
:1078C000EA22200EEE6EED6A2CCFE9FF2DCFEAFF03
:1078D000280EE926000EEA22EECF00F0EFCF01F0ED
:1078E000580EDBCFE9FF590EDBCFEAFF280EE92661
:1078F000000EEA2200C0EEFF01C0EDFF2CCFE9FF31
:107900002DCFEAFF2A0EE926000EEA22EECF00F084
:10791000EFCF01F0580EDBCFE9FF590EDBCFEAFFC6
:107920002A0EE926000EEA2200C0EEFF01C0EDFF9C
:10793000580EDBCFE6FF590EDBCFE6FFD9502C0FF8
:10794000E66E000EDA20E66EC8D8E552E552E55242
:10795000E552E66A010EE66ED9502C0FE66E000E77
:10796000DA20E66E580EDBCFE6FF590EDBCFE6FFDE
:10797000F4EC08F0006E060EE15C02E2E16AE5520A
:10798000E16E0050E76E5A0EE7CFDBFFDBCF00F071
:10799000016A00BE01680050011003E0F368F4685A
:1079A00037D0010EE66E580EDBCFE9FF590EDBCF64
:1079B000EAFF220EE926000EEA22E9CF00F0EACF24
:1079C00001F000C0E6FF01C0E6FF580EDBCFE6FF86
:1079D000590EDBCFE6FFDDEC2FF0026E050EE15C09
:1079E00002E2E16AE552E16E0250E76E5A0EE7CF1D
:1079F000DBFFDBCF00F0016A00BE01680050011020
:107A000004E1F36AF46A04D003D0F368F46800D0A8
:107A10005B0EE15C02E2E16AE552E16EE552E5CF20
:107A2000DAFFE7CFD9FF1200D9CFE6FFDACFE6FFC2
:107A3000E1CFD9FFE2CFDAFF0F012A51006E016AD0
:107A40000050011002E019EC44F0FC0EDBCFE9FF1E
:107A5000FD0EDBCFEAFF0A0EE926000EEA22EE6AEF
:107A6000EE6AEE6AEE6AFC0EDBCFE9FFFD0EDBCFBD
:107A7000EAFF080EEB6A090EEB6AFC0EDBCFE9FFAA
:107A8000FD0EDBCFEAFF060EEB6A070EEB6AFC0E7B
:107A9000DBCFE9FFFD0EDBCFEAFF020EE926000E89
:107AA000EA22EECF00F0EFCF01F0FC0EDBCFE9FFD2
:107AB000FD0EDBCFEAFF040EE926000EEA2200C02D
:107AC000EEFF01C0EDFF0F01246B256B00D0E552E6
:107AD000E5CFDAFFE7CFD9FF1200D9CFE6FFDACF43
:107AE000E6FFE1CFD9FFE2CFDAFF060EE12402E3A1
:107AF000E168E652E16EFC0EDBCF52F0FD0EDBCF0B
:107B000053F0020E52C0DBFF030E53C0DBFFFA0E30
:107B1000DBCF52F0FB0EDBCF53F0040E52C0DBFF85
:107B2000050E53C0DBFFDE522C0EDD6EDF6ADF5028
:107B3000006E016A010EDB50000101AE02D0D89048
:107B400003D0005C000E01581FE2DF50E76E040E08
:107B5000DBCFE9FF050EDBCFEAFFE750E926000E99
:107B6000EA22EF50E66EDF50E76E020EDBCFE9FF50
:107B7000030EDBCFEAFFE750E926000EEA22E552CA
:107B8000E750EF6EDF2AD3D7060EE15C02E2E16A2E
:107B9000E552E16EE552E5CFDAFFE7CFD9FF1200FB
:107BA000D9CFE6FFDACFE6FFE1CFD9FFE2CFDAFFA8
:107BB000E652E652E652020EDB6AFC0EDBCFE9FF2C
:107BC000FD0EDBCFEAFFEECFDEFFEDCFDDFFFC0EDB
:107BD000DBCFE6FFFD0EDBCFE6FFAFEC28F0E55292
:107BE000E552F3CF00F0F4CF01F0FA0EDBCFE9FF5E
:107BF000FB0EDBCFEAFF00C0EEFF01C0EDFFFA0E87
:107C0000DBCFE9FFFB0EDBCFEAFFEE50ED1006E124
:107C1000120EF36E020EF3CFDBFF86D0DECFE9FF4C
:107C2000DDCFEAFF1C0EE926000EEA22EF50006EBF
:107C3000016A010E001801E101502CE1E66AF80E1C
:107C4000E66E0F0EE66EFA0EDBCFE9FFFB0EDBCF22
:107C5000EAFFEECFE6FFEFCFE6FFDECFE6FFDDCFB8
:107C6000E6FF00EC57F0026E070EE15C02E2E16A0B
:107C7000E552E16E0250F3CF00F0F4CF01F00001C5
:107C8000001C01E1011C05E1080EF36E020EF3CFAA
:107C9000DBFF2AD0E66AF80EE66EE668FA0EDBCF66
:107CA000E9FFFB0EDBCFEAFFEECFE6FFEFCFE6FF0B
:107CB000DECFE6FFDDCFE6FF00EC57F0026E070EE9
:107CC000E15C02E2E16AE552E16E0250F3CF00F0BE
:107CD000F4CF01F00001001C01E1011C05E1080ED8
:107CE000F36E020EF3CFDBFF020EDBCF00F0016A72
:107CF00000BE01680050011017E1FA0EDBCFE9FF6A
:107D0000FB0EDBCFEAFFEECFE6FFEFCFE6FFDECFE5
:107D1000E6FFDDCFE6FF19D8E552E552E552E55220
:107D2000E76E020EE7CFDBFF020EDBCF00F0016A49
:107D300000BE0168005000D0E552E552E552E55220
:107D4000E5CFDAFFE7CFD9FF1200D9CFE6FFDACFD0
:107D5000E6FFE1CFD9FFE2CFDAFF060EE12402E32E
:107D6000E168E652E16E050EDB6AFA0EDBCFE6FF54
:107D7000FB0EDBCFE6FFFC0EDBCFE6FFFD0EDBCF1D
:107D8000E6FFB7D8E552E552E552E552010E50C084
:107D9000DBFF020E51C0DBFF030E52C0DBFF040EFF
:107DA00053C0DBFF0F012A51006E016A0050011021
:107DB00006E019EC44F0000902E0FF0E8CD00F0140
:107DC000246B256B2B51006E016A005001101BE1E2
:107DD000E66A020EE66EE66AFC0EDBCFE9FFFD0EF8
:107DE000DBCFEAFFEECFE6FFEFCFE6FFC7ECB3F065
:107DF000006E050EE15C02E2E16AE552E16E0050C0
:107E00000F01010E2B6FDF6ADF50026E036AFC0E5A
:107E1000DBCFE9FFFD0EDBCFEAFF1B0EE926000EEC
:107E2000EA22EF50000103AE02D0D89003D0025CEA
:107E3000000E035807E2050EDB50046E056A04507D
:107E4000051002E0000E01D0010E006E016A005024
:107E500001103EE0E66AFC0EDBCFE9FFFD0EDBCF52
:107E6000EAFFEECFE6FFEFCFE6FFD950010FE96E54
:107E7000000EDA20EA6EEFCF02F0EE2A000EEFCF0E
:107E800003F0EE22EFCF04F0EE22EFCF05F0EF2269
:107E900002C0E6FF03C0E6FF04C0E6FF05C0E6FF40
:107EA00019ECA4F0066E070EE15C02E2E16AE5520D
:107EB000E16E0650006E016A010E001801E10150EA
:107EC00005E0080EF36E050EF3CFDBFFDF2A9CD72B
:107ED000050EDB5000D0006E060EE15C02E2E16AA6
:107EE000E552E16E0050E552E5CFDAFFE7CFD9FF6A
:107EF0001200D9CFE6FFDACFE6FFE1CFD9FFE2CF1C
:107F0000DAFFE652E652E652E652D950FA0FE96E2F
:107F1000FF0EDA20EA6EEE50ED100DE0D950FA0FA8
:107F2000E96EFF0EDA20EA6E010EEE1801E1ED5067
:107F300002E0000E01D0010E006E016A0050011037
:107F400026E0FA0EDBCF00F0FB0EDBCF01F0026A79
:107F5000036AFC0EDBCFE9FFFD0EDBCFEAFF0A0E62
:107F6000E926000EEA22EE500026EE500122EE50E5
:107F70000222EE50032200C0DFFF010E01C0DBFF32
:107F8000020E02C0DBFF030E03C0DBFF5DD0FC0E60
:107F9000DBCFE9FFFD0EDBCFEAFF0E0EE926000E78
:107FA000EA22EECF0CF0EECF0DF0EECF0EF0EFCFD9
:107FB0000FF0FC0EDBCFE9FFFD0EDBCFEAFF1B0E5F
:107FC000E926000EEA22EF50086E096A0A6A0B6A77
:107FD00009AE02D00A680B68FA0EDBCF04F0FB0E84
:107FE000DBCF05F0066A076A020E045E000E055A32
:107FF000065A075A04C050F005C051F006C052F0AE
:1080000007C053F008C055F009C056F00AC057F039
:108010000BC058F058ECB5F04C5000010C24006E29
:108020004D500D20016E4E500E20026E4F500F200D
:10803000036E00C0DFFF010E01C0DBFF020E02C0B5
:10804000DBFF030E03C0DBFFDECF50F0DECF51F0CD
:10805000DECF52F0DDCF53F0DD52DD52040EE15C95
:1080600003E200D0E16AE552E16EE552E5CFDAFFC6
:10807000E7CFD9FF1200D9CFE6FFDACFE6FFE1CF95
:10808000D9FFE2CFDAFF1A0EE12402E3E168E652FB
:10809000E16EFA0EDBCF52F0FB0EDBCF53F0F80EA1
:1080A000DBCF57F0F90EDBCF58F03DECB3F050C00A
:1080B00000F051C001F0000E00C0DFFF010E01C052
:1080C000DBFF020EDB6A030EDB6AFC0EDBCF52F035
:1080D000FD0EDBCF53F0040E52C0DBFF050E53C084
:1080E000DBFF080EDB6A170EDB6A180EDB6AF60E82
:1080F000DBCFE9FFF70EDBCFEAFF120EE926000E19
:10810000EA22EF50010B006E016A0050011007E1F6
:10811000080EF36EF3CFDBFFF36AF46A7ED3D9CF98
:10812000E9FFDACFEAFFEECF00F0EECF01F0EECFBD
:1081300002F0EFCF03F0005001100210031003E132
:10814000F36AF46A6AD306ECA5F0000908E0160E9B
:10815000F36E080EF3CFDBFFF36AF46A5ED30F0110
:108160002B6BF60EDBCFE9FFF70EDBCFEAFF060E37
:10817000EECFDBFF070EEDCFDBFFF60EDBCFE9FF27
:10818000F70EDBCFEAFF080EE926000EEA22090E01
:10819000EECFDBFF0A0EEDCFDBFFF60EDBCFE9FF04
:1081A000F70EDBCFEAFF0A0EE926000EEA220F0ED9
:1081B000EECFDBFF100EEECFDBFF110EEECFDBFFBD
:1081C000120EEECFDBFFF60EDBCFE9FFF70EDBCFB3
:1081D000EAFF040EE926000EEA22EECFE6FFEFCF1B
:1081E000E6FF060EDBCFE6FF070EDBCFE6FF81DE04
:1081F000E552E552E552E5520B0E50C0DBFF0C0E86
:1082000051C0DBFF0D0E52C0DBFF0E0E53C0DBFF73
:10821000F60EDBCFE9FFF70EDBCFEAFF060EE9260D
:10822000000EEA22EECF00F0EFCF01F0026A036AFF
:10823000D9500B0FE96E000EDA20EA6E0050EE26E0
:108240000150EE220250EE220350EE2224CF00F025
:1082500025CF01F0F60EDB50001803E1F70EDB50DE
:10826000011813E00F012A51006E016A005001103D
:1082700006E0DFDA000903E0F36AF46ACED2F60E14
:10828000DBCF24FFF70EDBCF25FFD9500B0FE96EB4
:10829000000EDA20EA6E0F012651EE1809E127518F
:1082A000EE1806E12851EE1803E12951EE1800E11D
:1082B00043E02A51006E016A0050011006E0B9DA6D
:1082C000000903E0F36AF46AA8D20F012B6B060ED3
:1082D000DBCFE9FF070EDBCFEAFFEECFE6FFEFCF04
:1082E000E6FFD9500B0FE96E000EDA20EA6EEECFF2
:1082F000E6FFEECFE6FFEECFE6FFEFCFE6FF8DEC39
:10830000A1F0006E060EE15C02E2E16AE552E16E68
:108310000050000905E1070EF36E080EF3CFDBFFF6
:108320000B0EDBCF26FF0C0EDBCF27FF0D0EDBCFB6
:1083300028FF0E0EDBCF29FFF60EDBCFE9FFF70E8D
:10834000DBCFEAFF0E0EE926000EEA22130EEECF77
:10835000DBFF140EEECFDBFF150EEECFDBFF160EAC
:10836000EECFDBFF080EDBCF02F0036A02BE03682C
:10837000025003100EE1D9CFE9FFDACFEAFFD8802F
:10838000000EEE54000EEE54000EEE54000EEE54AD
:1083900002E3000E01D0010E006E016A00500110D0
:1083A00001E1E8D10F0EDBCF00F0100EDBCF01F0C2
:1083B000110EDBCF02F0120EDBCF03F0D950130FFA
:1083C000E96E000EDA20EA6E0050EE1809E1015065
:1083D000EE1806E10250EE1803E10350EE1800E13A
:1083E0000BE1F60EDBCFE9FFF70EDBCFEAFF120E53
:1083F000E926000EEA22EF82D950090FE96E000E3D
:10840000DA20EA6EEE5002E1020EED1801E039D1F9
:10841000010EF36E190EF3CFDBFF0F012A51006E30
:10842000016A0050011006E004DA000903E0F36875
:10843000F468F3D1090EDB6A0A0EDB6AF60EDBCFB5
:10844000E9FFF70EDBCFEAFF060EE926000EEA226F
:10845000EE2AEF22F60EDBCFE9FFF70EDBCFEAFFC5
:10846000060EE926000EEA22EECF00F0EFCF01F073
:10847000060EDBCFE9FF070EDBCFEAFF1B0EE92676
:10848000000EEA22EF50026E036A0250001802E169
:108490000350011843E1F60EDBCFE9FFF70EDBCF07
:1084A000EAFF060EEB6A070EEB6AF60EDBCFE9FF7A
:1084B000F70EDBCFEAFF120EE926000EEA22EF509C
:1084C000020B01E0010E006E016A0050011013E082
:1084D000E66AF60EDBCFE6FFF70EDBCFE6FFC5EC74
:1084E00027F0E552E552E552E76E080EE7CFDBFFD5
:1084F000190EDB6A13D0010EE66EE66AF60EDBCFCC
:10850000E6FFF70EDBCFE6FF1FEC0EF0E552E5527B
:10851000E552E552E76E080EE7CFDBFF080EDBCF32
:1085200000F0016A00BE0168120E001801E101505E
:1085300003E1F36AF46A71D1080EDBCF00F0016A3F
:1085400000BE01680050011001E09BD0F60EDBCFA9
:10855000E9FFF70EDBCFEAFF040EE926000EEA2260
:10856000EECFE6FFEFCFE6FF060EDBCFE6FF070E0E
:10857000DBCFE6FFBEDCE552E552E552E5520B0EDD
:1085800050C0DBFF0C0E51C0DBFF0D0E52C0DBFFF5
:108590000E0E53C0DBFFF60EDBCFE9FFF70EDBCF8D
:1085A000EAFF060EE926000EEA22EECF00F0EFCF3A
:1085B00001F0026A036AD9500B0FE96E000EDA204F
:1085C000EA6E0050EE260150EE220250EE220350D9
:1085D000EE22F60EDBCF24FFF70EDBCF25FF190EC0
:1085E000DB50006E016A005001103FE0060EDBCF49
:1085F000E9FF070EDBCFEAFFEECFE6FFEFCFE6FFA6
:10860000D9500B0FE96E000EDA20EA6EEECFE6FFCE
:10861000EECFE6FFEECFE6FFEFCFE6FF8DECA1F069
:10862000006E060EE15C02E2E16AE552E16E005086
:1086300000090EE1070EF36E080EF3CFDBFF0F010A
:108640002669276928692969F36AF46AE6D00CD09B
:108650000B0EDBCF26FF0C0EDBCF27FF0D0EDBCF83
:1086600028FF0E0EDBCF29FF0CD00B0EDBCF26FF31
:108670000C0EDBCF27FF0D0EDBCF28FF0E0EDBCF5E
:1086800029FF080EDBCF00F0016A00BE0168005030
:1086900001106FE1040EDBCFE9FF050EDBCFEAFF2F
:1086A000EFCF02F0036A02BE0368090EDBCF00F0D1
:1086B000DB2A0A0EDBCF01F001E3DB2A060EDBCF5B
:1086C000E9FF070EDBCFEAFF0050EE24E76E015012
:1086D000EE20EA6EE7CFE9FF02C0EFFF010EE76E82
:1086E000040EDBCF00F0050EDBCF01F0E7500026D3
:1086F000000E0122040E00C0DBFF050E01C0DBFFEF
:10870000D9500F0FE96E000EDA20EA6EEE2A000E45
:10871000EE22EE22EE22D9CFE9FFDACFEAFFEE0613
:10872000EE5AEE5AEE5A170EDB2A180E01E3DB2A38
:10873000F60EDBCFE9FFF70EDBCFEAFF120EE926DC
:10874000000EEA22EF50020B01E0010E006E016AFA
:10875000005001100BE0D950130FE96E000EDA2023
:10876000EA6EEE2A000EEE22EE22EE220F01010E3C
:108770002A6FF8D5F60EDBCFE9FFF70EDBCFEAFF65
:10878000080EE926000EEA22090EDBCFEEFF0A0EE4
:10879000DBCFEDFFF60EDBCFE9FFF70EDBCFEAFF15
:1087A0000A0EE926000EEA220F0EDBCFEEFF100EB6
:1087B000DBCFEEFF110EDBCFEEFF120EDBCFEEFFB5
:1087C000F60EDBCFE9FFF70EDBCFEAFF0E0EE92650
:1087D000000EEA22130EDBCFEEFF140EDBCFEEFF0E
:1087E000150EDBCFEEFF160EDBCFEEFF170EDBCF45
:1087F00052F0180EDBCF53F0FA0EDBCF57F0FB0E22
:10880000DBCF58F0E2ECB5F052C000F053C001F0FD
:1088100000C0F3FF01C0F4FF00D01A0EE15C02E2D9
:10882000E16AE552E16EE552E5CFDAFFE7CFD9FF25
:108830001200D9CFE6FFDACFE6FFE1CFD9FFE2CFD2
:10884000DAFF090EE12402E3E168E652E16E060E6A
:10885000DB6A070E24CFDBFF080E25CFDBFF070EF8
:10886000DBCFE9FF080EDBCFEAFF040EEECFDBFF24
:10887000050EEDCFDBFF070EDBCFE9FF080EDBCFE8
:10888000EAFF040EE926000EEA22EECFE6FFEFCF64
:10889000E6FF040EDBCFE6FF050EDBCFE6FF79EC4B
:1088A0003FF0E552E552E552E55250C0DEFF51C0BF
:1088B000DEFF52C0DEFF53C0DDFFDD52DD52070E8A
:1088C000DBCFE9FF080EDBCFEAFF060EE926000E3C
:1088D000EA22EECF00F0EFCF01F0026A036A005007
:1088E000DE260150DE220250DE220350DD22DD5260
:1088F000DD52E66A040EDBCFE9FF050EDBCFEAFFAF
:10890000EECFE6FFEFCFE6FFD9CFE9FFDACFEAFF00
:10891000EECFE6FFEECFE6FFEECFE6FFEFCFE6FFCE
:1089200019ECA4F0006E070EE15C02E2E16AE55288
:10893000E16E0050000907E1080EF36E060EF3CF5A
:10894000DBFFFF0E04D00F012A6B000E00D0006E7B
:10895000090EE15C02E2E16AE552E16E0050E55287
:10896000E5CFDAFFE7CFD9FF1200D9CFE6FFDACFA4
:10897000E6FFE1CFD9FFE2CFDAFFFC0EDBCFE9FF64
:10898000FD0EDBCFEAFF0A0EE926000EEA22EECF4B
:1089900002F0EECF03F0EECF04F0EFCF05F0FC0EC7
:1089A000DBCFE9FFFD0EDBCFEAFF0E0EE926000E5E
:1089B000EA220250EE1809E10350EE1806E10450D5
:1089C000EE1803E10550EE1800E102E0000E01D0C0
:1089D000010E006E016A00C0F3FF01C0F4FF00D079
:1089E000E552E5CFDAFFE7CFD9FF1200D9CFE6FF96
:1089F000DACFE6FFE1CFD9FFE2CFDAFF150EE124AF
:108A000002E3E168E652E16EFA0EDBCF52F0FB0EB4
:108A1000DBCF53F0F80EDBCF57F0F90EDBCF58F079
:108A20003DECB3F050C000F051C001F0000E00C0AA
:108A3000DFFF010E01C0DBFF020EDB6A030EDB6A03
:108A4000FC0EDBCF52F0FD0EDBCF53F0040E52C014
:108A5000DBFF050E53C0DBFF120EDB6A130EDB6A71
:108A6000140EDB6AF60EDBCFE9FFF70EDBCFEAFF71
:108A7000060EEECFDBFF070EEDCFDBFFF60EDBCFF2
:108A8000E9FFF70EDBCFEAFF080EE926000EEA2227
:108A9000100EEECFDBFF110EEDCFDBFFF60EDBCFBE
:108AA000E9FFF70EDBCFEAFF0A0EE926000EEA2205
:108AB000080EEECFDBFF090EEECFDBFF0A0EEECF86
:108AC000DBFF0B0EEECFDBFFF60EDBCFE9FFF70E81
:108AD000DBCFEAFF120EE926000EEA22EF50010B6F
:108AE000006E016A0050011003E0F36AF46A4FD28D
:108AF0000F012A51006E016A0050011006E099DE54
:108B0000000903E0F368F46842D224CF02F025CFD5
:108B100003F0F60EDB50021803E1F70EDB500318EA
:108B20000BE0D950100FE96E000EDA20EA6EEE501D
:108B300002E1020EED1802E1000E01D0010E006EFE
:108B4000016A0050011001E184D0F60EDBCF24FF52
:108B5000F70EDBCF25FFF60EDBCFE9FFF70EDBCFFD
:108B6000EAFF040EE926000EEA22EECFE6FFEFCF81
:108B7000E6FF060EDBCFE6FF070EDBCFE6FF79EC64
:108B80003FF0E552E552E552E5520C0E50C0DBFFD6
:108B90000D0E51C0DBFF0E0E52C0DBFF0F0E53C097
:108BA000DBFFF60EDBCFE9FFF70EDBCFEAFF060EA9
:108BB000E926000EEA22EECF00F0EFCF01F0026AC4
:108BC000036AD9500C0FE96E000EDA20EA6E0050ED
:108BD000EE260150EE220250EE220350EE220F014B
:108BE0002B6B060EDBCFE9FF070EDBCFEAFFEECFE4
:108BF000E6FFEFCFE6FFD9500C0FE96E000EDA204A
:108C0000EA6EEECFE6FFEECFE6FFEECFE6FFEFCF68
:108C1000E6FF8DECA1F0006E060EE15C02E2E16A77
:108C2000E552E16E0050000908E1070EF36E120EE6
:108C3000F3CFDBFFF36AF46AAAD10C0EDBCF26FF79
:108C40000D0EDBCF27FF0E0EDBCF28FF0F0EDBCF85
:108C500029FFD9CFE9FFDACFEAFFEECF00F0EECF60
:108C600001F0EECF02F0EFCF03F000500110021040
:108C7000031001E14FD1080EDBCF00F0090EDBCF6E
:108C800001F00A0EDBCF02F00B0EDBCF03F0F60E85
:108C9000DBCFE9FFF70EDBCFEAFF0E0EE926000E71
:108CA000EA220050EE1809E10150EE1806E10250E8
:108CB000EE1803E10350EE1800E106E13D0EF36EFD
:108CC000120EF3CFDBFF26D1D950100FE96E000E44
:108CD000DA20EA6EEE5002E1020EED1801E0D9D082
:108CE000100EDB6A110EDB6AF60EDBCFE9FFF70E22
:108CF000DBCFEAFF060EE926000EEA22EE2AEF227B
:108D0000F60EDBCFE9FFF70EDBCFEAFF060EE92612
:108D1000000EEA22EECF00F0EFCF01F0060EDBCF1F
:108D2000E9FF070EDBCFEAFF1B0EE926000EEA2261
:108D3000EF50026E036A0250001802E1035001185E
:108D400026E1F60EDBCFE9FFF70EDBCFEAFF060EDA
:108D5000EB6A070EEB6A010EE66EE66AF60EDBCFF3
:108D6000E6FFF70EDBCFE6FF1FEC0EF0E552E55213
:108D7000E552E552E76E120EE7CFDBFFDBCF00F0E6
:108D8000016A00BE01680050011001E0C3D0F60E78
:108D9000DBCFE9FFF70EDBCFEAFF040EE926000E7A
:108DA000EA22EECFE6FFEFCFE6FF060EDBCFE6FFCF
:108DB000070EDBCFE6FF79EC3FF0E552E552E552D6
:108DC000E5520C0E50C0DBFF0D0E51C0DBFF0E0E46
:108DD00052C0DBFF0F0E53C0DBFFF60EDBCFE9FF07
:108DE000F70EDBCFEAFF060EE926000EEA22EECFF1
:108DF00000F0EFCF01F0026A036AD9500C0FE96E60
:108E0000000EDA20EA6E0050EE260150EE220250EB
:108E1000EE220350EE22F60EDBCF24FFF70EDBCF5F
:108E200025FF0F012B6B060EDBCFE9FF070EDBCF13
:108E3000EAFFEECFE6FFEFCFE6FFD9500C0FE96E69
:108E4000000EDA20EA6EEECFE6FFEECFE6FFEECFC1
:108E5000E6FFEFCFE6FF8DECA1F0006E060EE15CC1
:108E600002E2E16AE552E16E0050000906E1070EF8
:108E7000F36E120EF3CFDBFF4DD00C0EDBCF26FFCF
:108E80000D0EDBCF27FF0E0EDBCF28FF0F0EDBCF43
:108E900029FF100EDBCF00F0DB2A110EDBCF01F033
:108EA00001E3DB2A060EDBCFE9FF070EDBCFEAFF8B
:108EB0000050EE24E76E0150EE20EA6EE7CFE9FFA6
:108EC000EF50E66E040EDBCFE9FF050EDBCFEAFFC5
:108ED000E552E750EF6E040EDB2A050E01E3DB2AB4
:108EE000D950080FE96E000EDA20EA6EEE2A000E65
:108EF000EE22EE22EE22130EDB2A140E01E3DB2A11
:108F0000D9CFE9FFDACFEAFFEE06000EEE5AEE5AAD
:108F1000EE5A9FD6F60EDBCFE9FFF70EDBCFEAFF66
:108F2000080EE926000EEA22100EDBCFEEFF110E2E
:108F3000DBCFEDFFF60EDBCFE9FFF70EDBCFEAFF6D
:108F40000A0EE926000EEA22080EDBCFEEFF090E1C
:108F5000DBCFEEFF0A0EDBCFEEFF0B0EDBCFEEFF1B
:108F6000130EDBCF52F0140EDBCF53F0FA0EDBCF33
:108F700057F0FB0EDBCF58F0E2ECB5F052C000F03A
:108F800053C001F000C0F3FF01C0F4FF00D0150E84
:108F9000E15C02E2E16AE552E16EE552E5CFDAFF1B
:108FA000E7CFD9FF1200D9CFE6FFDACFE6FFE1CF56
:108FB000D9FFE2CFDAFF140EE12402E3E168E652C2
:108FC000E16E130EDB6ADB50006E016AD89001502F
:108FD00004E60B0E005C000E015812E2130EDB508B
:108FE000E76EFA0EDBCFE9FFFB0EDBCFEAFFE750BF
:108FF000E926000EEA22200EEF6E130EDB2AE3D7DD
:10900000FC0EDBCFE9FFFD0EDBCFEAFFEFCF02F076
:10901000036A02BE03682E0E021801E1035010E03D
:10902000FC0EDBCFE9FFFD0EDBCFEAFFEFCF04F054
:10903000056A04BE05680450051002E0000E01D068
:10904000010E006E016A0050011002E0000E2ED1E8
:10905000FC0EDBCFE6FFFD0EDBCFE6FF16ECB4F037
:10906000E552E552020EF3CFDBFF030EF4CFDBFF38
:10907000D950020FE96E000EDA20EA6E0C0ED8808D
:10908000EE54000EED5425E3FC0EDBCFE6FFFD0EA3
:10909000DBCFE6FFD950040FE66E000EDA20E66E55
:1090A000F5ECB3F0E552E552E552E552F90EDB502E
:1090B000E66EE66AD950040FE66E000EDA20E66E20
:1090C00003D9E552E552E552E552000904E1000EEC
:1090D000EDD0000EEBD02E0EE66ED950040FE66EEA
:1090E000000EDA20E66EE1ECB3F0E552E552E5520F
:1090F000F3CFDEFFF4CFDDFFDECF00F0DDCF01F0F8
:10910000005001101DE0DECFE9FFDDCFEAFFEF6A7E
:10911000DF2A010E01E3DB2ADECFE6FFDDCFE6FF2B
:1091200016ECB4F0E552E552F3CF00F0F4CF01F0C5
:10913000030ED8800054000E015402E2000EB6D097
:10914000D950040FE66E000EDA20E66E16ECB4F08D
:10915000E552E552F3CF00F0F4CF01F0080ED880CD
:109160000054000E015402E2000EA0D0130EDB6A80
:10917000DBCF00F000C0E6FFD950040FE66E000E12
:10918000DA20E66E16ECB4F0E552E552E552E7CF90
:1091900000F0F3CF01F0F4CF02F00150005C000EBC
:1091A000025425E2D950040F026E000EDA20036E3D
:1091B000130EDB500F010224E96E000E0320EA6E4D
:1091C000EFCF00F0016A00BE0168130EDB50E76EBE
:1091D000FA0EDBCFE9FFFB0EDBCFEAFFE750E92613
:1091E000000EEA2200C0EFFF130EDB2AC1D7D9CF51
:1091F000E9FFDACFEAFFEE50ED100CE0DECFE9FF39
:10920000DDCFEAFFEFCF02F0036A02BE036802502F
:10921000031002E1000E01D0010E006E016A005041
:10922000011042E0130EDB6ADBCF00F000C0E6FF66
:10923000DECFE6FFDDCFE6FF16ECB4F0E552E552F7
:10924000E552E7CF00F0F3CF01F0F4CF02F0015088
:10925000005C000E025428E2130EDB50E76E000E95
:10926000DFCFE9FF010EDBCFEAFFE750E926000E72
:10927000EA22EFCF00F0016A00BE0168130EDB5056
:10928000E76EFA0EDBCFE9FFFB0EDBCFEAFFE7501C
:10929000E926000EEA22080EE926000EEA2200C0A6
:1092A000EFFF130EDB2AC0D7010E00D0006E140EA4
:1092B000E15C02E2E16AE552E16E0050E552E5CF81
:1092C000DAFFE7CFD9FF1200D9CFE6FFDACFE6FF0A
:1092D000E1CFD9FFE2CFDAFFE652E652E652E6529C
:1092E000FC0EDBCFE6FFFD0EDBCFE6FF16ECB4F0A5
:1092F000E552E552F3CFDEFFF4CFDDFF020EDB6A6D
:10930000030EDB6A020EDBCF00F0030EDBCF01F0B1
:10931000DECF02F0DDCF03F001500318E8AE02D03B
:10932000033404D00250005C0350015801E3E7D03D
:10933000FB0EDB50006E016A0050011064E1FA0E72
:10934000DB50E66E020EDBCF04F0030EDBCF05F040
:10935000FC0EDB500424E96EFD0EDB500520EA6EA6
:10936000EFCF02F0036A02BE03680250E66ED7D860
:10937000E552E552006E016A020E001801E101504B
:109380003FE0030E001801E101503AE0010E001821
:1093900001E1015006E0005001E1015001E000D080
:1093A00031D0020EDBCF04F0030EDBCF05F0FC0E54
:1093B000DB500424E96EFD0EDB500520EA6EEFCF92
:1093C00002F0036A02BE036802C0E6FF03C0E6FFC4
:1093D00044ECB5F0E552E552F350E66E020EDBCFF9
:1093E00000F0030EDBCF01F0FC0EDB500024E96E31
:1093F000FD0EDB500120EA6EE552E750EF6E02D021
:10940000000E7FD076D0FB0EDB50006E016A010E9D
:10941000001801E101506DE1FA0EDB50E66E020E1C
:10942000DBCF04F0030EDBCF05F0FC0EDB50042491
:10943000E96EFD0EDB500520EA6EEFCF02F0036A05
:1094400002BE03680250E66E30DAE552E552006E65
:10945000016A020E001801E101504AE0010E0018F5
:1094600001E1015016E0005001E1015001E041D05E
:10947000020EDBCF00F0030EDBCF01F0FC0EDB5061
:109480000024E96EFD0EDB500120EA6E5F0EEF6EE8
:1094900030D0020EDBCF04F0030EDBCF05F0FC0E64
:1094A000DB500424E96EFD0EDB500520EA6EEFCFA1
:1094B00002F0036A02BE036802C0E6FF03C0E6FFD3
:1094C00044ECB5F0E552E552F350E66E020EDBCF08
:1094D00000F0030EDBCF01F0FC0EDB500024E96E40
:1094E000FD0EDB500120EA6EE552E750EF6E01D031
:1094F00000D0020EDB2A030E01E3DB2A03D7010EA4
:1095000000D0006E040EE15C02E2E16AE552E16E19
:109510000050E552E5CFDAFFE7CFD9FF1200D9CFEF
:10952000E6FFDACFE6FFE1CFD9FFE2CFDAFFFD0EAB
:10953000DBCF22F0236A22BE2368D890235004E6B2
:10954000410E225C000E23580DE3FD0EDBCF24F00C
:10955000256A24BE2568253404E224505A08000EEA
:10956000255402E2000E01D0010E206E216A205027
:10957000211025E1FD0EDBCF28F0296A28BE2968DD
:10958000D890295004E6300E285C000E29580DE3CF
:10959000FD0EDBCF2AF02B6A2ABE2B682B3404E2A7
:1095A0002A503908000E2B5402E2000E01D0010EA1
:1095B000266E276A2650271002E1000E01D0010E08
:1095C0001E6E1F6A1E501F100DE1FD0EDBCF2CF02A
:1095D0002D6A2CBE2D68240E2C1801E12D5002E0BE
:1095E000000E01D0010E1C6E1D6A1C501D100DE1F5
:1095F000FD0EDBCF2EF02F6A2EBE2F68250E2E1803
:1096000001E12F5002E0000E01D0010E1A6E1B6A1C
:109610001A501B100DE1FD0EDBCF30F0316A30BE69
:109620003168270E301801E1315002E0000E01D000
:10963000010E186E196A185019100DE1FD0EDBCFDE
:1096400032F0336A32BE33682D0E321801E13350E6
:1096500002E0000E01D0010E166E176A16501710A8
:109660000DE1FD0EDBCF34F0356A34BE35685F0E98
:10967000341801E1355002E0000E01D0010E146EE5
:10968000156A145015100DE1FD0EDBCF36F0376A68
:1096900036BE3768400E361801E1375002E0000E42
:1096A00001D0010E126E136A125013100DE1FD0E5F
:1096B000DBCF38F0396A38BE39687E0E381801E1E0
:1096C000395002E0000E01D0010E106E116A1050E8
:1096D00011100DE1FD0EDBCF3AF03B6A3ABE3B685C
:1096E000600E3A1801E13B5002E0000E01D0010E7D
:1096F0000E6E0F6A0E500F100DE1FD0EDBCF3CF029
:109700003D6A3CBE3D68210E3C1801E13D5002E03F
:10971000000E01D0010E0C6E0D6A0C500D100DE103
:10972000FD0EDBCF3EF03F6A3EBE3F68280E3E187E
:1097300001E13F5002E0000E01D0010E0A6E0B6AFB
:109740000A500B100DE1FD0EDBCF40F0416A40BE28
:109750004168290E401801E1415002E0000E01D09D
:10976000010E086E096A085009100DE1FD0EDBCFED
:1097700042F0436A42BE43685E0E421801E1435024
:1097800002E0000E01D0010E066E076A06500710B7
:109790000DE1FD0EDBCF44F0456A44BE4568230E63
:1097A000441801E1455002E0000E01D0010E046EA4
:1097B000056A045005100DE1FD0EDBCF46F0476A47
:1097C00046BE4768260E461801E1475002E0000EEB
:1097D00001D0010E026E036A025003100DE1FD0E6E
:1097E000DBCF48F0496A48BE49682E0E481801E1AF
:1097F000495002E0000E01D0010E006E016A0050D7
:10980000011003E0000E4BD04AD0FD0EDBCF02F07A
:10981000036A02BE0368D890035004E6610E025C3E
:10982000000E03580DE3FD0EDBCF04F0056A04BE05
:109830000568053404E204507A08000E055402E27B
:10984000000E01D0010E006E016A0050011003E00D
:10985000010E25D024D0FC0EDB50006E016A0050B2
:1098600001100DE0FD0EDBCF00F0016A00BE0168C3
:109870002A0E001801E1015002E1000E10D0FD0E89
:10988000DBCF00F0016A00BE0168200E001801E184
:10989000015003E1030E03D002D0020E00D0E552C6
:1098A000E5CFDAFFE7CFD9FF1200D9CFE6FFDACF55
:1098B000E6FFE1CFD9FFE2CFDAFFFC0EDB50006E0E
:1098C000016A005001100BE0FD0EDB50006E016AD2
:1098D0002A0E001801E1015002E1020E67D1FD0ECF
:1098E000DB50246E256AD890255004E6200E245CB7
:1098F000000E255809E2FD0EDB50266E276A050E84
:10990000261801E1275002E1000E01D0010E226E5F
:10991000236A225023100BE1FD0EDB50286E296ACA
:10992000220E281801E1295002E0000E01D0010E9C
:10993000206E216A205021100BE1FD0EDB502A6EB3
:109940002B6A2A0E2A1801E12B5002E0000E01D0EA
:10995000010E1E6E1F6A1E501F100BE1FD0EDB5024
:109960002C6E2D6A2B0E2C1801E12D5002E0000EFA
:1099700001D0010E1C6E1D6A1C501D100BE1FD0E66
:10998000DB502E6E2F6A2C0E2E1801E12F5002E0B4
:10999000000E01D0010E1A6E1B6A1A501B100BE14B
:1099A000FD0EDB50306E316A2E0E301801E1315061
:1099B00002E0000E01D0010E186E196A185019103D
:1099C0000BE1FD0EDB50326E336A2F0E321801E1CF
:1099D000335002E0000E01D0010E166E176A1650C9
:1099E00017100BE1FD0EDB50346E356A3A0E341859
:1099F00001E1355002E0000E01D0010E146E156A2F
:109A0000145015100BE1FD0EDB50366E376A3B0E1D
:109A1000361801E1375002E0000E01D0010E126E3F
:109A2000136A125013100BE1FD0EDB50386E396AC9
:109A30003C0E381801E1395002E0000E01D0010E51
:109A4000106E116A105011100BE1FD0EDB503A6ED2
:109A50003B6A3D0E3A1801E13B5002E0000E01D096
:109A6000010E0E6E0F6A0E500F100BE1FD0EDB5053
:109A70003C6E3D6A3E0E3C1801E13D5002E0000E96
:109A800001D0010E0C6E0D6A0C500D100BE1FD0E95
:109A9000DB503E6E3F6A3F0E3E1801E13F5002E050
:109AA000000E01D0010E0A6E0B6A0A500B100BE17A
:109AB000FD0EDB50406E416A5B0E401801E14150E3
:109AC00002E0000E01D0010E086E096A085009106C
:109AD0000BE1FD0EDB50426E436A5C0E421801E161
:109AE000435002E0000E01D0010E066E076A0650D8
:109AF00007100BE1FD0EDB50446E456A5D0E441805
:109B000001E1455002E0000E01D0010E046E056A2D
:109B1000045005100BE1FD0EDB50466E476A7C0ECB
:109B2000461801E1475002E0000E01D0010E026E1E
:109B3000036A025003100DE1FD0EDB50486E496AC6
:109B4000493404E248507F08000E495402E3000EF5
:109B500001D0010E006E016A0050011003E0000EFA
:109B600025D024D0FD0EDB50026E036AD89003503E
:109B700004E6610E025C000E03580BE3FD0EDB50A1
:109B8000046E056A053404E204507A08000E055498
:109B900002E2000E01D0010E006E016A00500110B9
:109BA00003E0010E03D002D0020E00D0E552E5CF53
:109BB000DAFFE7CFD9FF1200D9CFE6FFDACFE6FF11
:109BC000E1CFD9FFE2CFDAFF0B0EE12402E3E16837
:109BD000E652E16EFC0EDBCFE9FFFD0EDBCFEAFFC4
:109BE000080EEECFDBFF090EEDCFDBFFF60EDBCF6D
:109BF00052F0F70EDBCF53F0525001E153505BE0CF
:109C0000020E521801E1535027E0010E521801E1F3
:109C1000535001E050D0FC0EDBCFE9FFFD0EDBCF4F
:109C2000EAFF0A0EE926000EEA22EECF00F0EECFA0
:109C300001F0EECF02F0EFCF03F0D950F80FE96E4C
:109C4000FF0EDA20EA6E0050EE260150EE2202509E
:109C5000EE220350EE2230D0F80EDBCF04F0F90EE6
:109C6000DBCF05F0FA0EDBCF06F0FB0EDBCF07F003
:109C7000FC0EDBCFE9FFFD0EDBCFEAFF0E0EE9267F
:109C8000000EEA220450EE5C006E0550EE58016EA4
:109C90000650EE58026E0750EE58036EF80E00C0E4
:109CA000DBFFF90E01C0DBFFFA0E02C0DBFFFB0E8B
:109CB00003C0DBFF01D000D00F012A51006E016A02
:109CC0000050011007E019EC44F0000903E0F368CC
:109CD000F4681BD3FC0EDBCFE9FFFD0EDBCFEAFF00
:109CE000020EE926000EEA22EECF00F0EFCF01F0DF
:109CF000040E00C0DBFF050E01C0DBFF060EDB6AB1
:109D0000070EDB6AFC0EDBCFE9FFFD0EDBCFEAFFBF
:109D1000040EE926000EEA22040EDBCFEEFF050E4C
:109D2000DBCFEDFFFC0EDBCFE9FFFD0EDBCFEAFF63
:109D30000E0EE926000EEA22040EEECFDBFF050E22
:109D4000EECFDBFF060EEECFDBFF070EEECFDBFF25
:109D5000040EDBCF00F0050EDBCF01F0060EDBCFEB
:109D600002F0070EDBCF03F0D950F80FE96EFF0EBB
:109D7000DA20EA6EEE50005CEE500158EE500258C8
:109D8000EE50035804E2F368F468BFD2BBD2FC0E75
:109D9000DBCFE9FFFD0EDBCFEAFF120EE926000E56
:109DA000EA22EF92FC0EDBCFE9FFFD0EDBCFEAFFEC
:109DB0000A0EE926000EEA22F80EDBCFEEFFF90EBE
:109DC000DBCFEEFFFA0EDBCFEEFFFB0EDBCFEEFFBD
:109DD000F80EDBCF50F0F90EDBCF51F0FA0EDBCFEF
:109DE00052F0FB0EDBCF53F0556A020E566E576AE7
:109DF000586ADCECB2F050C0DEFF51C0DEFF52C04A
:109E0000DEFF53C0DDFFDD52DD52D9CFE9FFDACFEF
:109E1000EAFFEECF04F0EECF05F0EECF06F0EFCF85
:109E200007F0090ED8900436053606360736E806E0
:109E3000F9E1D950F80FE96EFF0EDA20EA6E04500E
:109E4000EE5C006E0550EE58016E0650EE58026E44
:109E50000750EE58036EF80E00C0DBFFF90E01C08C
:109E6000DBFFFA0E02C0DBFFFB0E03C0DBFFFC0EC4
:109E7000DBCFE9FFFD0EDBCFEAFF080EE926000E7F
:109E8000EA22F80EDBCFEEFFF90EDBCFEDFF080E76
:109E9000DBCFE9FF090EDBCFEAFF1B0EE926000E40
:109EA000EA22EF50006E016A026A036A01AE02D034
:109EB0000268036800C055F001C056F002C057F0B8
:109EC00003C058F0DFCF50F0010EDBCF51F0020E8F
:109ED000DBCF52F0030EDBCF53F0BEECB5F0040E37
:109EE00050C0DBFF050E51C0DBFF060E52C0DBFF8A
:109EF000070E53C0DBFFD9CFE9FFDACFEAFFEECF81
:109F000004F0EECF05F0EECF06F0EFCF07F0080E2D
:109F1000DBCFE9FF090EDBCFEAFF1B0EE926000EBF
:109F2000EA22EF50086E096A0A6A0B6A09AE02D08B
:109F30000A680B6808C050F009C051F00AC052F01E
:109F40000BC053F0040EDBCF55F0050EDBCF56F0FF
:109F5000060EDBCF57F0070EDBCF58F058ECB5F00C
:109F60004C50045C006E4D500558016E4E50065822
:109F7000026E4F500758036E00C0DFFF010E01C094
:109F8000DBFF020E02C0DBFF030E03C0DBFFFC0E93
:109F9000DBCFE9FFFD0EDBCFEAFF060EE926000E60
:109FA000EA22DFCFEEFF010EDBCFEDFFD950040F29
:109FB000E96E000EDA20EA6ED880000EEE54000E34
:109FC000EE54000EEE54000EEE5401E316D1040ED2
:109FD000DBCFE6FF050EDBCFE6FFFC0EDBCFE6FFB7
:109FE000FD0EDBCFE6FF1FEC0EF0E552E552E55229
:109FF000E552E76E0A0EE7CFDBFFDB50006E016A29
:10A000000050011001E1F9D00A0EDB50006E016A28
:10A010003C0E001801E1015001E0ECD0FC0EDBCF5A
:10A02000E9FFFD0EDBCFEAFF120EE926000EEA2261
:10A03000EF50010B006E016A0050011065E0FC0E4C
:10A04000DBCFE9FFFD0EDBCFEAFF020EE926000EB3
:10A05000EA22EECF00F0EFCF01F0FC0EDBCFE9FFFC
:10A06000FD0EDBCFEAFF040EE926000EEA2200C057
:10A07000EEFF01C0EDFFD950040FE96E000EDA20AB
:10A08000EA6E010EEE1805E1EE5003E1EE5001E13B
:10A09000EE5025E0040EDBCF00F0050EDBCF01F023
:10A0A000060EDBCF02F0070EDBCF03F00006000E3A
:10A0B000015A025A035A00C0E6FF01C0E6FFFC0E37
:10A0C000DBCFE6FFFD0EDBCFE6FF1FEC0EF0E55227
:10A0D000E552E552E552E76E0A0EE7CFDBFFE66A8E
:10A0E000FC0EDBCFE6FFFD0EDBCFE6FFC5EC27F075
:10A0F000E552E552E552006E016A0050011003E09E
:10A10000F368F46802D175D0FC0EDBCFE9FFFD0ED9
:10A11000DBCFEAFF020EE926000EEA22EECF00F0C6
:10A12000EFCF01F0FC0EDBCFE9FFFD0EDBCFEAFF46
:10A13000040EE926000EEA2200C0EEFF01C0EDFF8A
:10A14000040EDBCF00F0050EDBCF01F0060EDBCFF7
:10A1500002F0070EDBCF03F00006000E015A025A90
:10A16000035A00C0E6FF01C0E6FFFC0EDBCFE6FFAE
:10A17000FD0EDBCFE6FF1FEC0EF0E552E552E55297
:10A18000E552E76E0A0EE7CFDBFFDB50006E016A97
:10A190000050011003E0F368F468B7D0FC0EDBCF89
:10A1A000E9FFFD0EDBCFEAFF080EE926000EEA22EA
:10A1B000EE6A020EED6E080EDBCFE9FF090EDBCF73
:10A1C000EAFF1B0EE926000EEA22EF50006E016A3C
:10A1D0000006000E015AFC0EDBCFE9FFFD0EDBCFBF
:10A1E000EAFF060EE926000EEA2200C0EEFF01C0DB
:10A1F000EDFF03D0F368F46888D0FC0EDBCFE9FFF5
:10A20000FD0EDBCFEAFF040EE926000EEA22EECFB8
:10A21000E6FFEFCFE6FF080EDBCFE6FF090EDBCF50
:10A22000E6FF79EC3FF0E552E552E552E552040EC7
:10A2300050C0DBFF050E51C0DBFF060E52C0DBFF36
:10A24000070E53C0DBFFFC0EDBCFE9FFFD0EDBCFBB
:10A25000EAFF060EE926000EEA22EECF00F0EFCF6D
:10A2600001F000C0DFFF010E01C0DBFF020EDB6A60
:10A27000030EDB6AD950040FE96E000EDA20EA6E95
:10A28000DF50EE26010EDB50EE22020EDB50EE22F6
:10A29000030EDB50EE220F01246B256B2B6B080E97
:10A2A000DBCFE9FF090EDBCFEAFFEECFE6FFEFCF12
:10A2B000E6FFD950040FE96E000EDA20EA6EEECF09
:10A2C000E6FFEECFE6FFEECFE6FFEFCFE6FF8DEC49
:10A2D000A1F0006E060EE15C02E2E16AE552E16E79
:10A2E0000050000903E1F368F4680FD0040EDBCFDF
:10A2F00026FF050EDBCF27FF060EDBCF28FF070E5C
:10A30000DBCF29FFF36AF46A00D00B0EE15C02E2B6
:10A31000E16AE552E16EE552E5CFDAFFE7CFD9FF1A
:10A320001200D9CFE6FFDACFE6FFE1CFD9FFE2CFC7
:10A33000DAFF0E0EE12402E3E168E652E16E0D0E53
:10A34000DB6ADB50006E016AD890015004E60D0E06
:10A35000005C000E015831E20D0EDB50046E056A00
:10A36000066A05BE0668D950FB0FE96EFF0EDA20BB
:10A37000EA6EEE500424F36EEE500520F46EEE50BB
:10A380000620F86EF4CFF7FFF3CFF6FF0800F5CF05
:10A3900002F0036A02BE0368D9CF00F0DACF01F001
:10A3A0000D0EDB500F010024E96E000E0120EA6E55
:10A3B00002C0EFFF0D0EDB2AC4D7F90EDBCFE6FF9C
:10A3C000FA0EDBCFE6FFD9CFE6FFDACFE6FF04ECEB
:10A3D00031F0E552E552E552E5520E0EE15C03E242
:10A3E00000D0E16AE552E16EE552E5CFDAFFE7CF52
:10A3F000D9FF1200D9CFE6FFDACFE6FFE1CFD9FFD0
:10A40000E2CFDAFF100EE12402E3E168E652E16EEA
:10A410000F0EDB6ADB50006E016AD890015004E633
:10A420000D0E005C000E015831E20F0EDB50046E81
:10A43000056A066A05BE0668D950FB0FE96EFF0E75
:10A44000DA20EA6EEE500424F36EEE500520F46E2E
:10A45000EE500620F86EF4CFF7FFF3CFF6FF0800BA
:10A46000F5CF02F0036A02BE0368D9CF00F0DACF5D
:10A4700001F00F0EDB500F010024E96E000E0120E9
:10A48000EA6E02C0EFFF0F0EDB2AC4D70F0EDB6AA5
:10A49000DB50006E016AD890015004E6020E005CA9
:10A4A000000E015833E20F0EDB50046E056A066A97
:10A4B00005BE0668D950F80FE96EFF0EDA20EA6E85
:10A4C000EE500424F36EEE500520F46EEE5006209C
:10A4D000F86EF4CFF7FFF3CFF6FF0800F5CF02F0E8
:10A4E000036A02BE0368D9500D0F006E000EDA2019
:10A4F000016E0F0EDB500F010024E96E000E0120EB
:10A50000EA6E02C0EFFF0F0EDB2AC2D7D9500D0F43
:10A51000E66E000EDA20E66ED9CFE6FFDACFE6FF70
:10A52000E4EC37F0E552E552E552E552100EE15CFD
:10A5300003E200D0E16AE552E16EE552E5CFDAFFD1
:10A54000E7CFD9FF1200D9CFE6FFDACFE6FFE1CFA0
:10A55000D9FFE2CFDAFF0E0EE12402E3E168E65212
:10A56000E16EFB0EDBCFF6FFFC0EDBCFF7FFFD0E3F
:10A57000DBCFF8FF0800F5CF00F0016A00BE0168EC
:10A580000D0EDB6A0D0EDB50006E016A0D0E005CD5
:10A59000000E015815E20900F550E66ED9CF00F023
:10A5A000DACF01F00D0EDB500F010024E96E000E32
:10A5B0000120EA6EE552E750EF6E0D0EDB2AE2D77E
:10A5C000D9CFE6FFDACFE6FFE8EC3BF0E552E55203
:10A5D00000D00E0EE15C02E2E16AE552E16EE55266
:10A5E000E5CFDAFFE7CFD9FF1200D9CFE6FFDACF08
:10A5F000E6FFE1CFD9FFE2CFDAFF0E0EE12402E35E
:10A60000E168E652E16EFB0EDBCFF6FFFC0EDBCF1E
:10A61000F7FFFD0EDBCFF8FF0800F5CF00F0016A71
:10A6200000BE01680D0EDB6A0D0EDB50006E016A84
:10A630000D0E005C000E015815E20900F550E66EA3
:10A64000D9CF00F0DACF01F00D0EDB500F0100245E
:10A65000E96E000E0120EA6EE552E750EF6E0D0E36
:10A66000DB2AE2D7F70EDBCFE6FFF80EDBCFE6FF03
:10A67000F90EDBCFE6FFFA0EDBCFE6FFD9CFE6FF20
:10A68000DACFE6FF58EC7CF0006E060EE15C02E2E9
:10A69000E16AE552E16E005000D00E0EE15C02E28C
:10A6A000E16AE552E16EE552E5CFDAFFE7CFD9FF87
:10A6B0001200D9CFE6FFDACFE6FFE1CFD9FFE2CF34
:10A6C000DAFF0D0EE12402E3E168E652E16EFC0ED2
:10A6D000DBCFE9FFFD0EDBCFEAFF1C0EE926000E03
:10A6E000EA22EF50026E036A020E021801E10350E3
:10A6F00012E0FC0EDBCFE9FFFD0EDBCFEAFF1C0E04
:10A70000E926000EEA22EF50046E056A010E0418D5
:10A7100001E1055002E1000E01D0010E006E016A58
:10A720000050011003E0F368F4685ED30F012B6B57
:10A73000FC0EDBCFE9FFFD0EDBCFEAFF1C0EE926A6
:10A74000000EEA22EF50006E016A020E001801E1CD
:10A7500001501BE1FA0EDBCF50F0FB0EDBCF51F0C6
:10A76000526A536A020E556E566A576A586A58EC16
:10A77000B5F0010E4CC0DBFF020E4DC0DBFF030E37
:10A780004EC0DBFF040E4FC0DBFFFC0EDBCFE9FF4A
:10A79000FD0EDBCFEAFF1C0EE926000EEA22EF5089
:10A7A000006E016A010E001801E101503EE1FA0E4F
:10A7B000DBCF50F0FB0EDBCF51F0526A536A030E31
:10A7C000556E566A576A586A58ECB5F0010E4CC07F
:10A7D000DBFF020E4DC0DBFF030E4EC0DBFF040E9D
:10A7E0004FC0DBFF010E006E016A026A036AD95096
:10A7F000010FE96E000EDA20EA6EEE500016EE5000
:10A800000116EE500216EE5003160050DF6ED950BE
:10A81000010FE96E000EDA20EA6ED890030EEB32DB
:10A82000020EEB32010EEB32EF32010EDBCF00F005
:10A83000020EDBCF01F0030EDBCF02F0040EDBCF04
:10A8400003F0090ED8900332023201320032E806DA
:10A85000F9E1FC0EDBCFE9FFFD0EDBCFEAFF060ED0
:10A86000E926000EEA22EE500026EE500122EE50BC
:10A870000222EE500322050E00C0DBFF060E01C0CF
:10A88000DBFF070E02C0DBFF080E03C0DBFFD95061
:10A89000010FE96E000EDA20EA6EEE52010EEE169E
:10A8A000EE6AEE6AD950050FE96E000EDA20EA6E04
:10A8B0000F011F51EE1809E12051EE1806E1215158
:10A8C000EE1803E12251EE1800E101E04BD1FC0E3D
:10A8D000DBCFE9FFFD0EDBCFEAFF1C0EE926000E01
:10A8E000EA22EF50006E016A020E001801E10150E9
:10A8F00011E1010EDBCFE9FF020EDBCFEAFF000E14
:10A90000E9260A0EEA22090EEECFDBFF0A0EEDCF92
:10A91000DBFF27D1FC0EDBCFE9FFFD0EDBCFEAFF2B
:10A920001C0EE926000EEA22EF50006E016A010EAD
:10A93000001801E1015001E014D1010EDBCFE9FF65
:10A94000020EDBCFEAFF000EE9260A0EEA22EF50E4
:10A95000E66ED950090FE96E000EDA20EA6EE55274
:10A96000E750EE6EED6ADF50006E016A0050011094
:10A970000FE0D950090FE96E000EDA20EA6E040EDE
:10A980000F0B06E0EC52D890ED32EF32E806FAE118
:10A99000010EDBCF00F0020EDBCF01F0030EDBCFA8
:10A9A00002F0040EDBCF03F0002A000E0122022287
:10A9B0000322010E0116026A036A00C0DBFF020EC9
:10A9C00001C0DBFF030E02C0DBFF040E03C0DBFF90
:10A9D000010EDBCF00F0020EDBCF01F0030EDBCF68
:10A9E00002F0040EDBCF03F0005001100210031040
:10A9F0006DE10F012351006E016A0050011020E04B
:10AA0000010EE66E000EE66EE66AE66EE66AFC0E83
:10AA1000DBCFE6FFFD0EDBCFE6FFF2D9026E070EBD
:10AA2000E15C02E2E16AE552E16E0250F3CF00F030
:10AA3000F4CF01F00050011003E0F368F468D4D1C2
:10AA4000000EE66E0A0EE66E010E006E016A026AE4
:10AA5000036AD950050FE96E000EDA20EA6EEE5057
:10AA60000026EE500122EE500222EE50032200C0DA
:10AA7000E6FF01C0E6FF02C0E6FF03C0E6FF8DEC83
:10AA8000A1F0046E060EE15C02E2E16AE552E16EBD
:10AA90000450000909E10F011F692069216B226B35
:10AAA000F368F468A1D112D0050EDBCF1FFF060EAC
:10AAB000DBCF20FF070EDBCF21FF080EDBCF22FF0D
:10AAC0000F011F2B000E202321232223010EDBCF99
:10AAD000E9FF020EDBCFEAFF000EE9260A0EEA22AA
:10AAE000EF50E66ED9500B0FE96E000EDA20EA6ED9
:10AAF000E552E750EE6EED6ADF50006E016A0050DD
:10AB0000011017E00B0EDBCF00F00C0EDBCF01F0D5
:10AB1000040ED89000360136E804FBE1D950090F45
:10AB2000E96E000EDA20EA6E0050EE260150ED22AA
:10AB300018D00F0EE76E0B0EDBCF00F00C0EDBCF44
:10AB400001F0E7500016016A00C001F0006AD95018
:10AB5000090FE96E000EDA20EA6E0050EE26015071
:10AB6000ED2225D12351006E016A0050011020E032
:10AB7000010EE66E000EE66EE66AE66EE66AFC0E12
:10AB8000DBCFE6FFFD0EDBCFE6FF3AD9026E070E04
:10AB9000E15C02E2E16AE552E16E0250F3CF00F0BF
:10ABA000F4CF01F00050011003E0F368F4681CD109
:10ABB000000EE66E0A0EE66ED950050FE96E000E25
:10ABC000DA20EA6EEECFE6FFEECFE6FFEECFE6FF4D
:10ABD000EFCFE6FF8DECA1F0006E060EE15C02E225
:10ABE000E16AE552E16E0050000909E10F011F69B9
:10ABF0002069216B226BF368F468F6D0D8D0050E7B
:10AC0000DBCF1FFF060EDBCF20FF070EDBCF21FFC0
:10AC1000080EDBCF22FFFC0EDBCFE9FFFD0EDBCF02
:10AC2000EAFF1C0EE926000EEA22EF50006E016AD0
:10AC3000020E001801E1015011E1010EDBCFE9FF26
:10AC4000020EDBCFEAFF000EE9260A0EEA22090E09
:10AC5000EECFDBFF0A0EEDCFDBFFA9D0FC0EDBCF82
:10AC6000E9FFFD0EDBCFEAFF1C0EE926000EEA220B
:10AC7000EF50006E016A010E001801E1015001E081
:10AC800096D0010EDBCFE9FF020EDBCFEAFF000E0C
:10AC9000E9260A0EEA22EF50E66ED950090FE96E56
:10ACA000000EDA20EA6EE552E750EE6EED6ADF50F4
:10ACB000006E016A005001100FE0D950090FE96ED3
:10ACC000000EDA20EA6E040E0F0B06E0EC52D8906C
:10ACD000ED32EF32E806FAE1010EDBCF00F0020EB2
:10ACE000DBCF01F0030EDBCF02F0040EDBCF03F06D
:10ACF000002A000E012202220322010E0116026A1E
:10AD0000036A00C0DBFF020E01C0DBFF030E02C0BE
:10AD1000DBFF040E03C0DBFF010EDBCFE9FF020EF9
:10AD2000DBCFEAFF000EE9260A0EEA22EF50E66EBC
:10AD3000D9500B0FE96E000EDA20EA6EE552E750AB
:10AD4000EE6EED6ADF50006E016A0050011017E0F0
:10AD50000B0EDBCF00F00C0EDBCF01F0040ED89011
:10AD600000360136E804FBE1D950090FE96E000E08
:10AD7000DA20EA6E0050EE260150ED2218D00F0EB8
:10AD8000E76E0B0EDBCF00F00C0EDBCF01F0E750CF
:10AD90000016016A00C001F0006AD950090FE96E7F
:10ADA000000EDA20EA6E0050EE260150ED22090E68
:10ADB000DBCF00F00A0EDBCF01F0F80E005CFF0ED7
:10ADC000015807E3F80EF36E090EF3CFDBFF0A0E0E
:10ADD000DB68090EDBCF00F00A0EDBCF01F000C00C
:10ADE000F3FF01C0F4FF00D00D0EE15C02E2E16A66
:10ADF000E552E16EE552E5CFDAFFE7CFD9FF120069
:10AE0000D9CFE6FFDACFE6FFE1CFD9FFE2CFDAFF15
:10AE10000F0EE12402E3E168E652E16EFC0EDBCFA7
:10AE2000E9FFFD0EDBCFEAFF1C0EE926000EEA2249
:10AE3000EF50026E036A020E021801E1035012E0A5
:10AE4000FC0EDBCFE9FFFD0EDBCFEAFF1C0EE9268F
:10AE5000000EEA22EF50046E056A010E041801E1AB
:10AE6000055002E1000E01D0010E006E016A005093
:10AE7000011003E0F368F468A3D30F012B6BF70E06
:10AE8000DB50006E016A0050011065E0DF6A070EBA
:10AE90001FCFDBFF080E20CFDBFF090E21CFDBFF2A
:10AEA0000A0E22CFDBFFDF50006E016AFC0EDBCF03
:10AEB000E9FFFD0EDBCFEAFF1A0EE926000EEA22BB
:10AEC000EF50000101AE02D0D89003D0005C000E1C
:10AED00001583CE2E66A000EE66E0A0EE66E1FCFEF
:10AEE000E6FF20CFE6FF21CFE6FF22CFE6FF19ECF9
:10AEF000A4F0006E070EE15C02E2E16AE552E16E49
:10AF00000050000903E1F368F4685AD3DF2AFC0E0D
:10AF1000DBCFE9FFFD0EDBCFEAFF180EE926000EBE
:10AF2000EA22EECF00F0EFCF01F0026A036AD950B7
:10AF3000070FE96E000EDA20EA6E0050EE2601508F
:10AF4000EE220250EE220350EE22ADD70F01236B0A
:10AF5000F36AF46A35D3FC0EDBCFE9FFFD0EDBCFDD
:10AF6000EAFF1C0EE926000EEA22EF50006E016A8D
:10AF7000020E001801E1015059E1FA0EDBCF50F04A
:10AF8000FB0EDBCF51F0526A536A020E556E566AC1
:10AF9000576A586A58ECB5F0030E4CC0DBFF040E3C
:10AFA0004DC0DBFF050E4EC0DBFF060E4FC0DBFFC2
:10AFB000030EDBCF00F0040EDBCF01F0050EDBCF7C
:10AFC00002F0060EDBCF03F0090ED89003320232F6
:10AFD00001320032E806F9E1FC0EDBCFE9FFFD0E9D
:10AFE000DBCFEAFF060EE926000EEA22EE5000262D
:10AFF000EE500122EE500222EE5003220B0E00C052
:10B00000DBFF0C0E01C0DBFF0D0E02C0DBFF0E0EDE
:10B0100003C0DBFFD950030FE96E000EDA20EA6EA1
:10B02000EE52010EEE16EE6AEE6A8FD0FC0EDBCF0A
:10B03000E9FFFD0EDBCFEAFF1C0EE926000EEA2237
:10B04000EF50006E016A010E001801E1015001E0AD
:10B050007CD0FA0EDBCF50F0FB0EDBCF51F0526A02
:10B06000536A030E556E566A576A586A58ECB5F023
:10B07000030E4CC0DBFF040E4DC0DBFF050E4EC0BF
:10B08000DBFF060E4FC0DBFF010E006E016A026A95
:10B09000036AD950030FE96E000EDA20EA6EEE5013
:10B0A0000016EE500116EE500216EE500316010E79
:10B0B00000C0DBFFD950030FE96E000EDA20EA6E04
:10B0C000D890030EEB32020EEB32010EEB32EF3270
:10B0D000030EDBCF00F0040EDBCF01F0050EDBCF5B
:10B0E00002F0060EDBCF03F0090ED89003320232D5
:10B0F00001320032E806F9E1FC0EDBCFE9FFFD0E7C
:10B10000DBCFEAFF060EE926000EEA22EE5000260B
:10B11000EE500122EE500222EE5003220B0E00C030
:10B12000DBFF0C0E01C0DBFF0D0E02C0DBFF0E0EBD
:10B1300003C0DBFFD950030FE96E000EDA20EA6E80
:10B14000EE52010EEE16EE6AEE6AD9500B0FE96E62
:10B15000000EDA20EA6E0F011F51EE1809E12051AE
:10B16000EE1806E12151EE1803E12251EE1800E13C
:10B1700001E19BD02351006E016A0050011062E092
:10B18000DF6A070E1FCFDBFF080E20CFDBFF090EA3
:10B1900021CFDBFF0A0E22CFDBFFDF50006E016AFA
:10B1A000FC0EDBCFE9FFFD0EDBCFEAFF1A0EE9262E
:10B1B000000EEA22EF50000101AE02D0D89003D079
:10B1C000005C000E01583CE2E66A000EE66E0A0ED4
:10B1D000E66E1FCFE6FF20CFE6FF21CFE6FF22CFAE
:10B1E000E6FF19ECA4F0006E070EE15C02E2E16AF2
:10B1F000E552E16E0050000903E1F368F468E0D124
:10B20000DF2AFC0EDBCFE9FFFD0EDBCFEAFF180ED5
:10B21000E926000EEA22EECF00F0EFCF01F0026A3D
:10B22000036AD950070FE96E000EDA20EA6E00506B
:10B23000EE260150EE220250EE220350EE22ADD750
:10B240000F01236B000EE66E0A0EE66ED9500B0F4F
:10B25000E96E000EDA20EA6EEECFE6FFEECFE6FFF3
:10B26000EECFE6FFEFCFE6FF8DECA1F0006E060E0D
:10B27000E15C02E2E16AE552E16E0050000909E199
:10B280000F011F692069216B226BF368F46898D164
:10B290000CD00B0EDBCF1FFF0C0EDBCF20FF0D0EF3
:10B2A000DBCF21FF0E0EDBCF22FFFC0EDBCFE9FF51
:10B2B000FD0EDBCFEAFF1C0EE926000EEA22EF505E
:10B2C000006E016A020E001801E1015025E1030E33
:10B2D000DBCFE9FF040EDBCFEAFF000EE9260A0E02
:10B2E000EA22F80EDBCFEFFFDBCF00F0F90EDBCF69
:10B2F00001F001C000F0016A030EDBCFE9FF040E8C
:10B30000DBCFEAFF000EE9260A0EEA22010EE9264B
:10B31000000EEA2200C0EFFFFC0EDBCFE9FFFD0EBE
:10B32000DBCFEAFF1C0EE926000EEA22EF50006E8A
:10B33000016A010E001801E1015001E03BD1030E4A
:10B34000DBCFE9FF040EDBCFEAFF000EE9260A0E91
:10B35000EA22EF50E76E020EE7CFDBFF010EDB5073
:10B36000006E016A0050011020E00F0EE76EF80E2B
:10B37000DBCF00F0F90EDBCF01F0E7500016016AD9
:10B38000040ED89000360136E804FBE1020EDB50D3
:10B39000026E036A0F0E0216000E03160050021012
:10B3A000E76E020EE7CFDBFF0ED0FF0EE76EF80E62
:10B3B000DBCF00F0F90EDBCF01F0E7500016016A99
:10B3C000020E00C0DBFFDB50E66E030EDBCFE9FFB1
:10B3D000040EDBCFEAFF000EE9260A0EEA22E55250
:10B3E000E750EF6E030EDBCF00F0040EDBCF01F071
:10B3F000050EDBCF02F0060EDBCF03F0002A000EB5
:10B40000012202220322010E0116026A036A030EC0
:10B4100000C0DBFF040E01C0DBFF050E02C0DBFF36
:10B42000060E03C0DBFF030EDBCF00F0040EDBCF04
:10B4300001F0050EDBCF02F0060EDBCF03F000506B
:10B4400001100210031066E1010EE66E000EE66EBA
:10B45000E66AE66EE66AFC0EDBCFE6FFFD0EDBCFAA
:10B46000E6FFCEDC026E070EE15C02E2E16AE55225
:10B47000E16E0250F3CF00F0F4CF01F00050011064
:10B4800003E0F368F4689CD0000EE66E0A0EE66EE8
:10B49000010E006E016A026A036AD9500B0FE96E51
:10B4A000000EDA20EA6EEE500026EE500122EE5039
:10B4B0000222EE50032200C0E6FF01C0E6FF02C0F8
:10B4C000E6FF03C0E6FF8DECA1F0046E060EE15C22
:10B4D00002E2E16AE552E16E0450000909E10F0160
:10B4E0001F692069216B226BF368F46869D012D060
:10B4F0000B0EDBCF1FFF0C0EDBCF20FF0D0EDBCFC3
:10B5000021FF0E0EDBCF22FF0F011F2B000E202389
:10B5100021232223030EDBCFE9FF040EDBCFEAFF5A
:10B52000000EE9260A0EEA22EF50E76E020EE7CF80
:10B53000DBFF010EDB50006E016A0050011010E0CD
:10B54000F80EDBCF00F0F90EDBCF01F0040ED8903F
:10B5500001320032E804FBE1020E00C0DBFF1BD029
:10B56000F80EDBCF00F0F90EDBCF01F001C000F0E8
:10B57000016A0F0E0016000E0116020EDB50026E5D
:10B58000036AF00E0216000E031600500210E76E5A
:10B59000020EE7CFDBFFDB50E66E030EDBCFE9FFE9
:10B5A000040EDBCFEAFF000EE9260A0EEA22E5527E
:10B5B000E750EF6E0F01010E236FF36AF46A00D0BB
:10B5C0000F0EE15C02E2E16AE552E16EE552E5CF81
:10B5D000DAFFE7CFD9FF1200D9CFE6FFDACFE6FFD7
:10B5E000E1CFD9FFE2CFDAFFE66AE66AE66AFC0E4F
:10B5F000DBCFE6FFFD0EDBCFE6FFE66A35D8006E57
:10B60000060EE15C02E2E16AE552E16E005000D014
:10B61000E552E5CFDAFFE7CFD9FF1200D9CFE6FF39
:10B62000DACFE6FFE1CFD9FFE2CFDAFFFB0EDBCFC7
:10B63000E6FFFC0EDBCFE6FFFD0EDBCFE6FF000EE4
:10B64000E66EE66A010EE66E0FD8006E060EE15C4D
:10B6500002E2E16AE552E16E005000D0E552E5CF2A
:10B66000DAFFE7CFD9FF1200D9CFE6FFDACFE6FF46
:10B67000E1CFD9FFE2CFDAFF700EE12402E3E16807
:10B68000E652E16E010EF36E020EF3CFDBFF030E06
:10B69000DB6AFB0EDBCF52F0FC0EDBCF53F0060E65
:10B6A00052C0DBFF070E53C0DBFFD950F80FE96E25
:10B6B000FF0EDA20EA6E080EEECFDBFF090EEECFAA
:10B6C000DBFF0A0EEECFDBFFD950160F006E000E27
:10B6D000DA20016E6E0E00C0DBFF6F0E01C0DBFFD3
:10B6E0002CCFE6FF2DCFE6FF6E0EDBCFE6FF6F0E11
:10B6F000DBCFE6FF6DEC3DF0E552E552E552E55259
:10B70000FD0EDB50006E016A0050011012E0080EC1
:10B71000DBCFF6FF090EDBCFF7FF0A0EDBCFF8FF1A
:10B720000800F5CF00F0016A00BE01680050DF6E2E
:10B730000DD0060EDBCFE9FF070EDBCFEAFFEFCF20
:10B7400000F0016A00BE01680050DF6EDF50006E3D
:10B75000016A0050011004E1F368F468ACEF61F095
:10B76000DF50006E016A5C0E001801E1015001E13A
:10B77000A1D22E0E001801E101500BE0010EDB6A90
:10B78000FD0EDB50006E016A0050011001E1BAD3DA
:10B7900066D3FD0EDB50006E016A005001101CE004
:10B7A000D950080FE96E000EDA20EA6EEE2A000E7C
:10B7B000EE22EE22080EDBCFF6FF090EDBCFF7FFFD
:10B7C0000A0EDBCFF8FF0800F5CF00F0016A00BEDB
:10B7D00001680050DF6E12D0060EDB2A070E01E36F
:10B7E000DB2A060EDBCFE9FF070EDBCFEAFFEFCF48
:10B7F00000F0016A00BE01680050DF6EDF50006E8D
:10B80000016A2E0E001801E1015001E0D5D1FD0EB4
:10B81000DB50006E016A005001101CE0D950080F87
:10B82000E96E000EDA20EA6EEE2A000EEE22EE221B
:10B83000080EDBCFF6FF090EDBCFF7FF0A0EDBCFDA
:10B84000F8FF0800F5CF00F0016A00BE0168005063
:10B85000DF6E12D0060EDB2A070E01E3DB2A060E8E
:10B86000DBCFE9FF070EDBCFEAFFEFCF00F0016A85
:10B8700000BE01680050DF6E6E0EDBCFE9FF6F0E79
:10B88000DBCFEAFF280EE926000EEA22EE50ED108B
:10B8900005E1F368F468ACEF61F08DD16E0EDBCF9B
:10B8A000E9FF6F0EDBCFEAFF280EE926000EEA2241
:10B8B000EECF00F0EFCF01F06E0EDBCFE9FF6F0EA1
:10B8C000DBCFEAFF2A0EE926000EEA2200C0EEFFD7
:10B8D00001C0EDFF010EF36E020EF3CFDBFF030E8E
:10B8E000DB6A010EE66ED950020FE66E000EDA201A
:10B8F000E66E6E0EDBCFE6FF6F0EDBCFE6FFA0EC51
:10B9000020F0006E050EE15C02E2E16AE552E16EB4
:10B910000050040EF3CFDBFF050EF4CFDBFFD95050
:10B92000040FE96E000EDA20EA6EEE50ED1004E12D
:10B93000F368F468ACEF61F0040EDBCFE9FF050EAD
:10B94000DBCFEAFF1A0EE926000EEA22EECF00F066
:10B95000EFCF01F06E0EDBCFE9FF6F0EDBCFEAFF1A
:10B96000280EE926000EEA2200C0EEFF01C0EDFF1E
:10B970006E0EDBCFE9FF6F0EDBCFEAFF280EE92664
:10B98000000EEA22EECF00F0EFCF01F06E0EDBCF1B
:10B99000E9FF6F0EDBCFEAFF2A0EE926000EEA224E
:10B9A00000C0EEFF01C0EDFF6E0EDBCFE9FF6F0EB2
:10B9B000DBCFEAFF280EE926000EEA22EE50ED105A
:10B9C00036E16E0EDBCFE9FF6F0EDBCFEAFF170E1D
:10B9D000E926000EEA225C0EEF6EDE52010EDD6EED
:10B9E000DB50006E016AD890015004E60B0E005C3B
:10B9F000000E01581BE26E0EDBCFE9FF6F0EDBCFAE
:10BA0000EAFF170EE926000EEA22E9CF00F0EACF9E
:10BA100001F0010EDB500F010024E96E000E012041
:10BA2000EA6E200EEF6E010EDB2ADAD746D06E0EDC
:10BA3000DBCFE9FF6F0EDBCFEAFF170EE926000E22
:10BA4000EA222E0EEF6E6E0EDBCFE9FF6F0EDBCF1C
:10BA5000EAFF170EE926000EEA22010EE926000E83
:10BA6000EA222E0EEF6EDE52020EDD6E010EDB506C
:10BA7000006E016AD890015004E60B0E005C000EC7
:10BA800001581BE26E0EDBCFE9FF6F0EDBCFEAFF42
:10BA9000170EE926000EEA22E9CF00F0EACF01F006
:10BAA000010EDB500F010024E96E000E0120EA6E4A
:10BAB000200EEF6E010EDB2AD9D7020EDB6A030ED1
:10BAC000DB6A010EE66ED950020FE66E000EDA2038
:10BAD000E66E6E0EDBCFE6FF6F0EDBCFE6FFA0EC6F
:10BAE00020F0026E050EE15C02E2E16AE552E16ED1
:10BAF0000250F3CF00F0F4CF01F00050011004E148
:10BB0000F368F468ACEF61F0DF50006E016A5C0E20
:10BB1000001801E1015036E1FD0EDB50006E016AB4
:10BB2000005001101CE0D950080FE96E000EDA2019
:10BB3000EA6EEE2A000EEE22EE22080EDBCFF6FFB2
:10BB4000090EDBCFF7FF0A0EDBCFF8FF0800F5CFB9
:10BB500000F0016A00BE01680050DF6E12D0060ED0
:10BB6000DB2A070E01E3DB2A060EDBCFE9FF070E17
:10BB7000DBCFEAFFEFCF00F0016A00BE01680050A2
:10BB8000DF6EC2D7DF50006E016A0050011013E172
:10BB90006E0EDBCFE6FF6F0EDBCFE6FF2CCFE6FFAE
:10BBA0002DCFE6FF6DEC3DF0E552E552E552E55252
:10BBB000F36AF46AD1D37DD0DF50006E016A005081
:10BBC000011014E16E0EDBCFE6FF6F0EDBCFE6FF58
:10BBD0002CCFE6FF2DCFE6FF6DEC3DF0E552E552B0
:10BBE000E552E552F36AF46AB7D363D0DF50006ED2
:10BBF000016A5C0E001801E1015058E1DF50006E4F
:10BC0000016A5C0E001801E1015036E1FD0EDB50C7
:10BC1000006E016A005001101CE0D950080FE96E57
:10BC2000000EDA20EA6EEE2A000EEE22EE22080E58
:10BC3000DBCFF6FF090EDBCFF7FF0A0EDBCFF8FFF5
:10BC40000800F5CF00F0016A00BE01680050DF6E09
:10BC500012D0060EDB2A070E01E3DB2A060EDBCF2D
:10BC6000E9FF070EDBCFEAFFEFCF00F0016A00BE6D
:10BC700001680050DF6EC2D7DF50006E016A0050CD
:10BC8000011013E16E0EDBCFE6FF6F0EDBCFE6FF98
:10BC90002CCFE6FF2DCFE6FF6DEC3DF0E552E552EF
:10BCA000E552E552F36AF46A57D303D0F368F468B7
:10BCB00053D350D3FD0EDB50006E016A00500110CB
:10BCC0001CE0D950080FE96E000EDA20EA6EEE2A69
:10BCD000000EEE22EE22080EDBCFF6FF090EDBCFC0
:10BCE000F7FF0A0EDBCFF8FF0800F5CF00F0016A7E
:10BCF00000BE01680050DF6E12D0060EDB2A070E70
:10BD000001E3DB2A060EDBCFE9FF070EDBCFEAFFFC
:10BD1000EFCF00F0016A00BE01680050DF6EDF5017
:10BD2000006E016A5C0E001801E1015003E1F36846
:10BD3000F46812D3DF50006E016A0050011045E133
:10BD40002CCFE9FF2DCFEAFF280EEB6A290EEB6A14
:10BD50002CCFE9FF2DCFEAFF2A0EEB6A2B0EEB6A00
:10BD60002CCFE9FF2DCFEAFF170EE926000EEA22BD
:10BD70005C0EEF6EDE52010EDD6EDB50006E016A6E
:10BD8000D890015004E60B0E005C000E015819E239
:10BD90002CCFE9FF2DCFEAFF170EE926000EEA228D
:10BDA000E9CF00F0EACF01F0010EDB500F010024D3
:10BDB000E96E000E0120EA6E200EEF6E010EDB2A06
:10BDC000DCD7F36AF46AC8D249D06E0EDBCFE9FF44
:10BDD0006F0EDBCFEAFF280EEB6A290EEB6A6E0EC0
:10BDE000DBCFE9FF6F0EDBCFEAFF2A0EEB6A2B0EEB
:10BDF000EB6A6E0EDBCFE9FF6F0EDBCFEAFF170EAB
:10BE0000E926000EEA225C0EEF6EDE52010EDD6EB8
:10BE1000DB50006E016AD890015004E60B0E005C06
:10BE2000000E01581BE26E0EDBCFE9FF6F0EDBCF79
:10BE3000EAFF170EE926000EEA22E9CF00F0EACF6A
:10BE400001F0010EDB500F010024E96E000E01200D
:10BE5000EA6E200EEF6E010EDB2ADAD77BD2DF50BE
:10BE6000046E056A0450051008E0DF50066E076A8C
:10BE70005C0E061801E1075002E1000E01D0010E30
:10BE8000026E036A025003100CE0010EDB50086ED4
:10BE9000096AD890095004E60B0E085C000E095898
:10BEA00002E3000E01D0010E006E016A0050011085
:10BEB00028E0DF50E66E010EDBCFF3FFDB2AF35004
:10BEC000EA6ADC0FE96E020EEA22E552E750EF6EF5
:10BED000D950080FE96E000EDA20EA6EEF2AEECF95
:10BEE000F6FF000EEF22EECFF7FFEF22EECFF8FFC6
:10BEF0000800F5CF00F0016A00BE01680050DF6E57
